:100000000C94AC080C94DD080C94DD080C94DD080D
:100010000C94DD080C94DD080C94DD080C94DD08CC
:100020000C94DD080C94DD080C94DD080C94DD08BC
:100030000C94DD080C94DD080C94DD080C94784ACF
:100040000C94DD080C94DD080C94DD080C94DD089C
:100050000C94DD080C94DD080C94DD080C945B62B4
:100060000C94DD080C940E5C0C94E45B0C94DD089D
:100070000C94DD080C94DD080C94DD080C94DD086C
:100080000C94DD080C94DD080C94DD080C94DD085C
:100090000C94D45C0C94445C0C948B5C0C94904B4E
:1000A0000C94DD080C94DD080C94DD080C94DD083C
:1000B0000C94DD080C94DD080C94DD080C94DD082C
:1000C0000C94DD080C94DD080C94DD080C94AE5BF8
:1000D0000C94845B0C94DD080C94DD080C94DD0812
:1000E0000C94DD085C0A150A220A5C0A5C0A6A0A9A
:1000F000770A560A5C0A5C0A850D8A0D8F0D990DE8
:10010000A30D1C0EAD0DB50DBD0DC70DD10DDB0D35
:10011000EA0DF40D1C0EFE0D080E120E171009103C
:100120000910171017101B1029102910171017107D
:100130002215FD143D153D153D153D153D153D158B
:100140003D153D153D158C115B147C14751466141A
:100150003D153D153D153D153D153D153D1511153B
:10016000141B081B081B141B141BEF1AFC1AFC1A87
:10017000141B141B25291229122925292529252973
:100180003029302925292529E933EC3304341B345F
:10019000643477349734223A223A223A223A1F3A88
:1001A0001F3A263A263A263A263A263A263A263A56
:1001B000263A1F3A1F3A263A263A263A263A263A4D
:1001C000243A223A3B61376137613B613B613B61D5
:1001D000446105613B613B619E61A16190619461F5
:1001E0009A61D861A561A961AF61B361B761BD6171
:1001F000C161C561D861CB61CF61D361076342360C
:10020000B79BD8A71A39685618AEBAAB558C1D3CA7
:10021000B7CC5763BD6DEDFD753EF6177231BF006B
:100220000000803F08000000BE922449123EABAAA5
:10023000AA2ABECDCCCC4C3E00000080BEABAAAA00
:10024000AA3E00000000BF000000803F0000000048
:1002500000084178D3BB4387D1133D190E3CC3BD81
:100260004282AD2B3E68EC8276BED98FE1A93E4C2E
:1002700080EFFFBE01C4FF7F3F00000000000C9430
:10028000D6320C94F6420C942A320C9471310C94B0
:10029000A1610C948F0D0C94990D0C94BD0D0C94D0
:1002A000C64D0C941B340C94D6470C94CC590C942A
:1002B0001B100C94574E0C94C5610C94CF610C9498
:1002C0008E310C94B7610C94D8610C94235A0C9421
:1002D000E6320C94255A0C9444610C94AF610C9452
:1002E00094610C94220A0C9404340C942B430C94C7
:1002F000AA480C94B4490C940C590C94F40D0C9429
:10030000325E0C9429100C94850D0C94081B0C94EF
:100310001C0E0C9425290C9417430C94D3610C9457
:100320003B610C947C140C94C70D0C943F480C94C6
:10033000FD140C94C44F0C94B5480C94FE0D0C9411
:10034000B9320C94D10D0C94ED480C941B590C94BB
:10035000B24F0C943D150C9403470C9423320C942B
:10036000464F0C94FA420C9433330C9464340C943E
:1003700011150C94560A0C941A2E0C94CB610C9403
:100380009D480C9429490C941B1F0C942F590C94D4
:1003900005610C9409100C94DF080C94FE420C9437
:1003A000223A0C94C21B0C94F6520C94120E0C942C
:1003B00015460C9437610C945C0A0C9477340C94B9
:1003C0007F590C94BE310C9462310C94C6480C9445
:1003D0000E430C949E610C946A5A0C94D72A0C9488
:1003E000C1610C94A9610C94A8320C94770A0C9406
:1003F00022150C94EF350C94E2580C94365E0C9454
:10040000D8440C943D590C94B3610C94E9310C948C
:10041000FB310C94E0420C946A0A0C94A30D0C94EA
:100420005D460C943A4E0C943D480C94EC330C947D
:10043000335E0C94141B0C94EA0D0C949A610C948A
:1004400034460C94D6460C948C110C94485A0C9457
:1004500012290C9407490C94150A0C94A0480C948A
:10046000243A0C9417100C942E5E0C94E9330C94DF
:1004700075140C94DF2A0C946C4E0C941D480C944B
:1004800022430C94B0310C94E6430C94BD610C945F
:10049000DF420C94314E0C945B140C94EF1A0C94C4
:1004A000DB0D0C94CA440C94ED6A0C94FC1A0C9469
:1004B00071430C94AD0D0C94263A0C9490610C94FD
:1004C000084F0C9467470C9497340C94A3480C94F1
:1004D00058310C94080E0C942A430C9433480C9415
:1004E000B50D0C94E9480C948A0D0C94A5610C94FC
:1004F00066140C947D450C941F3A0C94DB2A0C94E2
:1005000030296364696E6F70737578585B003D00C5
:100510005643230020636D643D003D0056435F68F1
:1005200065617423003D0050696E3A003D005069DA
:100530006E3A002048616C7465640A003D005265A3
:1005400073746F7265643A20003A204E6F207374A2
:100550006F7265642076616C756573202D2064650B
:100560006661756C740A00466F726365205768692E
:1005700074650A00416C7265616479204163746935
:1005800076650A005475726E696E6720584F4E0A80
:1005900000584F464620736B69707065642E20507A
:1005A00072657620636D643A005475726E656420DE
:1005B0006F66662066726F6D3A00526573746F7273
:1005C00065642066726F6D3A003E20003C0020504A
:1005D00061723D200020436D643D00205375623DF3
:1005E00000204974656D3D0052414D3D00476F74D8
:1005F00020495020616464726573733A0027697002
:10060000205B69705B2C646E735B2C67775B2C736B
:1006100075626E65745D5D5D5D27202D2073657468
:10062000207374617469632049500A004661696CE3
:10063000656420746F20636F6E66696775726520EC
:1006400045746865726E6574207573696E672044C1
:100650004843502E20596F752063616E2073657476
:10066000206970206D616E75616C6C792100537426
:10067000617274696E67206C616E00246E6F6465D0
:10068000730024666F726D61740024646174617418
:1006900079706500302D31303000696E74656765A2
:1006A000720068737600636F6C6F72004F4E2C4F50
:1006B00046462C48414C542C524553542C584F4ECE
:1006C0002C584F46462C544F47474C4500656E7595
:1006D0006D00666C6F617400322E312E300024681C
:1006E0006F6D696500757074696D652C66726565FE
:1006F0006865617000326332363537375F323031CA
:10070000392D30342D3037004C6967687448756274
:100710002000246E616D650072656164790020744B
:10072000727920616761696E20696E20352073657A
:10073000636F6E6473006661696C65642C2072631C
:100740003D004177616974696E6720666F7220723F
:10075000657461696E656420746F706963730063AA
:100760006F6E6E65637465642061732000202E2EA9
:100770002E0020757365723A003A000A4174746560
:100780006D7074696E67204D51545420636F6E6EA6
:10079000656374696F6E20746F20002473746174D4
:1007A0006500646973636F6E6E656374656400559C
:1007B00073696E67204D5154542070617373776F65
:1007C00072642066726F6D20636F6E6669670044A5
:1007D0006576696365204E616D653A0052656269B0
:1007E0006E6420737563636573732E2049502061B6
:1007F0006464726573733A004572726F723A207264
:100800006562696E64206661696C0052656E657729
:10081000656420737563636573732E20495020618E
:100820006464726573733A004572726F723A207233
:10083000656E65776564206661696C004E6F206C3B
:10084000696E6B00416363657074696E6720636FE6
:100850006D6D616E64732E2E2E0A003E3E3E004E7C
:100860006F204D414320636F6E66696775726564E2
:100870003A20736574206669726D776172652773BB
:10088000204D41430A004D6F6462757320706F6C98
:100890006C696E67206572726F723D002D0020508A
:1008A000492056616C203A004D6F64627573207068
:1008B0006F6C6C696E67206572726F723D002D00FF
:1008C00020464D2056616C203A004D6F646275736E
:1008D00020706F6C6C696E67206572726F723D007C
:1008E0002056616C3A20004D423A20004E6F742031
:1008F000737570706F7274656420726567207479A7
:1009000070650A00496C6C6567616C20617267757F
:100910006D656E74730A00757074696D650066723A
:1009200065656865617000247374617473002000EC
:1009300020000A52414D3D00202D7461726765749C
:10094000207A6F6E652D00204F464600204F4E00E6
:10095000204F46460020636D643A00204375723A8A
:1009600000205365743A0020457870697265640A06
:10097000002F00496E3A20003D00494E3A00726750
:100980006200637376006865617400766F6C007056
:100990006F77657200736574706F696E74006D6F48
:1009A00064650074656D700073657400536574430D
:1009B0006D643A002056616C3D002053746F72657F
:1009C0002000444543524541534500494E4352455A
:1009D0004153450066616C7365007472756500581B
:1009E0004F464600584F4E0048414C5400544F4724
:1009F000474C450052455354004F4646004F4E0069
:100A00005265747279696E6720434D440A004E6FD7
:100A10007420737570706F727465642072656720DE
:100A2000747970650A00293A0028543A003D3E0066
:100A30004D6F64627573206F70206661696C6564C8
:100A40000A00636F756C64206E6F7420706172733E
:100A5000653A2000557064617465640A002B002DAE
:100A600000485454502F312E31202569002048541D
:100A700054502F312E310D0A486F73743A2025736C
:100A80000D0A4163636570743A202A2F2A0D0A43C8
:100A90006F6E6E656374696F6E3A20636C6F736519
:100AA0000D0A0025730020000D0A00474554002060
:100AB00074727920616761696E20696E20352073D8
:100AC00065636F6E64730A006661696C65642074A7
:100AD0006F20636F6E6E656374004552524F523AD9
:100AE000205365727665722072657475726E6564E6
:100AF0002000446F6E652E0A004170706C79696E3B
:100B0000672E0A00436F6E666967207061727369B1
:100B10006E67206661696C65640A00676F742043C4
:100B20006F6E6669670A00436F6E6669672055528B
:100B3000493A20687474703A2F2F006C617A796892
:100B40006F6D652E7275000A282D29524553544148
:100B500052545F4C414E5F4F4E5F4D5154545F4570
:100B600052524F5253000A282D29484152445245AF
:100B70005345542C207573696E6720736F6674003B
:100B80000A282D29434F554E544552000A282D2935
:100B9000444854000A282D294F57495245000A2835
:100BA0002B294D4F44425553000A282B29444D58B8
:100BB000000A282B294453323438322D313030008A
:100BC0000A282B294672656552616D207072696E24
:100BD00074696E670064653A61643A62653A656695
:100BE0003A66653A6564000A4669726D77617265B6
:100BF000204D4143204164647265737320006C6131
:100C00007A79686F6D652E7275000A436F6E66693A
:100C100067207365727665723A000A282B2957415E
:100C2000544348444F47003230313130334C002078
:100C3000432B2B2076657273696F6E3A00326332F4
:100C4000363537375F323031392D30342D3037007B
:100C50000A4C617A79686F6D652E7275204C6967F0
:100C6000687448756220636F6E74726F6C6C657225
:100C70002000000020002300260029002C002F0067
:100C80003200000100000301060109013D00494E48
:100C90003A0000002200250028002B002E00310021
:100CA000340002010000050108010B0100000A0BDD
:100CB00002090C0D0E0807030401000000000000EB
:100CC0000000000000000000000000000000000024
:100CD00000000000000000001211100000000000E1
:100CE0000000000000000000000000000000000004
:100CF000000000002100240027002A002D00300001
:100D0000330001010000040107010A010102102063
:100D10002008081020401020408002010201080431
:100D200002010102040810204080804020100804C5
:100D3000020180040201804020100804020108041E
:100D40000201010204081020408001020408102062
:100D5000408005050505070508080808020202028B
:100D60000A0A080804040404010101010101010147
:100D70000303030303030303040707070C0C0C0C12
:100D80000C0C0C0C020202020606060606060606FB
:100D90000B0B0B0B0B0B0B0B696E00735F6F7574FA
:100DA000006D79686F6D6500436F6E6E6563746585
:100DB000642E00436F6E6E2E2061626F72746564E4
:100DC0000043757272656E74204C414E20636F6EE5
:100DD0006669672869702C646E732C67772C73754D
:100DE000626E6574293A000A5573652074686573EC
:100DF0006520636F6D6D616E64733A202768656C62
:100E00007027202D207468697320746578740A2710
:100E10006D61632064653A61643A62653A65663A79
:100E200066653A3030272073657420616E642073E4
:100E3000746F7265204D41432D61646472657373F4
:100E400020696E20454550524F4D0A276970205B3E
:100E500069705B2C646E735B2C67775B2C737562B7
:100E60006E65745D5D5D5D27202D20736574207354
:100E700074617469632049500A277361766527207D
:100E80002D207361766520636F6E66696720696ED9
:100E9000204E5652414D0A2767657427205B636FC9
:100EA0006E66696720616464725D27202D20676526
:100EB0007420636F6E6669672066726F6D20707252
:100EC000652D636F6E666967757265642055524C57
:100ED00020616E642073746F726520616464720AAD
:100EE000276C6F616427202D206C6F616420636F15
:100EF0006E6669672066726F6D204E5652414D0ACC
:100F00002770776427202D20646566696E65204D03
:100F10005154542070617373776F72640A276B6940
:100F20006C6C27202D20746573742077617463685E
:100F3000646F670A27636C65617227202D20636CDC
:100F400065617220454550524F4D0A277265626FA8
:100F50006F7427202D207265626F6F7420636F6E2F
:100F600074726F6C6C657200536F66742072656288
:100F70006F6F74696E672E2E2E00444D58696E2077
:100F800042756666657220616C6C6F632065727273
:100F900000496E697420696E2063683A0052414DC1
:100FA0003D000A6D71747420000A6D6F6462757380
:100FB00020000A696E7075747320000A6974656D8B
:100FC0007320000A436F6E666967757265643A0044
:100FD0002C003D0050696E3A00444D58206F7574E6
:100FE00020737461727465642E204368616E6E654F
:100FF0006C733A2000444D5820696E2073746172FE
:101000007465642E204368616E6E656C733A004CA3
:101010006F61646564006C6F6164206661696C6512
:1010200064004E6F2073746F72656420636F6E6628
:101030006967004C6F6164696E6720436F6E666913
:10104000672066726F6D20454550524F4D000A7201
:10105000657175657374204D51545420436F6E66ED
:10106000696700536176656420746F20454550526E
:101070004F4D00536176696E6720636F6E666967D6
:1010800020746F20454550524F4D2E2E00536176EF
:1010900065640A005365742064796E616D6963202C
:1010A00049500A00454550524F4D20636C656172AE
:1010B00065640A0050617373776F726420757064A1
:1010C000617465640A002C20002E003E3E20004919
:1010D0006E76616C696420636F6D6D616E64004152
:1010E00063746976650A0047727020636865636B94
:1010F0003A0A002D3E005075623A2000556E6B6E24
:101100006F776E20636D64200A0053746174757389
:101110002064656666657265640A00206973200054
:1011200044656C6574696E6720636F6E662E20522D
:10113000414D207761733A00536B697070696E6737
:101140002E2E004F4F4D21005D20000A5B003A001B
:101150004D41433A0000ED6A11241FBECFEFD1E2AA
:10116000DEBFCDBF00E00CBF15E0A0E0B2E0E2E2E0
:10117000F8EF00E00BBF02C007900D92A833B10753
:10118000D9F72BE0A8E3B5E001C01D92A535B20761
:10119000E1F718E0CCEAD8E000E006C021970109A9
:1011A000802FFE010E94EE76CB3AD10780E008073F
:1011B000A9F70E94A5620C940F7C0C9400002F925A
:1011C0003F924F925F926F927F928F929F92AF92D7
:1011D000BF92CF92DF92EF92FF920F931F93CF9324
:1011E000DF93CDB7DEB769970FB6F894DEBF0FBEB9
:1011F000CDBF6C012B011A015901088BFD8AEC8AC5
:10120000DC011296ED91FC911397008111810E94EF
:10121000AA4D3B014C0168EE75E087EB97E00E9418
:10122000A85A2AE0B401A30187EB97E00E94E15A93
:1012300061EE75E087EB97E00E94A85AB80187EB52
:1012400097E00E94765B6BED75E087EB97E00E947C
:10125000A85A6C897D8987EB97E00E94563765ED27
:1012600075E087EB97E00E94A85AB20187EB97E000
:101270000E9456376EEC75E087EB97E00E94A85A03
:10128000F60182819381892B09F450C61B861A8648
:101290001D861C861F861E86A114B10459F1850186
:1012A0004E01FAE08F0E911CE12CF12CE214F304B4
:1012B0000CF523E0E216F104E9F0D801AD90BD9001
:1012C0008D01F401A192B1924F016CEC75E087EBB6
:1012D00097E00E94A85AB50187EB97E00E94563725
:1012E00069EC75E087EB97E00E94A85AFFEFEF1AD0
:1012F000FF0ADCCF87EB97E00E94725B60E070E052
:10130000C6010E9412203C0124E04216510451F013
:1013100037E04316510459F183E04816510409F0AF
:1013200053C007C0C6010E94C860892B09F025C1BF
:1013300002C6D60118968C91873009F41AC360E072
:10134000C6010E946520853009F0F2C56AEB75E0A0
:1013500087EB97E00E94A85A65E070E087EB97E082
:101360000E94563787EB97E00E94725BE4C5F60156
:101370008085873009F4FDC260E0C6010E946520C7
:10138000082F10E0863081F469EA75E087EB97E07A
:101390000E94A85AB80187EB97E00E94563787EB66
:1013A00097E00E94725BE9C061E975E087EB97E026
:1013B0000E94A85AB80187EB97E00E94563787EB46
:1013C00097E00E94725BB4C5F2E04F16510409F435
:1013D000D4C04CF44114510489F031E04316510457
:1013E00009F014C1A7C085E04816510409F4E6C00D
:1013F00096E04916510409F485C008C1D601189633
:101400008C91853021F06EE0C6010E944020F601EB
:10141000808590E08A30910508F069C0FC0188273A
:10142000EE58FF4F8F4F0C94EE768C859D85892B5F
:1014300049F4F3E02F16310491F48FE7D6011896A2
:101440008C9304C0B3E02B16310449F44A855B85C4
:101450000C851E85B801C6010E94B61F18C0C601C2
:101460000E94EE1F7B01182F0A85AB01682F702F99
:10147000C6010E94B61FEA86FB86812F110F990BC9
:101480009D878C87802F000F990B9F878E87E88917
:10149000EE2351F101E09E01265F3F4F43E050E013
:1014A00060E070E0C6010E94C45F1EC04A855B8593
:1014B0000C851E85B80114C0F889FF2359F001E09E
:1014C0009E01265F3F4F41E050E060E070E0C601C2
:1014D0000E94C45F4A855B85052E000C660B770B66
:1014E000C6010E94B61F03C013E0212E312C0E94BA
:1014F0004F62609338057093390580933A05909355
:101500003B0584C0C6010E94C860892B39F464E899
:1015100075E087EB97E00E94A85A0CC064E775E07D
:1015200087EB97E00E94A85AD60118968C918730D5
:1015300009F0FEC4F6018085813009F026C560E01F
:10154000C6010E946520813009F01FC50E944F62CC
:10155000009138051091390520913A0530913B05ED
:10156000DC01CB01801B910BA20BB30B853F91409B
:10157000A105B10508F0E3C408C560E0C6010E94FA
:1015800065208530B9F01B861A861D861C861F864D
:101590001E8662E0C6010E944020F889FF2351F0B8
:1015A00000E020E030E040E050E062E070E0C601A2
:1015B0000E94C45FA2E04A2E512C28C0C6010E949E
:1015C000C8601816190614F51B861A861D861C8617
:1015D0001F861E8660E0C6010E946520863011F4D9
:1015E00062E001C065E0C6010E94402000E020E00A
:1015F00030E040E050E062E070E0C6010E94C45F6D
:1016000063E375E087EB97E00E94A85AEC84FD84C1
:10161000C7010F2C000CAA0BBB0B8E8B9F8BA88FC6
:10162000B98FAE85BF85BB8BAA8B2FEF30E00E94B0
:101630000577F4E68F2E912CA12CB12CA5019401F5
:101640000E94AD768901F6018085843009F47FC15E
:1016500050F4813009F44CC0F0F1823089F18330CC
:1016600009F4EFC162C4883009F497C338F48630B6
:1016700009F4A7C1873009F058C47BC1893009F447
:10168000FFC28F3709F051C460E0C3010E94644B70
:1016900060E0C30101960E94644B60E0C3010296C2
:1016A0000E94644BAE85BF852FEF30E00E94057726
:1016B000A50194010E94AD76622FC301039644C137
:1016C0002FEF30E0D7010E940577A50194010E9419
:1016D000AD76D22E78C0AA85BB852FEF30E00E9470
:1016E0000577A50194010E94AD76622FC3012CC13C
:1016F00093012D5F3F4F290132E3E316F1040CF013
:1017000049C082E390E08E199F09EA89FB898E9F88
:10171000D0018F9FB00D9E9FB00D11242FEF30E0B0
:101720000E94057728E833E140E050E00E94AD7662
:10173000622FC2010E94644BEC84FD842EEF31E0E5
:10174000D7010E940577E2E32E2E312C412C512C3B
:10175000A20191010E94AD76AE85BF850E94FD7603
:10176000A50194010E94AD7649015A019701A5E6B1
:10177000BFEF0E94FD76A20191010E94AD76DD24AB
:10178000DA94D20E84010F3F1105E9F0E4F00FEF77
:1017900010E019C02E893F89488D598D2253310997
:1017A00041095109ABE9B0E00E94CC7622E330E078
:1017B00040E050E00E94AD7664E6D62ED20E60E0A6
:1017C000C2010E94644BAA85BB852FEF30E00E94C6
:1017D00005772DE631E040E050E00E94AD76322FF3
:1017E000122F1F71110F110F812F880F15E5682F10
:1017F000619F060E60E0611D1124922F907420728B
:1018000037FD24C091110CC0211104C0862F809592
:10181000F62E14C055E5F52EF60E10E06BEA36C034
:1018200021110FC0182F3AEA139F010E10E0111D6D
:1018300011248BEA811B4AEAF42EF60E682F10E081
:1018400025C080E0F62EF094162F0FC0911112C023
:1018500021110DC0182F2AEA129F010E10E0111D50
:1018600011243BEAF32EF11A1B5A60E00FC0162F29
:1018700010950BC0211104C085E5860F1BEA03C03B
:101880008AEA860F90E0161B682FF12CFFEFDF1617
:1018900009F42AC0DD2009F423C0662329F02D2D88
:1018A000629F060E60E0611DFF2039F03F2D2D2D57
:1018B000329F030E30E0311DF32E112329F03D2D10
:1018C000139F010E10E0111D11242D2D2095229F34
:1018D000020E20E0211D1124620FF20E120F04C02F
:1018E0001FEFFF24FA946FEF0F3F09F422C020E0AE
:1018F000002321F0009F212D09F02F5F2223B1F05A
:10190000662321F0629F060E60E0611DFF2031F02A
:101910003F2D329F030E30E0311DF32E112321F0B5
:10192000129F010E10E0111D112403C010E0F12CD4
:1019300060E0C3010E94644B6F2DC30101960E94B9
:10194000644B612FC30102960E94644BEEC2E48097
:10195000F580F7018085853009F0E7C2C7010E9454
:10196000123BA82EB12CF2E0AF16B1040CF02BC440
:10197000DCC2D6011496ED91FC91159780858530D7
:1019800009F0D3C2C680D780C114D10409F4CDC2F6
:10199000F60161857285CE0101960E94D125EC8801
:1019A000FD8808899E01265F3F4FA101B201CE014B
:1019B00001960E94DF08D6011296CD90DC90139715
:1019C000E3CF77FE06C071946194710801E010E0E6
:1019D00002C000E010E0F62C61E0862D0E94D96183
:1019E000012B69F0B1E04B16510429F061E0E6E00B
:1019F0004E16510409F460E0062F10E011C0F1E02A
:101A00004F16510451F091E080E026E04216510457
:101A100009F090E0092F182F02C001E010E0602FBC
:101A20008F2D0E9400416EE275E087EB97E00E94E7
:101A3000A85AB30187EB97E00E9456376CE275E035
:101A400011C177FE06C071946194710801E010E045
:101A500002C000E010E0F62C61E0862D0E94D96102
:101A60008091A100887F8093A10080919100887F60
:101A7000809391008091A10082608093A100809169
:101A80009100826080939100AA85BB85012B99F01B
:101A9000CD01BB0FAA0BBB0B9C01AD012456310934
:101AA00041095109AFEFB0E00E94CC762CE93FEF3D
:101AB0004FEF5FEF08C02FEF30E00E94057724E67C
:101AC00030E040E050E00E94AD76890161E08F2D6A
:101AD0000E94D9610115110509F4B1C00F3F11052C
:101AE00009F4AFC0F301FF27E455F34FE4918E2FC3
:101AF00090E0FC013197E231F10508F09DC08827A4
:101B0000E458FF4F8F4F0C94EE7684B5806884BD07
:101B100007BD9BC084B5806284BD08BD96C080911E
:101B20008000806880938000109389000093880073
:101B30008CC08091800080628093800010938B0025
:101B400000938A0082C0809180008860809380002A
:101B500010938D0000938C0078C08091B000806855
:101B60008093B0000093B30070C08091B000806299
:101B70008093B0000093B40068C0809190008068AA
:101B80008093900010939900009398005EC080911C
:101B9000900080628093900010939B0000939A00C5
:101BA00054C08091900088608093900010939D00B5
:101BB00000939C004AC08091A00080688093A000A0
:101BC0008091A0008F7B8093A0001093A9000093C8
:101BD000A8003BC08091A00080628093A000109379
:101BE000AB000093AA0031C08091A0008860809370
:101BF000A0001093AD000093AC0027C0809120019D
:101C000080688093200110932901009328011DC052
:101C10008091200180628093200110932B0100931A
:101C20002A0113C0809120018860809320011093C5
:101C30002D0100932C0109C00038110514F460E057
:101C400001C061E08F2D0E94004167E275E087EBE3
:101C500097E00E94A85AB30187EB97E00E9456379D
:101C600065E275E087EB97E00E94A85AB80187EB20
:101C700097E00E94563787EB97E00E94725B55C150
:101C80001A8560E070E0C6010E941220082FF92E2C
:101C900060E175E087EB97E00E94A85A602F7F2DE6
:101CA00087EB97E00E9456376EE075E087EB97E090
:101CB0000E94A85A612F012E000C770B87EB97E04A
:101CC0000E94563787EB97E00E94725B8091050671
:101CD00090910606892B89F060E37AE087EB97E024
:101CE0000E94A85A642D6064C6010E944020412FC2
:101CF000110F550B660B770BB0C081E090E090930D
:101D000006068093050626E040E855E260E070E0B4
:101D10008AE197E00E94F637009305098AE197E08F
:101D200090930409809303091092100A1092120AEA
:101D30001092110A80ED97E090938B0980938A09A5
:101D400010928D0910928C09112339F085E090E0F2
:101D500090938F0980938E0904C010928F0910927E
:101D60008E0986E00E945B3862E370E080E090E0DC
:101D70000E94156282ED97E090938B0980938A0907
:101D800010928D0910928C0934E61302A0011124DF
:101D900050938F0940938E09C1C00480F581E02DD6
:101DA00061857285CE0101960E94D125CE010196F2
:101DB0000E94A91F882309F4B8C08985893009F0D9
:101DC000B4C0142DEA8460E070E0CE0101960E9458
:101DD0001220082FF92E6CE175E087EB97E00E9446
:101DE000A85A602F7F2D87EB97E00E9456376AE153
:101DF00075E087EB97E00E94A85A6E2D0E2C000C20
:101E0000770B87EB97E00E94563764E175E087EB2C
:101E100097E00E94A85A642D042C000C770B87EBE6
:101E200097E00E94563787EB97E00E94725B8091A3
:101E3000050690910606892BA1F060E37AE087EB16
:101E400097E00E94A85A642D6064C6010E94402059
:101E50004E2DEE0C550B660B770BC6010E94B61F7C
:101E600064C081E090E0909306068093050626E02A
:101E700040E855E260E070E08AE197E00E94F637C2
:101E8000009305098AE197E0909304098093030980
:101E90001092100A1092120A1092110A123009F4CC
:101EA000F7C1153009F4F4C16E2DEE0C770B880BD9
:101EB000990B0E94287822E538EB42E152E40E9417
:101EC0000D7720E030E040E251E40E94DD782DEE15
:101ED0003EE94CE35EE30E947E776B017C0120E0EB
:101EE00030E0A9010E94D87820E030E040E05FE3D4
:101EF00087FDC9C1C701B6010E940D770E94F07726
:101F000083ED97E090938B0980938A0910928D0955
:101F100010928C0970938F0960938E0986E00E945D
:101F20005B381092060610920506B5C18FEF01C00E
:101F30008DEF9FEFB0C144244394512CFBCA67E658
:101F400075E087EB97E00E94A85A8FE7F60180873B
:101F50001D861C8684E690E09F878E874A855B8578
:101F600060E074E6C6010E94B61FF889FF2309F4F9
:101F70004DCB00E09E01265F3F4F43E050E060E024
:101F800070E0C6010E94C45F41CB642DC6010E946F
:101F90004020C6010E94EE1FF62EE72E8C01D601CE
:101FA00018962C91233008F0FCC0213070F46A3070
:101FB0007105810591052CF4B2E3FB2EE12C00E0C4
:101FC00010E04F2D5E2D602F0AC06115710581054F
:101FD000910519F01A300CF412E3AB01682F712F40
:101FE000C6010E94B61F4F2D5E2DB80114161506AE
:101FF00016061706E4F5D60118968C9190E08A3003
:10200000910538F5FC018827E257FF4F8F4F0C945C
:10201000EE76C7019A878B87802F000F990B9D87DB
:102020008C87812F110F990B9F878E8753C05B87F9
:102030004A8701E07FC05B874A87B889BB2309F4E0
:10204000E5CA00E020E030E040E050E061E070E010
:102050000AC0E889EE2309F4A8C000E020E030E0DF
:1020600040E050E0B201C6010E94C45F9EC02AE079
:1020700030E087EB97E00E942A5B69E475E087EB2C
:1020800097E00E94A85AD60118968C918530C9F025
:10209000A0F48150823008F041C084E690E09B8734
:1020A0008A871D861C869F878E8744E650E060E005
:1020B00074E6C6010E94B61F0DC08630C9F0883094
:1020C00069F584E190E09B878A8744E150E060E015
:1020D00070E02CC001E09E01265F3F4F43E050E0DE
:1020E00060E070E0C6010E94C45F03E010E02EC013
:1020F00084E690E09B878A8744E650E060E070E0E9
:10210000C6010E94B61FB889BB23F1F000E020E0B1
:1021100030E040E050E061E070E013C084E690E021
:102120009B878A8744E650E060E070E0C6010E9429
:10213000B61F00E09E01265F3F4F41E050E060E0A7
:1021400070E0C6010E94C45F01E010E05E01EAE0B9
:10215000AE0EB11CE12CF12CD5018D909D905D014E
:102160006EE375E087EB97E00E94A85AB70187EB12
:1021700097E00E9456376CE375E087EB97E00E948A
:10218000A85AB40187EB97E00E94563787EB97E097
:102190000E94725BBFEFEB1AFB0A0E151F05E1F6FA
:1021A00004C0243009F403CF1ECFF60180858130AE
:1021B00009F02CCA8C859D85892B09F027CA8FE7E9
:1021C000F601808723CA60E0C7010E947037DC01F6
:1021D00019968D919C911A97998B888B61E0C70114
:1021E0000E947037FC0141845284638474842A8481
:1021F0003B84F2E0AF16B104E9F162E0C7010E944E
:102200007037DC0119960D911C911A97B3E0AB164B
:10221000B10491F163E0C7010E947037FC01818431
:102220009284F4E0AF16B10451F064E0C7010E945B
:102230007037DC011996AD90BC901A9703C032E05C
:10224000A32EB12C8114910461F09401D1010E945C
:10225000FD7624E630E040E050E00E94AD76790162
:1022600001C071019501A20168897989C6010E94A6
:10227000ED255BCE0FEF1FEF8FE3882E912C92E0C0
:10228000A92EB12CE2CFC701B6010E940C7736CE41
:1022900060E070E035CE69960FB6F894DEBF0FBEF1
:1022A000CDBFDF91CF911F910F91FF90EF90DF9005
:1022B000CF90BF90AF909F908F907F906F905F90E6
:1022C0004F903F902F9008954F925F926F927F9220
:1022D0008F929F92AF92BF92CF92DF92EF92FF9236
:1022E0000F931F93CF93DF93CDB7DEB7C15AD14081
:1022F0000FB6F894DEBF0FBECDBFE091A805F091F8
:10230000A9053B96E831F10508F0B7C38827E856E0
:10231000FF4F8F4F0C94EE760E944F62009109069A
:1023200010910A0620910B0630910C06061717072C
:102330002807390708F0A1C301E213E0CF56DE4FAA
:1023400019830883C159D140CD56DE4F18821982B6
:102350001A821B82C359D140CF57DE4F198308839D
:10236000C158D140CD57DE4F188219821A821B8284
:10237000C358D140CF59DE4F19830883C156D1408D
:10238000CD59DE4F188219821A821B82C356D14062
:10239000CF5BDE4F19830883C154D140CD5BDE4F44
:1023A000188219821A821B82C354D1406EE676E0ED
:1023B00087EB97E00E94A85ABE016F567E4F86E0D9
:1023C00090E00E94F53D892B09F467C16EE773E048
:1023D00087EB97E00E94765B1A830983CD56DE4F28
:1023E00088819981AA81BB81C359D1408B839C8309
:1023F000AD83BE83CE0101960E947B55BE016F570F
:102400007E4F8AE090E00E94F53D892B09F42EC1B1
:1024100064E973E087EB97E00E94765B1A83098397
:10242000CD57DE4F88819981AA81BB81C358D140A5
:102430008B839C83AD83BE83CE0101960E947B5526
:10244000BE016F597E4F8EE090E00E94F53D892BD2
:1024500009F4DFC06AE973E087EB97E00E94765BDE
:102460001A830983CD59DE4F88819981AA81BB8166
:10247000C356D1408B839C83AD83BE83CE0101962E
:102480000E947B55BE016F5B7E4F82E190E00E940F
:10249000F53D892B09F477C06FE973E087EB97E08E
:1024A0000E94765B1A830983CD5BDE4F8881998118
:1024B000AA81BB81C354D1408B839C83AD83BE83EF
:1024C000CE0101960E947B551A830983CD5BDE4FB6
:1024D00088819981AA81BB81C354D1408B839C831D
:1024E000AD83BE83CF57DF4F19830883C158D040D7
:1024F000CD59DE4F88819981AA81BB81C356D140D5
:10250000CD57DF4F88839983AA83BB83C358D040BC
:10251000CF53DF4F19830883C15CD040CD57DE4FC6
:1025200088819981AA81BB81C358D140CD53DF4FA7
:1025300088839983AA83BB83C35CD040CF5FDE4F7F
:1025400019830883C150D140CD56DE4F88819981CF
:10255000AA81BB81C359D140CD5FDE4F8883998367
:10256000AA83BB83C350D1409E012F5F3F4FAE0172
:102570004F575F4FBE016F537F4FCE018F5F9E4F0E
:102580000E94BF4185C01A830983CD59DE4F8881DF
:102590009981AA81BB81C356D1408B839C83AD8333
:1025A000BE83CF57DF4F19830883C158D040CD5722
:1025B000DE4F88819981AA81BB81C358D140CD5714
:1025C000DF4F88839983AA83BB83C358D040CF53FE
:1025D000DF4F19830883C15CD040CD56DE4F888120
:1025E0009981AA81BB81C359D140CD53DF4F8883E4
:1025F0009983AA83BB83C35CD040AE014F5F5F4F1A
:10260000BE016F577F4FCE018F539F4F0E940B42E9
:102610003FC01A830983CD57DE4F88819981AA81F3
:10262000BB81C358D1408B839C83AD83BE83CF577E
:10263000DF4F19830883C158D040CD56DE4F8881C3
:102640009981AA81BB81C359D140CD57DF4F88837F
:102650009983AA83BB83C358D040BE016F5F7F4F6D
:10266000CE018F579F4F0E945D4212C01A8309838B
:10267000CD56DE4F88819981AA81BB81C359D14053
:102680008B839C83AD83BE83CE0101960E94A842BA
:1026900087EB97E00E94725B0BC166EA73E087EB01
:1026A00097E00E94765B0FB6F894A8958091600041
:1026B000886180936000109260000FBE80919A053F
:1026C000811107C08FE795E00E94CC4381E08093A1
:1026D0009A058CE395E090936108809360080E94CE
:1026E0002F41CE0101960E94F02989819A810E9492
:1026F000264946E050E067E97AE089E090E00E94F0
:10270000DC3681E293E09A8389831B821C821D82DE
:102710001E82CE0103960E9410490E942549809195
:10272000600890916108DC0192961D921D921D92A5
:102730001C929597FC0116A217A210A611A69A96B4
:102740001D921D921D921C929D9740EE5EE260E0EC
:1027500070E046AB57AB60AF71AF40EA5FE060E05E
:1027600070E0DA964D935D936D937C93DD973E9682
:1027700024E1DF011D922A95E9F726E0E7E9FAE076
:10278000DC01189601900D922A95E1F7FC01EE5BB1
:10279000FF4F10820E94283C8C01019709F04AC02B
:1027A000CE0101960E94F02989819A810E942649D2
:1027B0006091600870916108625F7F4FCE01019661
:1027C0000E94785BCE0103960E94104960916008D8
:1027D000709161086A5E7F4FCE0101960E94785B1E
:1027E000CE0103960E941E496091600870916108B5
:1027F0006E5E7F4FCE0101960E94785BCE010396FC
:102800000E9417490E9425496091600870916108F3
:10281000625E7F4FCE0101960E94785B8B819C8126
:10282000AD81BE8180935C0890935D08A0935E08A3
:10283000B0935F0899E288E10FB6F894A895809369
:1028400060000FBE90936000A895012B19F56CE213
:1028500076E087EB97E00E94A85A6DEF75E087EB72
:1028600097E00E94A85A86EF9FEF9093A905809366
:10287000A8050E944F62DC01CB01805A9541AF4F01
:10288000BF4F8093090690930A06A0930B06B0935E
:102890000C06F3C06DEE75E087EB97E00E94A85A36
:1028A000CE0101960E94D155CE0101960E947B5522
:1028B00081E090E0DEC08091A20581111AC060E045
:1028C00070E080E090E00E94202FD3C00E944F6211
:1028D0000091090610910A0620910B0630910C0612
:1028E0000617170728073907C8F10E94D226811159
:1028F000C4C082E090E0BDC0A895CF55DE4F1882DD
:10290000C15AD140FE01EF56FE4F119211928EE056
:10291000DF011D928A95E9F70091230B1091240B9A
:102920000115110529F0C8010E94123B811137C21F
:102930000E94D2268111A1C0E090230BF090240BBD
:10294000E114F10409F499C0C7010E94123B082F59
:1029500010E0023011050CF03FC28FC020E030E0E3
:1029600043E050E060E48E010F5F1F4FC8010E94FA
:10297000194D68EF74E0C8010E94257BF8010190B1
:102980000020E9F7CF01801B910B08968138910553
:1029900038F50E94D226882319F18091E808909199
:1029A000E908019611F481E090E09093E9088093A2
:1029B000E8088091E8089091E90890936D08809369
:1029C0006E0847E050E068E678E0C8010E940B27F7
:1029D000AC014550510968E678E082EA0E942B2755
:1029E00083E090E09093A9058093A80564E478E0E3
:1029F00087EB97E00E94A85A40C00E944F62009166
:102A0000090610910A0620910B0630910C06061754
:102A100017072807390788F51092A9051092A8050D
:102A20002CC00E944F620091090610910A06209165
:102A30000B0630910C06061717072807390708F40C
:102A400058CF1BC00E949352892B09F052CF0E948D
:102A50004F62DC01CB0188579C4EAF4FBF4F809334
:102A6000090690930A06A0930B06B0930C0686EF16
:102A70009FEF9093A9058093A8050FB6F894A895A9
:102A800080916000886180936000109260000FBEAA
:102A90008091A8059091A905181619060CF059C146
:102AA00000916008109161080115110509F451C1E8
:102AB0000E944F624B015C017801FEE3EF0EF11CB6
:102AC000F70180819181A281B381A5019401281B26
:102AD000390B4A0B5B0BCA01B901683E33E073073F
:102AE0008105910508F446C028EE33E040E050E04F
:102AF0000E948B76861A970AA80AB90AD7018D9286
:102B00009D92AD92BC921397F80186A597A5A0A9B6
:102B1000B1A969017A01CC0CDD1CEE1CFF1C8C15DF
:102B20009D05AE05BF0528F416A617A610AA11AA82
:102B300009C0821B930BA40BB50BF80186A797A7BE
:102B4000A0ABB1ABF80182A993A9A4A9B5A98C1532
:102B50009D05AE05BF0528F412AA13AA14AA15AA4A
:102B600009C0821B930BA40BB50BF80182AB93AB8E
:102B7000A4ABB5ABF80186A597A5A0A9B1A9892BEF
:102B80008A2B8B2B69F4EE5BFF4F8081833041F4FD
:102B900084E08083C8010E94283C01967C0102C029
:102BA000E12CF12CF80182A993A9A4A9B5A9892B3C
:102BB0008A2B8B2BA1F4EE5BFF4F8081833011F0C9
:102BC00081110DC01082F8013E9684E1DF011D9253
:102BD0008A95E9F7C8010E94283C03967C01B2E07F
:102BE000EB16F10429F0E4E0EE16F10409F04AC016
:102BF000CE0101960E94F02989819A810E9426497E
:102C00006091600870916108625F7F4FCE0101960C
:102C10000E94785BCE0103960E9410496091600883
:102C2000709161086A5E7F4FCE0101960E94785BC9
:102C3000CE0103960E941E49609160087091610860
:102C40006E5E7F4FCE0101960E94785BCE010396A7
:102C50000E9417490E94254960916008709161089F
:102C6000625E7F4FCE0101960E94785B8B819C81D2
:102C7000AD81BE8180935C0890935D08A0935E084F
:102C8000B0935F08F3E0EF16F10409F451C064F467
:102C900031E0E316F10451F142E0E416F10409F0E9
:102CA00058C06BE078E049C054E0E516F10409F43F
:102CB00042C085E0E816F10409F04BC06CE378E00F
:102CC00087EB97E00E94A85A87EB97E00E94725B1F
:102CD0000E94D22681110E94FE550E944F62DC01A3
:102CE000CB01805D9A48AF4FBF4F13C068E278E0D8
:102CF00087EB97E00E94A85A0E94D22681110E9479
:102D0000FE550E944F62DC01CB0188519C4FAF4FB2
:102D1000BF4F8093090690930A06A0930B06B093C9
:102D20000C0686EF9FEF9093A9058093A80511C02C
:102D300068EF77E0DDCF6CED77E087EB97E00E94FE
:102D4000A85ACE0101960E94D155CE0101960E944B
:102D50007B5599E288E10FB6F894A89580936000BE
:102D60000FBE909360008091A8059091A905CF5562
:102D7000DE4F0FB6F894DEBF0FBECDBFDF91CF910F
:102D80001F910F91FF90EF90DF90CF90BF90AF9089
:102D90009F908F907F906F905F904F90089560E02C
:102DA000C8010E947037DC0119960D911C911A9789
:102DB0001093A90A0093A80A6FEC77E087EB97E0DD
:102DC0000E94A85AB80187EB97E00E94765B87EBD8
:102DD00097E00E94725BACCD61E0C7010E94703742
:102DE000FC01618472840230110509F43BC362E086
:102DF000C7010E947037FC01818492840330110561
:102E000051F063E0C7010E947037DC011996ED9024
:102E1000FC901A9704C0FE01EF55FE4F7F0140E180
:102E200050E0BE016F567E4F86E390E00E94A72ED1
:102E3000892B21F4053011050CF01DC38E010F56AE
:102E40001E4F7092FC086092FB089092FE088092E0
:102E5000FD0886E39EE59093F4088093F3085E01F5
:102E6000FFE7AF1AFEEFBF0A40E150E062EA77E009
:102E7000C5010E942C6F6E012FE9C21A2EEFD20AF3
:102E800020E030E041E050E060E2C6010E94194DD0
:102E900040E250E06BE977E0C6010E941C6F6BE7EF
:102EA00077E087EB97E00E94A85AB30187EB97E0A1
:102EB0000E94765B69E777E087EB97E00E94A85A6B
:102EC000B40187EB97E00E94563762E777E087EB23
:102ED00097E00E94A85AB70187EB97E00E94765BC3
:102EE0006DE677E087EB97E00E94A85A8090A80AE9
:102EF0009090A90A0E94D22681113BC16091FB08E3
:102F00007091FC0880916608909167084091FD08D7
:102F10005091FE08DC01ED91FC916115710521F0E5
:102F20000088F189E02D16C00684F785E02D21E2A6
:102F300033E03A8329834090F7085090F808609076
:102F4000F9087090FA084B825C826D827E82BE0125
:102F50006F5F7F4F19958130910509F003C1909300
:102F6000E9088093E80887E0E2E1F2E0DE011196EB
:102F700001900D928A95E1F7FE013196ADE6B8E039
:102F8000CE01089621912D93E817F907D9F7E1149E
:102F9000F10429F00115110521F086EF03C086E345
:102FA00001C086EB80937408109275088FE08093BF
:102FB0007608F40101900020E9F7CF0188199909FA
:102FC00040968138910508F0C1C04FE050E068E6B6
:102FD00078E0C4010E940B27F60101900020E9F778
:102FE0003197EC19FD09E80FF91F3296E138F10528
:102FF00008F0ACC0AC0168E678E0C6010E940B277F
:10300000F50101900020E9F73197EA19FB09E80F73
:10301000F91F3296E138F10508F098C0AC0168E676
:1030200078E0C5010E940B27E114F10479F1F70162
:1030300001900020E9F73197EE19FF099C012E5FFE
:103040003F4FE20FF31FE138F10508F07FC0AC01FC
:1030500068E678E0C7010E940B2701151105B1F061
:10306000F80101900020E9F73197E01BF10B9C017A
:103070002E5F3F4FE20FF31FE138F10508F066C005
:10308000AC0168E678E0C8010E940B27AC0145500E
:10309000510968E678E080E10E942B270E944F6288
:1030A0006093EA087093EB088093EC089093ED0826
:1030B0006093EE087093EF088093F0089093F10806
:1030C0008091660890916708DC01ED91FC91008485
:1030D000F185E02D1995892BC1F40E944F62009172
:1030E000EE081091EF082091F0083091F108DC0112
:1030F000CB01801B910BA20BB30B88399A43A1051E
:10310000B105F0F28CEF9FEF1DC0CE018F579F4F9E
:103110000E9433530497D1F480916B08811111C040
:103120000E944F626093EE087093EF088093F0085E
:103130009093F1081092F20810920209109201097E
:1031400018C090E09093020980930109809166086D
:1031500090916708DC01ED91FC910488F589E02DE0
:1031600019959CC18EEF9FEF9093020980930109FE
:1031700095C10091A80A1091A90A6FE577E087EB45
:1031800097E00E94A85AB80187EB97E00E94765B0F
:1031900087EB97E00E94725B81E08093A20520E0BC
:1031A00030E043E050E060E4CE018F5F9E4F0E942C
:1031B000194D68EF74E0CE018F5F9E4F0E94257B12
:1031C000CE018F5F9E4F0E94B53D20E030E042E08F
:1031D00050E060E4CE018F5F9E4F0E94194D68EF72
:1031E00074E0CE018F5F9E4F0E94257BBE016F5F12
:1031F0007E4F87EB97E00E94CC5A87EB97E00E94C6
:10320000725BCE018F5F9E4F0E94B53D20E030E0A3
:1032100041E050E060E4CE018F5F9E4F0E94194D67
:1032200068EF74E0CE018F5F9E4F0E94257BBE0148
:103230006F5F7E4F87EB97E00E94CC5A87EB97E059
:103240000E94725BCE018F5F9E4F0E94B53DFE01D2
:10325000EF53FF4F119211921EE3DF01212F1D92B8
:103260002A95E9F71A821982FE0133968EE7DF016B
:103270001D928A95E9F720E030E041E050E060E4FB
:10328000CE018F539F4F0E94194D40E450E06BE9EF
:1032900077E0CE018F539F4F0E941C6F40E850E0B3
:1032A00068E177E0CE0101960E942C6FBE016F5F4E
:1032B0007F4FCE018F539F4F0E94E42720E030E0E4
:1032C00041E050E060E4CE018F539F4F0E94194DC2
:1032D00040E450E062E177E0CE018F539F4F0E94BF
:1032E0001C6F40E850E068E077E0CE0101960E9454
:1032F0002C6F40E850E065EF76E0CE0101960E9429
:103300001C6FBE016F5F7F4FCE018F539F4F0E9496
:10331000E42720E030E041E050E060E4CE018F534C
:103320009F4F0E94194D40E450E067E279E0CE01E2
:103330008F539F4F0E941C6F40E850E065EE76E08F
:10334000CE0101960E942C6FBE016F5F7F4FCE01B0
:103350008F539F4F0E94E42720E030E041E050E08F
:1033600060E4CE018F539F4F0E94194D40E450E01E
:103370006EED76E0CE018F539F4F0E941C6F40E8A8
:1033800050E068ED76E0CE0101960E942C6FBE0100
:103390006F5F7F4FCE018F539F4F0E94E427A09114
:1033A0000706B0910806109709F443C080911902EE
:1033B00090911A02AE014F5B5E4FFA018193919397
:1033C0002EE111922A95E9F79E012F573F4FF901FF
:1033D0008193919311921A95E9F716960D911C918C
:1033E0001797E0900706F0900806E114F10471F0D9
:1033F0000115110559F0D80118968C918530A9F75F
:10340000C8010E94123B882381F370C020E030E0A5
:1034100041E050E060E4CE018F539F4F0E94194D70
:1034200040E450E06BE776E0CE018F539F4F0E945F
:103430001C6F84E090E09093A9058093A8050E94FA
:103440004F62DC01CB0188579C4EAF4FBF4F80933A
:10345000090690930A06A0930B06B0930C0662E44B
:1034600077E0C6CA8BE5882E87E0982E9E012F55FF
:103470003E4F7901D4CC64E08091230B9091240BD2
:103480000E947037DC0119960D911C911A976FEA12
:1034900077E087EB97E00E94A85AD3CC009101090E
:1034A0001091020966E377E087EB97E00E94A85A43
:1034B000B80187EB97E00E9456376EE177E087EB23
:1034C00097E00E94A85A0E944F62DC01CB01885706
:1034D0009C4EAF4FBF4F8093090690930A06A0936E
:1034E0000B06B0930C068CE090E0C3CA60E0C80104
:1034F0000E947037FC0181859285A385B4858A304E
:10350000910508F463C020E030E041E050E060E461
:10351000CE018F539F4F0E94194DF8016081718138
:1035200040E450E0CE018F539F4F0E944B7B62ECF2
:1035300073E0CE018F539F4F0E94257B40E450E003
:103540006AE876E0CE018F539F4F0E941C6FBE0148
:103550006F5B7E4FCE018F539F4F0E94E427CF5762
:10356000DF4F8881C158D040882361F120E030E0EE
:1035700041E050E060E4CE018F539F4F0E94194D0F
:10358000D8016D917C9140E450E0CE018F539F4F64
:103590000E944B7B62EC73E0CE018F539F4F0E94E1
:1035A000257B40E450E062E876E0CE018F539F4FE8
:1035B0000E941C6FBE016F577F4FCE018F539F4FEC
:1035C0000E94E427F801028113810BCFFC0140E245
:1035D00050E08827E055FF4F8F4F0C94EE7662ED58
:1035E00076E0CE018F5B9E4F0E942C6FCF57DF4F4E
:1035F0001882C158D04087CF6DEC76E0CE018F5B4A
:103600009E4F0E942C6F40E450E06CEA76E017C0B9
:1036100066EA76E0CE018F5B9E4F0E942C6F40E4FD
:1036200050E062EA76E00BC06AE976E0CE018F5B9B
:103630009E4F0E942C6F40E450E064E976E0CE019A
:103640008F579F4F0E942C6F5ECFBC018230910537
:1036500008F40895613E8EE1780748F49B0195E0F7
:10366000369527959A95E1F748E0420F01C04FEF54
:1036700091E0242F30E0290F311D35952795229FA9
:10368000F001239FF00DF00D11246E177F0718F441
:103690004FEF420F04C02F3F39F091E0920F4917CE
:1036A00040F78FEF890F08958FEF0895CF93DF9341
:1036B000009709F447C0FC012081222309F442C08D
:1036C000EC0168EA79E00E94136F892BF1F163EA5B
:1036D00079E0CE010E94136F892BD1F16EE979E078
:1036E000CE010E94136F892BB1F165E979E0CE011B
:1036F0000E94136F892B91F16FE879E0CE010E944F
:10370000136F892B71F16BE879E0CE010E94136F82
:10371000892B51F166E879E0CE010E94136F892B65
:1037200031F162E879E0CE010E94136F892B11F12B
:103730006EE779E0CE010E94136F892BF1F489E0E6
:1037400090E01DC080E090E01AC081E090E017C0DA
:1037500082E090E014C083E090E011C084E090E04B
:103760000EC085E090E00BC086E090E008C087E0E6
:1037700090E005C088E090E002C08FEF9FEFDF91FE
:10378000CF9108952F923F924F925F926F927F92C6
:103790008F929F92AF92BF92CF92DF92EF92FF9261
:1037A0000F931F93CF93DF93CDB7DEB72A970FB652
:1037B000F894DEBF0FBECDBF5C016B01042F790111
:1037C000672B09F487C021153105F9F0D9018C91D7
:1037D0008823D9F06FE270E0C9010E94307B009726
:1037E00039F0FC011192CF010E94561B4C0102C01E
:1037F000812C912CC7010E94561B7C01019739F046
:103800008A94892809F065C002C0E12CF12C6DEF83
:1038100079E0C6010E94136F892B09F40BC269EF8E
:1038200079E0C6010E94136F892B09F41FC264EF6F
:1038300079E0C6010E94136F892B09F408C26DEE6E
:1038400079E0C6010E94136F892B09F403C268EE68
:1038500079E0C6010E94136F892B09F4FEC164EE62
:1038600079E0C6010E94136F892B09F4F9C16FED4D
:1038700079E0C6010E94136F892B09F4F4C16AED47
:1038800079E0C6010E94136F892B09F4D3C164ED5E
:1038900079E0C6010E94136F892B09F4E7C16BEC34
:1038A00079E0C6010E94136F892B09F4E2C162EC32
:1038B00079E0C6010E94136F892B09F4DDC1D6019E
:1038C0008C918D3251F090ED980F9A3030F0833218
:1038D000B9F1E0C180E090E0DDC1FE0131964F0119
:1038E000412C512C1E2F9A8632012FEF621A720A38
:1038F0002301C6010E94EC6E1C016CE270E0C6015F
:103900000E94307B6C01892B19F03FEFC31AD30A58
:10391000D4012D923D924D01C114D10439F0F3E050
:103920006F16710409F743E0442E512CD501ED9137
:10393000FC910190F081E02D212F3A85A20175C004
:10394000CE0107969E01275F3F4F3F932F93215053
:1039500031093F932F939F938F9385E494E09F9336
:103960008F93DF92CF920E94E47B0FB6F894DEBF74
:103970000FBECDBF039709F0ACCF1F818884998417
:10398000812F811608F4882DC92C891508F4C82EBA
:103990001C198C189C189C2D90959F3F09F448C0C9
:1039A00080E090950E94251BD82ED094882D90E021
:1039B000810F911D890D911D892BE9F5CD2CC094A6
:1039C000D12C10E0212F30E0ADE6B1E00E94DF768F
:1039D000412C512C32014A94A30192010E94AD76F0
:1039E0003A8329832D2D30E0A4E6B0E00E94DF76F3
:1039F000A30192010E94AD763C832B832C2D30E0F5
:103A0000A4E6B0E00E94DF76A30192010E94AD76A9
:103A10003E832D83D501ED91FC910190F081E02D45
:103A20009E012F5F3F4F43E050E060E070E030C107
:103A3000DD24DA94BBCFBFEFDB16F9F0D11002C062
:103A4000DD24D3944D2C512C612C712C6FEF7FEF22
:103A500080E090E0A30192010E94AD76A12FB0E03A
:103A60000E94CC76172FA82DB0E00E94CC76872E2E
:103A7000A92DB0E00E94CC76972E682C712C610E97
:103A8000711C690C711CEFEF6E167104FCF461146B
:103A9000710419F466246394712C930140E050E0A2
:103AA0006FEF7FEF80E090E00E94AD76A12FB0E055
:103AB0000E94CC76172FA82DB0E00E94CC76872EDE
:103AC000A92DB0E00E94CC76972E05C0FFEF6F16AF
:103AD000710409F06CF42C2D362D230F08F42FEF10
:103AE000922F2F3F29F080E00E94251BC82E02C094
:103AF000CC24CA94892D911608F4812F881508F4D6
:103B0000882D81132FC081100DC0182F20E8121BA3
:103B100008F410E020E6129F010E10E0111D1124A0
:103B2000105386C0282D30E0482F50E0421B530B25
:103B30002417350744F4182D20E6129F010E10E0DB
:103B4000111D112475C016E5180D181B24E0121B59
:103B500008F410E020E6129F010E10E0111D112460
:103B6000105E66C0881139C091101AC03BEA232F3D
:103B7000211B08F420E04FE2249F020E20E0211DCB
:103B80001124482F431B08F440E0142F30E6139F04
:103B9000010E10E0111D1124120F1695105C48C083
:103BA000292D30E090E0821B930B192D281739073F
:103BB00044F420E6129F010E10E0111D1124105A4A
:103BC00037C025E5121B08F410E020E3129F010E18
:103BD00010E0111D112410582BC011110DC0192D0A
:103BE00020E8121B08F410E020E3129F010E10E001
:103BF000111D112418571CC0212F30E0892D90E091
:103C0000821B930B2817390744F420E6129F010EFC
:103C100010E0111D112410560BC025E5121B08F4ED
:103C200010E020E6129F010E10E0111D1124105427
:103C30001F5FC8CED501ED91FC910190F081E02D80
:103C400020E030E040E050E061E070E021C063E05F
:103C500070E014C064E070E011C065E070E00EC078
:103C600066E070E00BC067E070E008C062E070E002
:103C700005C068E070E002C069E070E0D501ED9138
:103C8000FC910190F081E02D20E030E040E050E038
:103C9000C50119952A960FB6F894DEBF0FBECDBFA9
:103CA000DF91CF911F910F91FF90EF90DF90CF9018
:103CB000BF90AF909F908F907F906F905F904F904C
:103CC0003F902F9008958F929F92AF92BF92CF9284
:103CD000DF92EF92FF920F931F93CF93DF93E091C8
:103CE0000706F0910806309709F468C0812EC02FAE
:103CF000932EC22EA52ED42EB72ED62FBC01CF01C7
:103D00000E947D378C01009709F45BC0DC01189696
:103D10008C91853009F055C060E0C8010E94703771
:103D20007C0161E0C8010E947037FC0101851285A9
:103D3000D70119962D913C911A972130310569F0E0
:103D40002CF4232BF1F56C2FC80118C0223031055B
:103D500049F027303105A9F034C06C2FC801039613
:103D60000E94644B6D2FC8010E94644B6D2DC801E9
:103D700001960E94644B6C2DC80102960E94644B10
:103D800020C0892BF1F080858530D9F4E680F7805A
:103D9000E114F104B1F00C2F182D2C2D392D4D2DDF
:103DA0005A2D6D2F7B2DF701818592850E94631E10
:103DB000D7011296ED90FC901397EACF80E090E047
:103DC00002C081E090E0DF91CF911F910F91FF90B1
:103DD000EF90DF90CF90BF90AF909F908F9008951D
:103DE000CF92DF92EF92FF920F931F93CF93DF93C7
:103DF000E091270BF091280B3097A1F0908595303A
:103E000089F469017A01EB01682FCF010E947037B4
:103E1000FC0181859285009729F09601A701BE01DA
:103E20000E94631EDF91CF911F910F91FF90EF9041
:103E3000DF90CF900895AF92BF92CF92DF92EF9232
:103E4000FF920F931F93CF93DF938091200B90915C
:103E5000210B892B09F472C0E1E0F0E0C0E0D0E072
:103E6000CC24C394D12CB6010C2E02C0660F771F50
:103E70000A94E2F74091F3055091F4057F0184E044
:103E8000E80EF11CCF01B12C9C01A0910602B0916B
:103E90000702A817B90720F4209106023091070203
:103EA000A0913A0BB0913B0BA20FB31FAC90A09125
:103EB000200BB091210B9C0121503109A20FB31F9F
:103EC0000A2D10E02C9130E00217130729F0462B41
:103ED000572BAC92BB24B3940196E816F906A1F6D1
:103EE0005093F4054093F305BB2011F18091200B12
:103EF0009091210BE80FF91F028110E0218130E041
:103F0000408150E03197608170E0CE010E94F01E48
:103F10000E944F62DC01CB01845D9E4FAF4FBF4FCB
:103F20008093EF059093F005A093F105B093F2050F
:103F30002196F701C430D10509F095CFDF91CF91DB
:103F40001F910F91FF90EF90DF90CF90BF90AF90B7
:103F50000895DC011296ED91FC911397309721F0B2
:103F600081E09085953009F080E00895CF92DF924E
:103F7000EF92FF92CF93DF93DC011696ED91FC91C7
:103F80001797309721F12085223009F56A017B01CE
:103F9000EC016AEB79E087EB97E00E94A85A64EBAA
:103FA00079E087EB97E00E94A85A2AE030E0B70159
:103FB000A60187EB97E00E942A5B87EB97E00E94BF
:103FC000725BEE81FF81C186D286E386F486DF9143
:103FD000CF91FF90EF90DF90CF900895FC01868104
:103FE0009781009789F0FC012085223041F025302F
:103FF00079F460E00E947037009779F0FC016185E8
:1040000072858385948508956FEF7FEFCB010895C6
:104010006EEF7FEF8FEF9FEF08956DEF7FEF8FEFE4
:104020009FEF08950F931F93CF93DF93FC01C481FB
:10403000D581209799F08885823029F4672B71F417
:1040400089859A8518C0853061F48B01CE010E9464
:10405000123B90E0081719073CF003C08FEF9FEF69
:104060000AC08EEF9FEF07C0602FCE010E9470370D
:10407000FC0181859285DF91CF911F910F91089569
:10408000CF93C62F63E0FC01828193810E94703739
:104090000097C9F04C2F50E060E070E0FC014187D0
:1040A0005287638774876CEA79E087EB97E00E9418
:1040B000A85A6C2F87EB97E00E94983787EB97E020
:1040C000CF910C94725BCF910895CF93C62F63E08C
:1040D000FC01828193810E947037009731F0FC01CE
:1040E0008185C11103C08F7001C08FEFCF910895FA
:1040F000BF92CF92DF92EF92FF920F931F93CF93D5
:10410000DF93EC010E94A91F882309F441C08A8132
:104110009B810E94123B082F10E0C801880F991F55
:104120009C012B593D4F790132E0B32E043011052B
:10413000D4F4F701C190D1907F010E94BC35009763
:1041400051F0FC01B086A601DD0C660B770B4187B0
:10415000528763877487BC018A819B810E949F3745
:104160000F5F1F4FE3CF0A811B8160E0C8010E94EF
:104170007037FC018185888761E0C8010E94703733
:104180009D838C8362E0C8010E9470379F838E8379
:10419000DF91CF911F910F91FF90EF90DF90CF9023
:1041A000BF900895CF93DF93EC01FB01248135810B
:1041B00040815181628173810E942A5BCE01DF912F
:1041C000CF9108958F929F92AF92BF92CF92DF923C
:1041D000EF92FF920F931F93CF93DF93CDB7DEB78C
:1041E000C054D1090FB6F894DEBF0FBECDBF8C010D
:1041F0005B01FC01F3806AE779E087EB97E00E94BE
:10420000A85A6F2D87EB97E00E94983768E779E00E
:1042100087EB97E00E94A85AB50187EB97E00E94D0
:10422000563787EB97E00E94725BF801C080D1801F
:1042300060E574E0C6010E947D374C0165E574E0DD
:10424000C6010E947D378C016AE574E0C6010E94B8
:104250007D377C016FE574E0C6010E947D376C01FB
:104260000097D1F0FC016185728540E450E0CE01F9
:1042700001960E94697B0E94D226882369F0809172
:10428000A505882309F44BC007C0F8016185728534
:10429000FB018081811167C08114910409F468C019
:1042A000F40161857285CE0101960E94D125CE016F
:1042B00001960E94A91F882309F45AC0AB2879F0FF
:1042C0000115110551F4E12CF12C01E020E030E062
:1042D00040E050E061E070E00EC0F80112C0E1146F
:1042E000F10471F4E12CF12C01E020E030E040E039
:1042F00050E062E070E0CE0101960E94DF0838C015
:10430000F70161857285FB018081882389F120E0B6
:1043100030E041E0CE0101960E94C21B29C06FE24D
:1043200070E0CE0101960E94307B892B51F4F6019A
:104330002185328543E050E060E4CE0101960E9481
:10434000194DA114B10439F00115110509F09DCFE3
:1043500064E674E008C0E114F10419F467E674E05F
:1043600002C0F70193CFCE0101960E94E42794CFBB
:10437000C05CDF4F0FB6F894DEBF0FBECDBFDF913C
:10438000CF911F910F91FF90EF90DF90CF90BF9052
:10439000AF909F908F900895FF920F931F93CF93AC
:1043A000DF93EC011D821C821A821B820881198115
:1043B0000115110509F452C0F8018085863009F015
:1043C0004DC080910D0690910E06892B09F446C0D0
:1043D0006BE674E0C8010E947D37009719F0FC017C
:1043E00081858A83F801808191810E94EC6EF82E8C
:1043F0008B836DE674E0C8010E947D37009759F504
:104400001A8163E779E087EB97E00E94A85A6F2D45
:1044100087EB97E00E94983761E779E087EB97E0B8
:104420000E94A85A612F87EB97E00E94983787EB8C
:1044300097E00E94725B40E050E06DE674E0888196
:1044400099810E94BC376DE674E0888199810E9451
:104450007D37009719F009969D838C83DF91CF916A
:104460001F910F91FF900895EF92FF920F931F936A
:10447000CF93DF938091F3059091F405C4E0D0E0F1
:1044800021E030E0AC0142235323452B29F0A90160
:104490004095509584239523220F331F219791F740
:1044A0009093F4058093F3050E944F620091EF050D
:1044B0001091F0052091F1053091F2056017710718
:1044C0008207930708F457C0012B022B032B09F432
:1044D00052C01092EF051092F0051092F105109263
:1044E000F205E12CF12CE091200BF091210BEC0F67
:1044F000FD1F038110E0228130E0418150E06081A6
:1045000070E0C7010E94F01E8FEFE81AF80A2496A7
:1045100084E0E816F10439F7C1E0D0E080910602AA
:10452000909107028C179D0728F4809106029091C4
:10453000070201C0CE0120913A0B30913B0BF901EB
:10454000E80FF91F608187EB97E00E9498376FE6CC
:1045500074E087EB97E00E94765B2196C131D1052C
:10456000E9F687EB97E0DF91CF911F910F91FF90D4
:10457000EF900C94725BDF91CF911F910F91FF90A0
:10458000EF9008952F923F924F925F926F927F9299
:104590008F929F92AF92BF92CF92DF92EF92FF9253
:1045A0000F931F93CF93DF93CDB7DEB728970FB646
:1045B000F894DEBF0FBECDBF8C016B010E94E334C7
:1045C000019609F4D3C2D801ED91FC910284F385E0
:1045D000E02DC80119957C018F3FBFEF9B0709F4BF
:1045E000C5C2D801ED91FC910684F785E02D682FB6
:1045F000C8011995B2E2EB16F10429F4B601C8011D
:104600000E940435B5C2EDE2EE16F10429F0C701AF
:10461000C0970A9708F044C1D801ED91FC9102843B
:10462000F385E02DC80119957C018F3FBFEF9B07F3
:1046300009F49CC28D9789F4D801ED91FC91028414
:10464000F385E02DC80119957C01019609F48EC20D
:10465000EFEFFFEFF887EF8304C021E030E0388709
:104660002F83C701C097A12CB12C0A97C8F49AE0F8
:10467000992E9A9CC0019B9C900D1124B701605308
:1046800071095B01A80EB91ED801ED91FC9102845D
:10469000F385E02DC80119957C01C0970A9748F36E
:1046A000BEE2EB16F104D1F0C7018F7D8534910590
:1046B000A9F0EF81F885AE9EC001AF9E900DBE9E21
:1046C000900D1124092E000CAA0BBB0BF60181875B
:1046D0009287A387B48782E08087D8C0B501BB0CDE
:1046E000880B990B0E9428782B013C01FEE2EF1603
:1046F000F104A1F5D801ED91FC910284F385E02D40
:10470000C80119957C01212C312C20E030E040E2D9
:1047100051E4C301B2010E94DD784B015C01B70195
:1047200060537109072E000C880B990B0E942878A2
:10473000A50194010E940D772B013C01B1E02B1AD9
:104740003108D801ED91FC910284F385E02DC80178
:1047500019957C01C0970A97C0F202C0212C312C18
:10476000C7018F7D8534910509F042C0D801ED91D4
:10477000FC910284F385E02DC80119957C018B32F0
:10478000910559F4D801ED91FC910284F385E02D57
:10479000C80119957C01B1E00CC08D9761F4D80176
:1047A000ED91FC910284F385E02DC80119957C01FF
:1047B000BFEFBE8302C0E1E0EE83A12CB12C8AE002
:1047C000982EC701C0978A309105B0F49A9C900149
:1047D0009B9C300D11245C01A20EB31ED801ED91FB
:1047E000FC910284F385E02DC80119957C01E9CF85
:1047F000B1E0BE83A12CB12CEF81F885BF01FF0F82
:10480000880B990B0E942878A30192010E94DD7801
:104810002B013C01B501BB0C880B990B0E94287839
:104820004B015C01FE816F2FFF0F770B880B990BFB
:104830000E9428789B01AC01C501B4010E94DD787B
:104840004B015C01B101330C880B990B0E94287855
:104850009B01AC01C501B4010E940D779B01AC0125
:1048600060E070E080E291E40E944A799B01AC0133
:10487000C301B2010E94DD78D60119966D937D9334
:104880008D939C931C9783E018968C93D801ED919F
:10489000FC910684F785E02D6E2DC801199522C084
:1048A000BBE5EB16F10409F060C0D801ED91FC9175
:1048B0000284F385E02DC80119958B35910509F027
:1048C00055C185E0F6018087C8010E94E334D80114
:1048D000ED91FC910284F385E02DC80119958D3589
:1048E000910519F480E090E043C1D801ED91FC916D
:1048F0000684F785E02D682FC8011995BB24BA946A
:104900000E94BC357C01009709F430C1BB2021F026
:10491000F6019783868308C0D40113969C938E93E7
:104920001297FC0195828482C8010E94E334B7018A
:10493000C8010E94C222892B09F018C1C8010E9437
:10494000E334D801ED91FC910284F385E02DC80198
:104950001995B12C47018C32910591F221E030E09C
:104960008D35910509F089C086C0BBE7EB16F104CF
:1049700009F088C0D801ED91FC910284F385E02D07
:10498000C80119958B37910509F0F0C086E0F60152
:104990008087C8010E94E334D801ED91FC91028424
:1049A000F385E02DC80119958D37910509F49ACF4B
:1049B000D801ED91FC910684F785E02D682FC801A0
:1049C000199599249A940E94BC357C01009709F4AA
:1049D000CDC0992021F0F6019783868308C0D501C8
:1049E00013969C938E931297FC01B582A482C80102
:1049F0000E94E334B701C8010E940435019609F40E
:104A0000B5C0C8010E94E334D70119968D919C91DD
:104A10001A9711969C938E931A961C921E92199730
:104A2000D801ED91FC910284F385E02DC801199520
:104A3000CA9709F09BC0C8010E94E334B701C801BE
:104A40000E94C222019609F491C0C8010E94E33479
:104A5000D801ED91FC910284F385E02DC8011995F0
:104A6000912C57018C32910509F4ADCF21E030E053
:104A70008D37910511F420E030E088279927821BBB
:104A8000930B76C0BEE6EB16F10411F519821A827B
:104A90001B821C82D801ED91FC910484F585E02DE8
:104AA00044E050E0BE016F5F7F4FC8011995049745
:104AB00009F05CC044E050E061E774E0CE0101968B
:104AC0000E945B7B009709F051C0F601108650C030
:104AD000F6E6EF16F10421F59E012F5F3F4F7901B5
:104AE00085E0D9011D928A95E9F7D801ED91FC91F5
:104AF0000484F585E02D45E050E0B901C801199521
:104B00000597A1F545E050E066E774E0C7010E9413
:104B10005B7B009759F521E0F6012087118628C0BC
:104B2000F4E7EF16F10411F519821A821B821C8238
:104B3000D801ED91FC910484F585E02D44E050E02E
:104B4000BE016F5F7F4FC8011995049779F444E067
:104B500050E06CE774E0CE0101960E945B7B009709
:104B600029F421E0F6012087218702C08FEF9FEF13
:104B700028960FB6F894DEBF0FBECDBFDF91CF9160
:104B80001F910F91FF90EF90DF90CF90BF90AF906B
:104B90009F908F907F906F905F904F903F902F905D
:104BA0000895CF93DF93EC0181E792E099838883A6
:104BB0006115710559F080910706909108060097DC
:104BC00029F00E947D379B838A8302C01B821A8250
:104BD000CE01DF91CF910C9478206F927F928F92CB
:104BE0009F92AF92BF92CF92DF92EF92FF920F937C
:104BF0001F93CF93DF93CDB7DEB72C970FB6F89402
:104C0000DEBF0FBECDBF4C01762E672E6A01590163
:104C10008091050690910606892BA1F060E37AE069
:104C200087EB97E00E94A85A60E4C4010E944020EC
:104C3000A701FF0C660B770BC4010E94B61F8FEF14
:104C40009FEF9BC081E090E090930606809305065D
:104C500026E240E855E260E070E08AE197E00E94D9
:104C6000F637709205098AE197E0909304098093E2
:104C700003091092100A1092120A1092110A0115DB
:104C8000110541F00130110539F4FE2CEE24EE241B
:104C9000EA9402C0FF24FA94C701A0E0B0E08F8339
:104CA0009887A987BA8780E190E09C878B87A601C7
:104CB00060E070E049835A836B837C839E838D839D
:104CC000672D762D87EB97E00E9456376DE27AE0EC
:104CD00087EB97E00E94A85ABE016F5F7F4F87EB7A
:104CE00097E00E94D2208C0169E27AE00E94A85AE3
:104CF000B501C8010E94563766E27AE0C8010E94F9
:104D0000A85ABE01695F7F4FC8010E94D2200E944D
:104D1000725BA114B10491F082E0A816B10409F508
:104D2000D0928B09C0928A0910928D0910928C0939
:104D3000F0928F09E0928E0986E010C0D0928B0924
:104D4000C0928A09E11003C080E090E002C080E0D8
:104D50009FEF90938D0980938C0985E00E945B38CA
:104D600006C06EE07AE087EB97E00E94A85A1092A6
:104D700006061092050680E090E02C960FB6F89497
:104D8000DEBF0FBECDBFDF91CF911F910F91FF907E
:104D9000EF90DF90CF90BF90AF909F908F907F90DB
:104DA0006F900895CF93809166089091670800975F
:104DB00071F1DC01ED91FC910688F789E02D1995E0
:104DC000C1E0811125C0C0E08091010990910209E4
:104DD000892BF1F48DEF9FEF9093020980930109E5
:104DE0008091660890916708DC01ED91FC91068046
:104DF000F781E02D19958091660890916708DC0194
:104E0000ED91FC910488F589E02D199501C0C0E071
:104E10008C2FCF910895CF93DF93EC01FA01329656
:104E2000E60FF71FDC01AD014C1B5D0BCF01861BAC
:104E3000970B2D91222311F02193F5CF9C01241B78
:104E4000350B620F731FFB013297508331964083FD
:104E5000DF91CF910895EF92FF920F931F93CF931D
:104E6000DF9300D01F92CDB7DEB77B01BA0130E0EF
:104E7000962F9F77660F672F661F770B71956115C9
:104E8000710509F0906821E0230FE1E0F0E0EC0FFC
:104E9000FD1FE30FF11D90836115710511F0322F95
:104EA000E7CF30E0B701621B730B6C5F7F4FDB0114
:104EB0008C93DE011196F701E21BF30B359685E02A
:104EC000E80EF11CEE16FF0619F08D918193FACFD2
:104ED00080916608909167082F5F3F4F8901040F0A
:104EE000151FDC01ED91FC910280F381E02DA801FA
:104EF00019957C010E944F626093EA087093EB0859
:104F00008093EC089093ED0881E00E151F0509F0E1
:104F100080E00F900F900F900F90DF91CF911F9135
:104F20000F91FF90EF900895DF92EF92FF920F9311
:104F30001F93CF93DF938C01D62EE72EEA01F22E3A
:104F40000E94D2268823B9F1F80101900020E9F7E8
:104F50003197E01BF10BCE010796E80FF91FE138FE
:104F6000F10548F545E050E068E678E0C8010E94A8
:104F70000B27AC01ED2DFE2DDC01A859B74F9F0189
:104F80002C0F3D1FE217F30719F081918D93FACF93
:104F90002597FF2011F081E301C080E34C0F5D1FD6
:104FA00068E678E0DF91CF911F910F91FF90EF902D
:104FB000DF900C942B2780E0DF91CF911F910F9110
:104FC000FF90EF90DF900895FB0101900020E9F73A
:104FD0003197AF01461B570B21E00C949427CF92D9
:104FE000DF92EF92FF920F931F93CF93DF931F9265
:104FF0001F92CDB7DEB76C0161E00E946520182FCB
:1050000086FF1BC0C6010E94EE1F7A83698360E0A1
:105010007AE087EB97E00E94A85A612F70E06F7BDF
:10502000E12CF12C01E09E012F5F3F4F41E050E069
:10503000C6010E94DF0881E001C080E00F900F9060
:10504000DF91CF911F910F91FF90EF90DF90CF9064
:1050500008958F929F92AF92BF92CF92DF92EF927C
:10506000FF920F931F93CF93DF931F921F92CDB7A1
:10507000DEB76C017B0162E070E00E9412208C01BF
:1050800097FF03C080E090E099C063E070E0C60144
:105090000E941220AC011816190614F04FE350E0DC
:1050A000E982FA820130110531F48F2D880F880BC7
:1050B000F9828A8303C0023011052CF489819A8118
:1050C00099279A838983A981BA8124E630E00E94D6
:1050D00005779A01550F440B550B0E94AD76490197
:1050E0005A0189013A83298360E0C6010E94652044
:1050F000E82EF12CC6010E94EE1F092C000CAA0814
:10510000BB08681579058A059B0559F4012BE9F15F
:1051100082E0E816F10459F085E0E816F104A9F5FB
:1051200006C0012B71F182E0E816F10479F500E088
:1051300020E030E040E050E061E070E0C6010E9415
:10514000C45F00E09E012F5F3F4F41E050E060E010
:1051500070E0C6010E94C45F86E0E816F10439F0F1
:10516000EA94EF2821F061E0C6010E9440204981C5
:105170005A81052E000C660B770BC6010E94B61FE4
:1051800004C085E0E816F10431F418C085E0E816A3
:10519000F104B9F6CCCF82E0E816F104B1F362E095
:1051A000C6010E94402000E020E030E040E050E0F6
:1051B00062E070E0C6010E94C45FE7CF0F900F90DD
:1051C000DF91CF911F910F91FF90EF90DF90CF90E3
:1051D000BF90AF909F908F900895CF92DF92EF9203
:1051E000FF920F93CF93DF9300D000D0CDB7DEB7FF
:1051F0007C0161E00E94652085FF40C0C82ED12C53
:10520000C7010E94EE1F382F292FF701808590E0FB
:105210008A30910528F5FC018827E654FF4F8F4F0F
:105220000C94EE7669837A83832F330F990B9C83DA
:105230008B83822F220F990B9E838D8300E09E012A
:105240002F5F3F4F43E050E008C07A83698300E05E
:105250009E012F5F3F4F41E050E060E070E006C0EC
:1052600000E020E030E040E050E0B601C7010E94DD
:10527000C45FB6016F7DC7010E94402026960FB61D
:10528000F894DEBF0FBECDBFDF91CF910F91FF909D
:10529000EF90DF90CF9008958F929F92AF92BF9240
:1052A000EF92FF920F931F93CF93DF938C017B01BB
:1052B00049015A010E94BC35EC01892BF9F083E0C9
:1052C000888789869A86AB86BC8688819981009773
:1052D00011F00E94B46CC7010E94D97A9983888327
:1052E000BE01C801DF91CF911F910F91FF90EF9008
:1052F000BF90AF909F908F900C949F37DF91CF918C
:105300001F910F91FF90EF90BF90AF909F908F9063
:105310000895FB0101900020E9F73197AF01461B8A
:10532000570B20E00C9494270F931F93CF93DF9398
:10533000EC012097F9F00A811B81888587FD06C062
:105340008E819F81009711F00E9494298885843076
:1053500031F489859A85009711F00E94B46C888198
:105360009981009711F00E94B46CCE010E94B46C38
:10537000E801DFCFDF91CF911F910F9108950F9337
:105380001F93CF93DF93009791F08C010E94BC355F
:10539000EC01892B61F0C8010E94E334BE01C80111
:1053A0000E94C222019631F4CE010E94942980E02D
:1053B00090E001C0CE01DF91CF911F910F91089530
:1053C000CF93C82F462F61E070E00E94514461E006
:1053D00070E08C2F0E9427458111F9CFCF9108955D
:1053E00020E5FC01208311820895FC01848584302E
:1053F00011F00C94B74680E008958F929F92AF927F
:10540000BF92CF92DF92EF92FF920F931F93CF93B1
:10541000DF936B017C01142F9B01AC010E949A79F0
:10542000882319F061E874E027C046015701E89429
:10543000B7F82FEF3FEF4FE75FE7C501B4010E94D8
:105440009A7981110DC02FEF3FEF4FE75FE7C5015C
:10545000B4010E94797718161CF465E874E00CC05A
:105460002FEF3FEF4FE75FE4C701B6010E94D87806
:10547000181694F469E874E087EB97E0DF91CF9118
:105480001F910F91FF90EF90DF90CF90BF90AF9062
:105490009F908F900C94CC5A2FEF3FEF4FE75FEC2B
:1054A000C701B6010E94797787FDE4CF20E030E0A4
:1054B000A901C701B6010E94797787FF0BC06DE291
:1054C00087EB97E00E94635AEC01F7FAF094F7F843
:1054D000F09402C0C0E0D0E000E060E070E080E066
:1054E0009FE3101741F020E030E040E251E40E94D9
:1054F0007E770F5FF6CFA70196010E940D776B01B3
:105500007C010E94F7774B015C012AE0AB01BC01F2
:1055100087EB97E00E94E15AC80FD91F1123C9F108
:10552000C501B4010E9426789B01AC01C701B601F8
:105530000E940C776B017C016EE287EB97E00E9482
:10554000635AC80FD91F20E030E040E251E4C701A0
:10555000B6010E94DD784B015C010E94F7776B0178
:10556000E12CF12C2AE0B701A60187EB97E00E941D
:10557000E15AC80FD91FC701B6010E9426789B01C6
:10558000AC01C501B4010E940C776B017C01115084
:10559000D1F6CE01DF91CF911F910F91FF90EF9047
:1055A000DF90CF90BF90AF909F908F90089560E074
:1055B0008DE00C94004161E08DE00C9400410F936C
:1055C0001F93CF93DF93EB018CE99AE09F938F9326
:1055D0008BE99AE09F938F938AE99AE09F938F9348
:1055E00089E99AE09F938F9388E99AE09F938F933C
:1055F00087E99AE09F938F938DE894E09F938F9330
:105600008B818F938A818F930E94E47B2DB73EB765
:10561000205F3F4F0FB6F8943EBF0FBE2DBF0697D9
:1056200094F40A80DB81C02D62E47AE087EB97E096
:105630000E94A85ABE0187EB97E0DF91CF911F919E
:105640000F910C94765B0E940E5F07E91AE0C0E0B0
:10565000D0E0F80161918F01CE010E946D76219614
:10566000C630D105B1F764E57AE087EB97E0DF91CA
:10567000CF911F910F910C94A85A2F923F924F9265
:105680005F926F927F928F929F92AF92BF92CF92D2
:10569000DF92EF92FF920F931F93CF93DF93CDB7DB
:1056A000DEB7CD55D1090FB6F894DEBF0FBECDBF22
:1056B00000910F06109110060115110509F4A0C202
:1056C0000E944F62C0901506D0901606E090170613
:1056D000F0901806C616D706E806F90608F08AC044
:1056E000F801A680B780A114B10409F474C0F501D3
:1056F0008085863009F06BC06396BFAEAEAE63970F
:10570000CE018F5A9F4F0E94CC216596DFAC6597E2
:10571000DD2009F45CC067968EAD9FAD6797892B3D
:1057200009F455C06496FFAC6497F0E4FF1609F4E1
:105730009DC0FF1508F496C023E0C22ECF1408F4D4
:1057400046C0F1FC66C110E062E08D2D0E94D96177
:1057500065962FAD659730E0F901E455F34F8491DC
:10576000F901E45FF24F0491F901EE5AF24FF4901F
:10577000FF2009F451C181110E948361EF2DF0E0F7
:10578000EE0FFF1FEE58F34FA591B491EC910E234D
:1057900031E020E009F430E0832F922F212F30E018
:1057A00051E02817390709F050E0052F10E06796FF
:1057B000EEADFFAD6797628173810617170709F495
:1057C0004BC14181442309F42AC141504183F50171
:1057D000A280B38088CF0E944F62DC01CB01C296C9
:1057E000A11DB11D8093150690931606A093170670
:1057F000B09318060E944F62009111061091120694
:105800002091130630911406061717072807390749
:1058100008F0F6C1E0910F06F0911006068117819D
:105820000115110571F0F8018085863031F41A8375
:105830000983CE0101960E94CC21F80102811381D7
:10584000EFCF0E944F62DC01CB0188579C4EAF4FD7
:10585000BF4F8093110690931206A0931306B09346
:105860001406CEC192E4E92EFE10B1CF62EA74E0D4
:1058700063968EAD9FAD63970E947D378C01F1FCDE
:1058800002C062E001C060E08D2D0E94D961659682
:105890008FAD6597863308F0865390917B00282F53
:1058A0002870977F922B90937B0087708064809301
:1058B0007C0080917A00806480937A0080917A00E5
:1058C00086FDFCCFC090780080917900D12CD82A39
:1058D0000115110509F4DCC0F8018085853009F057
:1058E000D7C0C8010E94123B6E968FAF6E9784306E
:1058F00008F45EC063E0C8010E947037FC01818437
:10590000928462E0C8010E947037FC014184528495
:105910006384748461E0C8010E9470371C0160E0F8
:10592000C8010E947037FC0121853285438554856A
:105930006D962CAF3DAF4EAF5FAF6D97C601DD0CDE
:10594000AA0BBB0B9C01AD016D96CCACDDACEEACF3
:10595000FFAC6D972C193D094E095F09C401092C54
:10596000000CAA0BBB0BBC01CD016419750986099B
:1059700097090E947B76F101218532854385548504
:105980002C193D094E095F090E94AD76420E531E47
:10599000641E751E62016E96FFAD6E97F53041F480
:1059A00064E0C8010E947037FC018185928502C0C5
:1059B00081E090E08C149D040CF464016E96FFADC0
:1059C0006E97F23009F066C00D2C000CEE08FF084F
:1059D00060E0C8010E947037FC0181859285A38533
:1059E000B485C816D906EA06FB06D4F161E0C80101
:1059F0000E947037FC0181859285A385B4858C1542
:105A00009D05AE05BF050CF0E2CECC24C394D12C8D
:105A100029C011E060E099CE80E090E0BFCE6496AE
:105A20004FAD649740FF0AC02817390771F461E051
:105A30008081811160E0608370E002C05083B80112
:105A4000CE018F5A9F4F0E94E2206796EEADFFADC8
:105A5000679713830283BBCE33E0C32EC182B7CED8
:105A6000C12CD12C6796EEADFFAD679782819381F3
:105A70008C159D0519F1B601CE018F5A9F4F0E94DA
:105A8000E2206796EEADFFAD6797D382C28216C063
:105A900081E090E06796EEADFFAD6797228133819C
:105AA000A601421B530B9A0157FF03C03195219564
:105AB0003109821793070CF094C011826796EEADFE
:105AC000FFAD6797818185300CF081CE8281938113
:105AD0008C159D0509F47BCE6996DFAECEAE699735
:105AE00065961FAD65976EE87CE087EB97E00E94B6
:105AF000A85A612F87EB97E00E9498376CE87CE00A
:105B000087EB97E00E94A85AB60187EB97E00E94C6
:105B1000563787EB97E00E94725B63960EAD1FAD20
:105B2000639760E574E0C8010E947D373C016FE532
:105B300074E0C8010E947D378C01009769F1FC0177
:105B40006185728540E450E0CE0101960E94697B38
:105B50006FE270E0CE0101960E94307B892B51F4F8
:105B6000F8012185328543E050E060E4CE010196E2
:105B70000E94194D4AE0BE016F5B7F4F69968EAD62
:105B80009FAD69970E94666F0E94D226882321F0FC
:105B90008091A505882361F161147104D9F0F301A6
:105BA00061857285CE0101960E94D125CE010196B4
:105BB0000E94A91F882371F0E12CF12C01E09E01C5
:105BC000295A3F4F41E050E060E070E0CE0101967D
:105BD0000E94DF086796EEADFFAD6797D382C28261
:105BE000F6CD818186300CF069CF8F5F818366CFDF
:105BF000BE016F5B7F4FCE0101960E94E427CCCFA0
:105C0000C35ADF4F0FB6F894DEBF0FBECDBFDF9192
:105C1000CF911F910F91FF90EF90DF90CF90BF90A9
:105C2000AF909F908F907F906F905F904F903F903C
:105C30002F900895A8950E946411029724F00E9465
:105C400029540E943D2B0C9434228091A5058F5F2E
:105C50008093A505A8950E943D2B8091A5058150B4
:105C60008093A505089560E57CE087EB97E00E94AE
:105C7000A85A6DE37CE087EB97E00E94A85A6FE298
:105C80007CE087EB97E00E94A85A67E27CE087EB14
:105C900097E00E94A85A87EB97E00E94725B6AE146
:105CA0007CE087EB97E00E94A85A6AE07CE087EBF3
:105CB00097E00E94A85A6EEF7BE087EB97E00E9486
:105CC000A85A67EE7BE087EB97E00E94A85A65ED43
:105CD0007BE087EB97E00E94A85A60EC7BE087EBC3
:105CE00097E00E94A85A61EB7BE087EB97E00E9467
:105CF000A85A69EA7BE087EB97E00E94A85A6EE910
:105D00007BE087EB97E00E94A85A64E97BE087EB91
:105D100097E00E94A85A6CE87BE087EB97E00E942E
:105D2000A85A60E87BE087EB97E00E94A85A66E6F5
:105D30007BE087EB97E00E94A85A67E47BE087EB63
:105D400097E00E94A85A87EB97E00C94725BAF92A1
:105D5000BF92CF92DF92EF92FF920F931F93CF9358
:105D6000DF936C017B018A010E94657681508E3F32
:105D7000A0F45701C0E0D0E001501109C017D107CD
:105D80007CF4C6018C0F9D1F0E946576F5018193FE
:105D90005F01882329F02196F1CF80E090E005C0D3
:105DA000CE0DDF1D188281E090E0DF91CF911F9131
:105DB0000F91FF90EF90DF90CF90BF90AF9008953C
:105DC000CF92DF92EF92FF920F931F93CF93DF93C7
:105DD0006C01EB0109900020E9F72197C61BD70B56
:105DE000C032D10514F0CFE1D0E08B01E12CF12CD1
:105DF000EC16FD0664F4F80161918F01C7018C0D6A
:105E00009D1D0E946D76FFEFEF1AFF0AF1CF60E053
:105E1000C6018C0F9D1FDF91CF911F910F91FF90B5
:105E2000EF90DF90CF900C946D76882319F06DE59C
:105E30007AE002C06FE57AE087EB97E00C94A85A0D
:105E4000AF92BF92CF92DF92EF92FF920F931F9388
:105E5000CF93DF93CDB7DEB7C856D1090FB6F8940C
:105E6000DEBF0FBECDBF1AA619A6FE01BB962EE15E
:105E7000DF011D922A95E9F78E01075D1F4F0297FA
:105E800074F0FB01628173814FE150E0C8010E9410
:105E9000697BB80186E190E00E94E02E10C040E2EC
:105EA00050E0B80186E190E00E94A72E892B39F4DA
:105EB00040E250E06BE37BE0C8010E942C6F8091D0
:105EC0009C0A1F928F9380919B0A1F928F938091BF
:105ED0009A0A1F928F938091990A1F928F938091B3
:105EE000980A1F928F938091970A1F928F9386EA48
:105EF00094E09F938F931F9288E28F93CE01019637
:105F00006C019F938F930E94787B67E27BE087EB25
:105F100097E00E94A85AB80187EB97E00E94765B51
:105F2000B60187EB97E00E94765B87EB97E00E94D3
:105F3000725B0FB6F894A895809160008861809399
:105F40006000109260000FBE7E0199E4E90EF11C22
:105F5000D70113961C921E92129788EE93E0A0E050
:105F6000B0E0F70184839583A683B78384E08487B8
:105F70008BEF92E09183808316870587108A1786BE
:105F800080E590E0928B818B158A63E373E38FEE5B
:105F900095E30E94AA6F8C010FB6F894DEBF0FBE86
:105FA000CDBF892BE1F183E090E00E941C6CD80109
:105FB0001D969C938E931C97FC01F182E0821282C5
:105FC000C7010E947143882319F0C7010E94D84479
:105FD000D7011F966D917C9150975196AD90BC90D2
:105FE00052976115710569F0CE01815A9F4F0E9449
:105FF000785BA501BE01615A7F4FC7010E94B44979
:1060000007C0F70165857685A501C7010E94C64DC9
:10601000181619060CF49AC0C8010E94C83500E091
:1060200010E0F701E388F48899E288E10FB6F8946C
:10603000A895809360000FBE909360000115110534
:1060400009F465C0F8ECEF16F10409F054C06BE1F7
:106050007BE087EB97E00E94A85AA3961FAE1EAE86
:10606000A397A5961FAE1EAEA5978FEF9FEFA7969D
:106070009FAF8EAFA79789E792E0A1969FAF8EAFB3
:10608000A197A9961FAF0EAFA997F8940E94685FD9
:10609000CE01815A9F4F0E94BF2990930E06809394
:1060A0000D067894C8010E94C83580910D06909124
:1060B0000E06892B79F464E07BE087EB97E00E9481
:1060C000A85A0E944F62DC01CB018856954CAF4F15
:1060D000BF4F31C069EF7AE087EB97E00E94A85A82
:1060E0000E942D5062EF7AE087EB97E00E94A85A59
:1060F00082E090E0CBC06AED7AE087EB97E00E9407
:10610000A85AB70187EB97E00E9456370CC068EC9D
:106110007AE087EB97E00E94A85A6FEA7AE087EB73
:1061200097E00E94A85A0E944F62DC01CB01885779
:106130009C4EAF4FBF4F8093090690930A06A093E1
:106140000B06B0930C0685EF9FEFA0C0D7011D96FC
:10615000BC901D971E96AC90DF92CF928BEA9AE08E
:106160009F938F931F930F930E943370DF92CF9270
:1061700086EA9AE09F938F931F930F930E94337048
:10618000D8011C96ED91FC911D9781E08283DF92EE
:10619000CF9283EA9AE09F938F931F930F930E946D
:1061A0003370D8011C96ED91FC911D971282AF922D
:1061B000BF928DE69AE09F938F931F930F930E9457
:1061C000337088EA9AE09F938F931F930F930E94F6
:1061D0003370F701148A138AD8011C96ED91FC9153
:1061E0001D97A080B1800FB6F894DEBF0FBECDBF63
:1061F00083E3C82ED12CD501ED91FC910084F1856B
:10620000E02DC501199541975CF4B1E0CB1AD10896
:1062100039F064E170E080E090E00E941562EBCF1D
:106220006E01FFE5CF0ED11CDF92CF9281E69AE09E
:106230009F938F931F930F930E9450700F900F9016
:106240000F900F900F900F90019709F0EACEF60192
:1062500080819181D70154969C938E935397D12C32
:1062600080E08A3039F4BAE0DB1609F4DACE9AE03D
:10627000D92E03C08D3009F0D82EC8010E94F56FC9
:106280008F3F79F7C8010E94C835CBCEC859DF4F80
:106290000FB6F894DEBF0FBECDBFDF91CF911F9137
:1062A0000F91FF90EF90DF90CF90BF90AF90089547
:1062B0000E94202F9093A9058093A8058DE19AE074
:1062C0000C94D844CF93DF93EC01E881F9810284E8
:1062D000F385E02DCE0119950196B9F7DF91CF91A5
:1062E0000895FC01A285B3851097A9F0868597854E
:1062F000029788F0CD010196938782876C938685FB
:1063000097850197978786870284F385E02D108211
:1063100081E090E0089580E090E00895FC0186819E
:1063200097818F3F2FEF920729F02FEF3FEF3783B1
:1063300026830895A085B185109789F02485358539
:106340002115310561F0CD010196918780878C91EF
:106350002150310935872487082E000C990B0895A8
:10636000FC0186819781019639F481E02485358589
:10637000232B19F480E0089581E00895CF92DF92F5
:10638000EF92FF920F931F93CF93DF937C016A01EB
:106390008B01C0E0D0E0CC15DD0589F0D701ED918F
:1063A000FC910284F385E02DC70119958F3FBFEF63
:1063B0009B0729F0F80181938F012196ECCFCE0144
:1063C000DF91CF911F910F91FF90EF90DF90CF90D1
:1063D0000895CF93C62FDC01ED91FC910088F189DF
:1063E000E02D1995DC01ED91FC910190F081E02DFB
:1063F0006C2FCF911994CF93DF93EC018E819F8105
:106400000196D9F4288539858A859B85820F931F4B
:1064100081159041A0F4E881F9810284F385E02D93
:10642000CE011995813291056CF3E881F9810684DA
:10643000F785E02D682FCE01199581E001C080E03D
:10644000DF91CF910895062E000C770BFC01778326
:1064500066830895CF93DF93EC018E819F8101962F
:1064600011F5E881F9810088F189E02DCE011995B7
:10647000DC01ED91FC910084F185E02D1995892BCB
:10648000A1F0E881F9810284F385E02DCE01199510
:106490008132910534F3E881F9810684F785E02D96
:1064A000682FCE01199581E001C080E0DF91CF9186
:1064B00008950F931F93CF93DF93EC018B0161ED50
:1064C00074E00E94765B01151105B9F1F801619144
:1064D0008F01662391F1603220F0623211F06C3549
:1064E00041F56CE5CE010E94635AF8013197808135
:1064F0008C30D1F044F48930D9F08A30B9F088304A
:1065000029F762E616C0823259F024F48D30F1F694
:1065100062E70FC08F3231F08C35C1F66CE509C0EF
:1065200062E207C06FE205C066E603C06EE601C026
:1065300064E7CE010E94635AC9CF62E2CE010E9495
:10654000635A80E090E0DF91CF911F910F91089501
:10655000FC012085318582859385AC014F5F5F4FBB
:1065600053874287820F931F0E946D7681E090E0EF
:106570000895FC01868197818F3F2FEF920729F0C4
:106580002FEF3FEF3783268308952085318582855D
:106590009385AC014F5F5F4F53874287820F931FF4
:1065A0000E946576082E000C990B0895FC018681E7
:1065B00097818F3F2FEF920729F02FEF3FEF37831F
:1065C00026830895808591850C94F56FCF92DF9294
:1065D000EF92FF92CF93DF93EC018E819F818F3FEB
:1065E0002FEF920759F02FEF3FEF3F832E83DF917C
:1065F000CF91FF90EF90DF90CF9008950E944F626F
:106600006B017C01A4EFCA0EA1E0DA1EE11CF11CB3
:10661000E881F9810088F189E02DCE011995DC012E
:10662000ED91FC910084F185E02D1995892B39F4C9
:106630000E944F626C157D058E059F0548F3E88129
:10664000F9810088F189E02DCE011995DC01ED91E9
:10665000FC910284F385E02DDF91CF91FF90EF90C4
:10666000DF90CF901994EF92FF920F931F93CF93E7
:10667000DF93009719F48FEF9FEF80C0FC01E48453
:10668000F584D7010D911C91D801ED91FC910688FC
:10669000F789E02DC8011995882369F3D801ED9198
:1066A000FC910084F185E02DC8011995D801ED9188
:1066B000FC91892B61F30284F385E02DC8011995C3
:1066C000EC010196C1F2F8018589882329F06C2F2D
:1066D00087EB97E00E949837D70112968C91882318
:1066E00009F44BC0C532D10509F047C0D801ED917E
:1066F000FC910084F185E02DC801199502975CF0AA
:10670000D801ED91FC910688F789E02DC801199513
:106710008111ECCFB0CFD1E0C0E0D801ED91FC9178
:106720000284F385E02DC80119958F3FBFEF9B07C9
:1067300009F4A1CF9C01215431092A31310530F0EF
:106740009C01215631092A31310538F48D2F82956B
:10675000807F829FC00D11240AC0C0978A309105A6
:1067600030F49D2F9295907F989FC00D1124D150A9
:10677000A0F68C2FCC0F990B01C0CE01DF91CF91E9
:106780001F910F91FF90EF9008958F929F92AF927B
:10679000BF92CF92DF92EF92FF920F931F93CF930E
:1067A000DF936115710509F4FFC0FB010085002E20
:1067B000000C110B220B330B0730110508F0F4C04D
:1067C000DB01EC01F8018827EC53FF4F8F4F0C944D
:1067D000EE7661E774E006C019968C91882389F003
:1067E0006CE774E0CE01DF91CF911F910F91FF9084
:1067F000EF90DF90CF90BF90AF909F908F900C94D0
:10680000CC5A66E774E0EECF19964D915D916D918B
:106810007C911C972AE030E0CE01DF91CF911F914F
:106820000F91FF90EF90DF90CF90BF90AF909F902F
:106830008F900C942A5B1996CD90DD90ED90FC9092
:106840001C9720E030E0A901C701B6010E947977CA
:1068500087FF09C063ED74E0CE010E94765BF7FA12
:10686000F094F7F8F094C701B6010E94F7774B0156
:106870005C012AE0AB01BC01CE010E94E15A65ED4A
:1068800074E0CE010E94765BC501B4010E942678B7
:106890009B01AC01C701B6010E940C772DEC3CECCA
:1068A0004CE45DE30E940D7720E030E040E251E4EB
:1068B0000E94DD780E94F777AB0160E070E02AE08B
:1068C000CE010E94E15A70C019966D917C911A9781
:1068D000CE01DF91CF911F910F91FF90EF90DF904C
:1068E000CF90BF90AF909F908F900C945932169696
:1068F0000D911C9117976BE5CE010E94635A01968A
:1069000019F48FEF9FEF52C00115110571F0B80116
:10691000CE010E94C5330196A1F3F80102811381D3
:106920000115110589F36CE2E7CF6DE52FC01696CE
:106930000D911C9117976BE7CE010E94635A019647
:1069400001F30115110509F1F80160817181CE0192
:106950000E9459320196A9F26AE3CE010E94635A5D
:10696000019679F2B801CE010E94C533019649F231
:10697000F801028113810115110519F36CE2CE01B2
:106980000E94635A0196E9F6BCCF6DE7CE010E94E2
:10699000635A21E030E0019611F020E030E08827D2
:1069A0009927821B930B02C080E090E0DF91CF918A
:1069B0001F910F91FF90EF90DF90CF90BF90AF901D
:1069C0009F908F900895CF93DF93EC01E881F98138
:1069D0000284F385E02DCE0119958F3F2FEF9207AA
:1069E00071F0E881F9818132910594F30684F7858D
:1069F000E02D682FCE01199580E090E002C08FEF66
:106A00009FEFDF91CF910895EF92FF920F931F9325
:106A1000CF93DF938C017B01DC01ED91FC9102842B
:106A2000F385E02D1995829709F078C084E0F7018D
:106A3000808786E090E00E941C6CEC01892B09F4B1
:106A40006DC0E9E1F6E0F983E88380E091E0DF01E1
:106A50009C011D9221503040E1F79B838A831D8267
:106A60001C82D801ED91FC910284F385E02DC801D0
:106A700019958F3FBFEF9B0709F44DC082329105F6
:106A800009F44FC0803291050CF44BC08C35910550
:106A900011F0BE013DC0D801ED91FC910284F38557
:106AA000E02DC80119958F3FBFEF9B07A1F18236FA
:106AB000910531F15CF48F329105F9F08C35910537
:106AC000C9F0829771F6BE0182E222C08E3691052E
:106AD000D1F034F48636910521F6BE018CE018C061
:106AE0008237910599F08437910509F0BACFBE013C
:106AF00089E00EC0BE018CE50BC0BE018FE208C06C
:106B0000BE0188E005C0BE018AE002C0BE018DE082
:106B10000E94195EA6CFCE010E94B46C8FEF9FEF4A
:106B200024C08C819D81009749F0E881F9818E0F06
:106B30009F1FFC0131978081882321F0BE0180E0F6
:106B40000E94195E8C819D810E941C6C8C010097B3
:106B500039F069E176E00E94447BCE010E94B46C7A
:106B6000F7011287018780E090E0DF91CF911F91BC
:106B70000F91FF90EF9008958DE090E00E941C6CC3
:106B8000009729F02DE0FC0111922A95E9F708956C
:106B90000F931F93CF93DF930097E1F0EC010C85E7
:106BA0001D850115110579F0D8018D919C910097F3
:106BB00039F0DC01ED91FC910488F589E02D1995FF
:106BC000C8010E94B46CCE01DF91CF911F910F914B
:106BD0000C94936FDF91CF911F910F910895AF9215
:106BE000BF92CF92DF92EF92FF920F931F93CF93BA
:106BF000DF9300D01F92CDB7DEB76115710509F4A0
:106C000096C06B01182FDB011C96AD90BC901D97B0
:106C1000F501E080F180D701ED91FC910688F789BC
:106C2000E02DC7011995811104C0C6010E94C83525
:106C30007EC0F5019281911114C0D701ED91FC91B4
:106C40000190F081E02D612FC7011995F701858929
:106C5000882309F469C0612F87EB97E00E94635A8B
:106C600063C0812F8F7D81548A3138F380ED810F8D
:106C70008A3018F383ED810F8230F8F21F35E9F284
:106C80001E37D9F21132B1F086EC810F823090F0CC
:106C90008AED810F873070F01D3361F0812F8F7E78
:106CA0008F3241F08DED810F823020F01B3511F0D5
:106CB0001D3511F491FFC1CF19821A821B821C82EB
:106CC000812F012E000C990B9F931F9387ED94E069
:106CD0009F938F938E010F5F1F4F1F930F930E94FF
:106CE000B57B6E01F4E0CF0ED11C0F900F900F908A
:106CF0000F900F900F90D701ED91FC910190F081D2
:106D0000E02DD8016C91C7011995F7018589882379
:106D100031F0D8016C9187EB97E00E94635A0F5FC6
:106D20001F4F0C151D0539F780E090E002C08FEF72
:106D30009FEF0F900F900F900F90DF91CF911F91C9
:106D40000F91FF90EF90DF90CF90BF90AF9008959C
:106D50002C9A08952C980895CF92DF92EF92FF928B
:106D60000F931F93CF93DF93EC017A018B016C019A
:106D7000C40ED51ECC15DD05A9F00E94AA368FE001
:106D80000E9495438D2F0E9495438C2F0E9495431E
:106D9000219680E00E949543F80181938F010E9423
:106DA000A836E8CFC701DF91CF911F910F91FF90D7
:106DB000EF90DF90CF900895CF92DF92EF92FF9205
:106DC0000F931F93CF93DF93EC017A018B016C013A
:106DD000C40ED51ECC15DD05A1F00E94AA3680EFA9
:106DE0000E9495438D2F0E9495438C2F0E949543BE
:106DF0002196F80181918F010E9495430E94A83647
:106E0000E9CFC701DF91CF911F910F91FF90EF90D4
:106E1000DF90CF9008951F93CF93DF93D82F192F32
:106E2000C62F0E94AA3680EF0E949543812F0E94B0
:106E300095438D2F0E9495438C2F0E9495430E946D
:106E4000A83681E0DF91CF911F9108951F93CF93D2
:106E5000DF93182F66E270E00E942745C82FD0E02C
:106E600067E270E0812F0E942745DC2FCC279E012E
:106E7000282BC901DF91CF911F9108951F93CF93C4
:106E8000DF93182F60E270E00E942745C82FD0E002
:106E900061E270E0812F0E942745DC2FCC279E0104
:106EA000282BC901DF91CF911F910895AB01770F76
:106EB000660B770B2AE030E00C942A5B0F931F934C
:106EC000CF93DF93EC010E94A85A8C01CE010E945F
:106ED000725B800F911FDF91CF911F910F910895E9
:106EE000FC0186819781009739F0662329F0615073
:106EF000FC0182819381F7CF08950F931F93CF9365
:106F0000DF938B01FC01C681D781209759F0B8012E
:106F1000888199810E94127B892B21F00A80DB8174
:106F2000C02DF3CFCE01DF91CF911F910F91089526
:106F3000462F50E060E070E02AE00C94E15ADC015A
:106F40001696ED91FC91179761157105A1F0309798
:106F500029F417967C936E931697089582819381F6
:106F6000009711F0FC01FACF73836283DB01159661
:106F7000FC93EE9314970895CF92DF92EF92FF92D5
:106F80000F931F93CF93DF938C017B016A010E94C3
:106F9000BC35EC01892B09F182E08887A601DD0C64
:106FA000660B770B49875A876B877C878881998125
:106FB000009711F00E94B46CC7010E94D97A99839E
:106FC0008883BE01C801DF91CF911F910F91FF907F
:106FD000EF90DF90CF900C949F37DF91CF911F916E
:106FE0000F91FF90EF90DF90CF900895CF92DF92B6
:106FF000EF92FF921F93CF93DF93EC016A017B0125
:10700000122FE889F98982E080834115514E61058C
:107010007105B1F060E079E08DE390E0A7019601A1
:107020000E948B76DA01C9010197A109B109B695D1
:10703000A795979587959C01211580E13807A8F0C1
:10704000E889F989108260E874E88EE190E0A70190
:1070500096010E948B76DA01C9010197A109B10955
:10706000B695A795979587959C01EC85FD8530830E
:10707000EE85FF852083188EEC89FD891083EA89CF
:10708000FB89808180618083EA89FB8980818860B7
:107090008083EA89FB89808180688083EA89FB8913
:1070A00080818F7D8083DF91CF911F91FF90EF9042
:1070B000DF90CF9008958F929F92AF92BF92CF9220
:1070C000DF92EF92FF920F931F93CF93DF93CDB791
:1070D000DEB7DA950FB6F894DEBF0FBECDBFC82E6F
:1070E000809105098983CA8221E0C216A0F074E06C
:1070F0007C1518F487E1C8120EC0809106099091A2
:1071000007099B838C8380910809909109099D83CD
:107110008E8386E001C082E08E010F5F1F4F90E1F9
:107120009C1528F0AFE0CA1630F49BEF01C09AEE30
:107130009C0D923078F420918A0990918B09F80186
:10714000E80FF11D908391E0980FF801E90FF11D10
:107150008E5F2083BFE0CB1641F1BC1558F0E5E00F
:10716000CE16A1F0F6E0CF12B6C020918E09909114
:107170008F0910C026E1C21609F48EC077E1C71648
:1071800009F459C090E1C912A6C055C020918C09DC
:1071900090918D09F801E80FF11D908391E0980F0F
:1071A000F801E90FF11D8E5F95C020918C09309197
:1071B0008D09F801E80FF11D308342E0480F91E09E
:1071C000980FF801E90FF11D2083B9016770772747
:1071D000A3E036952795AA95E1F7672B19F091E082
:1071E000920F01C0922FB3E0B80FF801E40FF11D28
:1071F00090838C5F60E070E0A0E04FEF480F9A133F
:1072000003C08B2F890F67C050E09B0135952795F0
:10721000400F511F220F331FF901E257F64FA0FD17
:1072200002C0208101C02181FA012083AF5F6F5F1E
:107230007F4F8F5FE2CF20918C0930918D09F8014B
:10724000E80FF11D308391E0980FF801E90FF11D6F
:10725000208392E0980FF801E90FF11D8D5F922FC6
:10726000990F908390E03327E92FF0E0E217F307BE
:1072700094F5EE0FFF1FE257F64F50814181F80160
:10728000E80FF11D408341E0480FF801E40FF11DC4
:107290008E5F50839F5FE8CF90918E0920918F0978
:1072A000F801E80FF11D208321E0280FF801E20F1B
:1072B000F11D9083209190099091910932E0380F4F
:1072C000F801E30FF11D908393E0980FF801E90FA7
:1072D000F11D8C5F20837801F8012FEF3FEFD02E56
:1072E0009E2F901B9817A0F49191292748E050E019
:1072F000B9017695679520FF06C09B0191E029278B
:1073000090EA392701C09B014150510989F7E8CF24
:10731000F801E80FF11D2083B2E0BB2EB80E8F5F9D
:10732000F801E80FF11D3083F801EB0DF11D10821B
:107330008091030990910409DC01ED91FC91028494
:10734000F385E02D1995019699F7E091190AF091CE
:107350001A0A309709F01995809103099091040950
:107360002E2D2D192B1558F4F70161917F01DC01A9
:10737000ED91FC910190F081E02D1995EDCFDC01AC
:10738000ED91FC910680F781E02D1995E0911B0AA3
:10739000F0911C0A309709F019950E944F624B0139
:1073A0005C01A8E0EA2EF12CD12C80910309909188
:1073B0000409DC01ED91FC910084F185E02D199523
:1073C000892BC1F08091030990910409DC01ED91B2
:1073D000FC910284F385E02D199590910509891798
:1073E00011F0FF2099F1F801EF0DF11D8083EA946F
:1073F000F39407C0E091170AF091180A309709F04A
:107400001995B5E0FB1222C0EA818E2F8F7790E0AC
:107410008C159D0509F0A2C0E7FF04C08B8188236D
:1074200081F181C08E2F90E0FC013197E731F105A9
:1074300068F48827E553FF4F8F4F0C94EE76F3E006
:10744000EF2E04C0EB8002C0E5E0EE2E0E944F62FA
:10745000DC01CB0188199909AA09BB09813D974034
:10746000A105B10538F480E0EE2031F0882309F45D
:107470009CCF59C082EEF8CF811155C0F4E0FF15C2
:10748000C0F58FEF9FEF60E0EF2DF0E09F012250FD
:107490003109462F50E0D80142175307BCF4A40F1E
:1074A000B51F4C91842748E050E0DC01B695A795C4
:1074B00080FF06C0CD0171E0872770EA972701C0E1
:1074C000CD014150510989F76F5FE3CFA20FB31F80
:1074D0002C9130E0AC0155274217530709F040C00A
:1074E000892F9927EC0FFD1F208130E08217930729
:1074F000B9F58A818530B0F58330B0F5813090F0F0
:107500005B81652F70E0759567952091160A40E0C4
:10751000842F90E0861797070CF452C02093160A28
:1075200050FD6CC080E01092100A1092120A109266
:10753000110A1092150AD3950FB6F894DEBF0FBE4C
:10754000CDBFDF91CF911F910F91FF90EF90DF9012
:10755000CF90BF90AF909F908F90089581EEE3CF32
:1075600083EEE1CF8731F1F66B8170E07595679519
:107570002091160A40E0842F90E0861797071CF0B0
:107580002093160ACFCF4034C0F49C012E5F3F4FAA
:10759000220F331F880F991FFC01ED5FF64FDE01AC
:1075A000A20FB31F8C9190E0982F8827D801A20FCB
:1075B000B31F2C91822B90878783242F4F5FDBCFC3
:1075C0004034C8F4880F991FFC01ED5FF64FA5E029
:1075D000B0E0AC0FBD1FA80FB91F2C9130E0322FC7
:1075E0002227A4E0B0E0AC0FBD1FA80FB91F8C91FB
:1075F000282B30872783242F4F5F8ACF403468F4AD
:10760000880F991FFC01ED5FF64FDE01A80FB91F2F
:1076100014968C9190E09087878381E0840F80930B
:10762000160A80CFDC011696ED91FC91179780E049
:10763000309729F08F5F0280F381E02DF9CF089514
:107640007F928F929F92AF92BF92CF92DF92EF92F2
:10765000FF920F931F93CF93DF93CDB7DEB7A6971B
:107660000FB6F894DEBF0FBECDBF8C01762E942EE0
:10767000852E20E2B22ECE0101967C01FC012B2D3D
:1076800011922A95E9F781E293E09AA389A38FEFFB
:107690008BA38CA38DA38EA3680183E4C80ED11C99
:1076A00043E450E0BE016F5D7F4FC6010E94D647A4
:1076B000019609F4B9C081E089838A8386E0A82E07
:1076C000AB821C82F80164817581868197810E945A
:1076D000F6766D837E838F83988789869A8680E885
:1076E00090E09C878B874CE150E0B701C6010E9477
:1076F0002B43F7012B2D11922A95E9F7480188E0D9
:10770000880E911CF401D70101900D92AA94E1F723
:1077100040E150E0B701C6010E942B43F7011192EE
:10772000BA94E9F796E0A92EB12C40E250E0B701F7
:10773000C6010E942B43F1E0AF1AB108B1F783E60E
:10774000898392E89A8393E59B838C8385E38D8379
:1077500081E08E837F829DE3988797E099878A876F
:1077600086E0F401DE011B9601900D928A95E1F707
:107770008CE0898B8A8B6DED74E0CE0143960E947C
:10778000447BF8016385CE0149960E940857F801B1
:107790006485CE014B960E940857F8016585CE019D
:1077A0004D960E9408574EE150E0B701C6010E9475
:1077B0002B43F3E07F121EC082E3898384E08A8337
:1077C000F80196859B8397859C8390899D839189F9
:1077D0009E8396E39F838887828D8987838D8A879E
:1077E000848D8B87858D8C874CE050E0B701C60176
:1077F0000E942B4387E3898386E08A8391E09B8301
:1078000093E09C838D838FE08E838AE38F838BE369
:1078100088878FEF898749E050E0B701C6010E9451
:107820002B43C6010E940347A6960FB6F894DEBF0D
:107830000FBECDBFDF91CF911F910F91FF90EF90C1
:10784000DF90CF90BF90AF909F908F907F900895E2
:107850002F923F924F925F926F927F928F929F9260
:10786000AF92BF92CF92DF92EF92FF920F931F934E
:10787000CF93DF9300D000D0CDB7DEB78C010E944C
:10788000886D2FEC37E040E050E00E94AD76DC01DF
:10789000CB010196A11DB11DF80184839583A683B8
:1078A000B78380839183A283B3835801F3E4AF0E3F
:1078B000B11CC5010E94CA4464E470E0C5010E9485
:1078C000D646882309F436C10E944F622B013C0141
:1078D000812C912CC8018E5B9F4F9E838D8348EE37
:1078E000C42E43E0D42EE12CF12C52E0252EAD81A4
:1078F000BE818C91833009F404C1811120C0F8014C
:1079000084819581A681B7810196A11DB11D8483D3
:107910009583A683B7830E944F626419750986090F
:107920009709A70196010E948B76A90161E0C80121
:107930000E94203B81E0AD81BE818C93CAC084301F
:10794000F9F4F80184819581A681B7810196A11D82
:10795000B11D84839583A683B7830E944F62641907
:10796000750986099709A70196010E948B76A901DE
:1079700063E0C8010E94203BAD81BE812C92A9C06A
:10798000813059F5F80142AD53AD64AD75AD9E013E
:107990002F5F3F4FC8010E941D57382EF2E08F1312
:1079A00092C089819A81AB81BC81F80184839583DF
:1079B000A683B7830E944F626419750986099709E7
:1079C000A70196010E948B76A90163E0C8010E947D
:1079D000203BAD81BE813C927CC0823009F079C0F1
:1079E000F80142AD53AD64AD75AD9E012F5F3F4FC1
:1079F000C8010E941D57382EF5E08F135DC0E3E0EB
:107A0000AD81BE81EC93F80182A193A1A4A1B5A19F
:107A1000892B8A2B8B2B41F484E893E0A0E0B0E023
:107A200082A393A3A4A3B5A3F80186A197A1A0A5BF
:107A3000B1A5892B8A2B8B2B61F482A193A1A4A1E0
:107A4000B5A1B695A7959795879586A397A3A0A767
:107A5000B1A7F80182A593A5A4A5B5A5892B8A2B6A
:107A60008B2BA9F482A193A1A4A1B5A1AC01BD0166
:107A700023E076956795579547952A95D1F7841B0E
:107A8000950BA60BB70B82A793A7A4A7B5A7F801E0
:107A900086A197A1A0A5B1A586A797A7A0ABB1ABDA
:107AA00082A593A5A4A5B5A582AB93ABA4ABB5ABBA
:107AB00088248394912C0DC0F6E08F1304C0AD810F
:107AC000BE811C9206C0BFEF3B1203C0ED81FE8158
:107AD0001082F1E08F16910409F409CF0E944F62E1
:107AE000DC01CB0184199509A609B709F80126A97B
:107AF00037A940AD51AD281739074A075B0708F091
:107B0000F6CEC5010E94CA44F80184819581A68100
:107B1000B7810196A11DB11D84839583A683B78388
:107B20000E944F62F801FE96608371838283938383
:107B3000C40102C080E090E026960FB6F894DEBF44
:107B40000FBECDBFDF91CF911F910F91FF90EF90AE
:107B5000DF90CF90BF90AF909F908F907F906F906D
:107B60005F904F903F902F900895CF93DF93FC014B
:107B700001900020E9F79F01281B390B285F3F4F38
:107B80002138310570F5EC010E94D226882349F195
:107B90008091E8089091E908019611F481E090E065
:107BA0009093E9088093E8088091E8089091E908AB
:107BB00090936D0880936E0847E050E068E678E0A7
:107BC000CE010E940B27FC01EE59F74F1682AC0143
:107BD0004450510968E678E082E8DF91CF910C9437
:107BE0002B2780E0DF91CF910895CF92DF92EF9223
:107BF000FF920F931F93CF93DF936C018B017B0157
:107C000082E0E80EF11CC0E0D0E0C6018C0F9D1FA1
:107C10000E946576F70181937F012196C430D105DA
:107C2000A1F7F8019281992319F081E09F3F09F4AF
:107C300080E090E0DF91CF911F910F91FF90EF9046
:107C4000DF90CF900895EF92FF920F931F93CF9301
:107C5000DF937C018B010E5F1F4FC0E0D0E0F80185
:107C600061918F01C7018C0F9D1F0E946D76219637
:107C7000C430D105A1F7DF91CF911F910F91FF90F3
:107C8000EF900895FC01DC018D918111FDCF40E062
:107C900050E020E030E08AE09191992301F1243016
:107CA00031055CF59E3271F44F3F510509F02CF51A
:107CB000DB01A20FB31F12964C932F5F3F4F40E0A2
:107CC00050E0EACF849FD001859FB00D1124492F49
:107CD000990F550B405351094A0F5B1FDDCF4F3FA2
:107CE000510509F054F4243031053CF4FB01E20F56
:107CF000F31F428381E090E0089580E090E00895D2
:107D00004F925F926F927F928F929F92AF92BF92AB
:107D1000CF92DF92EF92FF920F931F93CF93DF9357
:107D2000CDB7DEB763970FB6F894DEBF0FBECDBFF9
:107D30007C015B013A01FB0120E080E090E06AE019
:107D40003191332309F140ED430F4A3080F4689FAD
:107D5000A001699F500D1124CA01C097830F911D86
:107D600037FD9A958F3F910559F350F313C03E327A
:107D700089F4233079F0D301A20FB11D12968C93B0
:107D80002F5F80E090E0DCCF233021F4F301858386
:107D900081E021C0F7014281538164817581809126
:107DA000560890915708A0915808B0915908481763
:107DB00059076A077B0709F499C10E944F6287013E
:107DC000085F1F4F6F7077277C5FC8010E94D646FF
:107DD000813019F080E090E0FCC181E293E09A8369
:107DE0008983F70182819381A481B5818B839C83F0
:107DF000AD83BE8345E350E0BE016F5F7F4FC80196
:107E00000E94D647892B19F4C12CD12C6AC10E943B
:107E10004F62F701778366837627672776277A8311
:107E2000698342E050E0BE016F5F7F4FC8010E944E
:107E30002B4381E090E09E878D8742E050E0BE01B9
:107E4000635F7F4FC8010E942B4380E091E09E87D3
:107E50008D8742E050E0BE01635F7F4FC8010E9402
:107E60002B431E861D8642E050E0BE01635F7F4FBC
:107E7000C8010E942B4342E050E0BE01635F7F4F88
:107E8000C8010E942B4342E050E0BE01635F7F4F78
:107E9000C8010E942B434501F5018081882301F12F
:107EA00064015601F60181912F01882321F08E3261
:107EB00011F06201F6CFC818D9081C141D0474F41F
:107EC000CF8641E050E0BE01615F7F4FC8010E9454
:107ED0002B43A601B401C8010E942B434201DCCF11
:107EE0001F8641E050E0BE01615F7F4FC8010E94E4
:107EF0002B43C12CDD24D394DE86CD8642E050E0B6
:107F0000BE01635F7F4FC8010E942B43DE86CD8692
:107F100042E050E0BE01635F7F4FC8010E942B43E7
:107F2000C8010E940347892B09F46ECFE3E0AE2E0F
:107F3000B12C230122E0420E511C0E944F623B01F2
:107F40004C01C8010E945D4618161906B4F00E9443
:107F50004F62DC01CB0186199709A809B909813A5A
:107F60009F40A105B105E0F40E94252E61E070E07C
:107F700080E090E00E941562E4CFF70142815381D6
:107F800064817581808D918DA28DB38D48175907BD
:107F90006A077B0749F4848D958DC59729F409C03C
:107FA000CC24CA94DC2C92C05EEFC52EDD24DA947A
:107FB0008DC0F70181A192A10C970CF49FC04CE0F9
:107FC00050E0BE016F5F7F4FC8010E9415468B8154
:107FD0009C819827892798279A8B898B29813A81B8
:107FE000322723273227F701468157812417350787
:107FF00009F07FC097FF7DC08F709270892B09F0C8
:10800000E3C06F8078847624672476246114710439
:1080100009F4D5C0C12CD12C8D819E819827892748
:108020009827C816D90608F46EC0812C912C41E01F
:1080300050E0BE016D5E7F4FC8010E9415468B89DE
:10804000982F907C09F091C0811185C042E050E0EA
:10805000BE01615F7F4FC8010E94154642E050E0BB
:10806000BE01635F7F4FC8010E941546C8010E9490
:108070003446C8010E943446C8010E943446C801F3
:108080000E94344642E050E0BE016F5E7F4FC8015F
:108090000E9415468F8598898115914009F06DC021
:1080A000CD84DE84DC24CD24DC2481E0C816D10418
:1080B00009F063C089899A898115944009F07AC0D2
:1080C00044E050E0B201C8010E9415460E94252EEE
:1080D00081E0A81AB10829F0FFEFCF16DF0609F4F6
:1080E0002CCFC8010E94CA44C60173C08EEF9FEF17
:1080F00070C04CEFC42EDD24DA94E8CF9DEFC92E7A
:10810000DD24DA94E3CF41E050E0BE01635F7F4FAE
:10811000C8010E9415468D85882351F08D859FEFFB
:10812000980F9D87882321F0C8010E943446F6CF1E
:108130008D858111E8CFC8010E943446C8010E9494
:108140003446C8010E943446C8010E943446FFEFFD
:10815000CF1ADF0A61CF8B899FEF980F9B8B882303
:1081600041F0C8010E943446F6CFC8010E9434464F
:108170001B8A8B8981115BCF69CFC12CD12C898956
:108180009A89982789279827C816D90638F4C801EC
:108190000E943446FFEFCF1ADF0AF1CF2FEF821A89
:1081A000920A6814790409F042CF26EFC22EDD242A
:1081B000DA948CCF77EFC72EDD24DA9487CF3AEFAD
:1081C000C32EDD24DA9482CF8BEFC82EDD24DA941F
:1081D0007DCF63960FB6F894DEBF0FBECDBFDF91A3
:1081E000CF911F910F91FF90EF90DF90CF90BF90B4
:1081F000AF909F908F907F906F905F904F90089579
:108200001F93CF93DF93282F30E0F901E455F34F0C
:108210008491F901E45FF24FD491F901EE5AF24FE3
:10822000C491CC23C1F0162F81110E948361EC2FE1
:10823000F0E0EE0FFF1FEE56F34FA591B4919FB7FC
:10824000F894111104C08C91D095D82302C0EC9100
:10825000DE2BDC939FBFDF91CF911F9108951F9379
:10826000CF93DF931F921F92CDB7DEB76CE271E020
:1082700080E090E00E9415621FB7F89480919D0AFB
:10828000811127C0E7E8FDE08491E1E4FDE09491ED
:10829000E82FF0E0EE0FFF1FEE50F34FA591B491E1
:1082A000EC91E92321F461E085E30E94004161E063
:1082B00085E30E94D9618CB580618CBD8CB58064EA
:1082C0008CBD61E084E30E94D96161E083E30E9498
:1082D000D96180919D0A8F5F80939D0A1FBF249A68
:1082E000CE0101960E94F02989819A810E94264937
:1082F00067E080E090E00E940B3765E58BE190E05D
:108300000E940B3765E58AE190E00E940B370E94DE
:10831000254980E090E49093F6058093F50580E090
:1083200090E69093FE058093FD0580E098E490939D
:10833000F8058093F70580E098E690930006809317
:10834000FF0580E090E59093FA058093F90580E0C1
:1083500090E7909302068093010680E098E5909361
:10836000FC058093FB0580E098E7909304068093DA
:1083700003060F900F90DF91CF911F910895AF9258
:10838000BF92CF92DF92EF92FF920F931F93CF9302
:10839000DF931F921F92CDB7DEB75C018B016A019C
:1083A00079010E942F41CE0101960E94F029898116
:1083B0009A810E94264946E050E067E97AE089E028
:1083C00090E00E94DC36C50102960E941049C60169
:1083D00002960E941E49C70102960E9417490E94F8
:1083E0002549F80182819381A481B58180935C083D
:1083F00090935D08A0935E08B0935F080F900F9074
:10840000DF91CF911F910F91FF90EF90DF90CF9070
:10841000BF90AF900895CF92DF92EF92FF92CF93EB
:10842000DF93CDB7DEB768970FB6F894DEBF0FBE07
:10843000CDBFFA0121E233E03A8329835FEF5B830A
:108440005C835D831E8238872F83C280D380E48063
:10845000F580C986DA86EB86FC863E872D87FB0190
:1084600042815381648175814F87588B698B7A8BE8
:108470003C8B2B8BFC0182819381A481B5818D8BF8
:108480009E8BAF8BB88F9E012F5F3F4FAE01495F30
:108490005F4FBE01635F7F4FCE0143960E94BF4195
:1084A00068960FB6F894DEBF0FBECDBFDF91CF91B7
:1084B000FF90EF90DF90CF9008950F931F93CF938D
:1084C000DF93CDB7DEB768970FB6F894DEBF0FBE67
:1084D000CDBFFB01DC0112964D915D916D917C91B8
:1084E00015974D8B5E8B6F8B788F81E293E09A832B
:1084F000898321E0288F0D891E892F89388D0B8370
:108500001C832D833E8398878F830281138124816E
:10851000358109871A872B873C879E878D874F87F0
:10852000588B698B7A8BAE014F5F5F4FBE01695FDD
:108530007F4FCE010D960E940B4268960FB6F894BD
:10854000DEBF0FBECDBFDF91CF911F910F91089578
:10855000CF93DF93CDB7DEB762970FB6F894DEBF47
:108560000FBECDBFFC0182819381A481B5818F872D
:10857000988BA98BBA8B21E233E03A83298341E0BF
:108580004A8B4F85588969897A894B835C836D83CF
:108590007E8338872F8389879A87AB87BC87BE0104
:1085A0006F5F7F4FCE0107960E945D4262960FB6C5
:1085B000F894DEBF0FBECDBFDF91CF91089508952F
:1085C000CF93DF931F92CDB7DEB76983DC01ED91C6
:1085D000FC910280F381E02D41E050E0BE016F5F2D
:1085E0007F4F19950F90DF91CF910895FC01818DF8
:1085F000928D0895FC0184899589089521E233E0E4
:10860000FC0131832083FB01408951896289738990
:10861000FC0142835383648375830895DC01ED91EB
:10862000FC91048CF58DE02D199480E00895FC01F7
:108630009485FB018485981303C081E0943009F48C
:1086400080E0089521E0FC018485843009F420E075
:10865000822F089508958F929F92AF92BF92DF92DA
:10866000EF92FF920F931F93CF93DF931F921F926E
:10867000CDB7DEB77C014B018A01FC01A688B78823
:10868000D08CCE0101960E94F02989819A810E94A6
:1086900026498D2D0E94EC568017910720F48D2DD0
:1086A0000E94EC568C019801A401B5018D2D0E9409
:1086B00087560E942549F70186899789800F911F67
:1086C000978B868BC8010F900F90DF91CF911F91F0
:1086D0000F91FF90EF90DF90BF90AF909F908F90A1
:1086E0000895CF93DF93FC0124852430D1F0EC0171
:1086F0000E94F529843181F0882371F0883161F07E
:108700008C3161F4E881F9810084F185E02DCE019E
:10871000199521E0892B19F420E001C021E0822F76
:1087200001C080E0DF91CF9108958EBD00000DB4AF
:1087300007FEFDCF8EB50895DF92EF92FF920F9363
:108740001F93CF93DF931F921F92CDB7DEB7D82E22
:10875000CE0101960E94F02989819A810E942649C2
:10876000E12CF12C8D2D0E9426378C01892B21F0D4
:108770008D2D0E9426377C010E151F0599F70E944A
:108780002549C8010F900F90DF91CF911F910F9154
:10879000FF90EF90DF900895FC011382128288EE23
:1087A00093E0A0E0B0E084839583A683B78383E35E
:1087B00093E09183808381E293E097878687108A94
:1087C000118A128A138A84E0808F0895AF92BF9233
:1087D000CF92DF92EF92FF920F931F93CF93DF938D
:1087E000CDB7DEB7AF970FB6F894DEBF0FBECDBFE3
:1087F0007C015B016A0101E213E01A8309831B8299
:108800001C821D821E82CE0109960E94CC431BA7AA
:108810000AA71CA61DA61EA61FA680915C08909103
:108820005D08A0915E08B0915F088EA39FA3A8A7E2
:10883000B9A78B839C83AD83BE8318861F82AE014C
:10884000465D5F4FB501CE0101960E94803E8130AA
:108850009105B1F4D701ED91FC910488F589E02DE3
:108860001DA30CA38CA59DA5AEA5BFA58EA39FA3FC
:10887000A8A7B9A7A601BE016C5D7F4FC7011995D6
:10888000AF960FB6F894DEBF0FBECDBFDF91CF918C
:108890001F910F91FF90EF90DF90CF90BF90AF901E
:1088A00008959B0190E00496982F8827642F820FEB
:1088B000931F0C940B371F93CF93DF931F921F923C
:1088C000CDB7DEB7182FCE0101960E94F02989811D
:1088D0009A810E94264960E170E0812F0E94E02980
:1088E0004FEF62E070E0812F0E9451440E942549C1
:1088F0000F900F90DF91CF911F910895DF92EF922B
:10890000FF920F931F93CF93DF931F921F92CDB7C8
:10891000DEB7182FD62E7A01022F0E945B44CE01BB
:1089200001960E94F02989819A810E9426494D2D45
:10893000402B60E070E0812F0E945144E114F1046B
:1089400059F4E090A60AF090A70A8FEFE81AF80A07
:10895000F092A70AE092A60A4F2D64E070E0812F02
:108960000E9451444E2D65E070E0812F0E945144D9
:1089700061E070E0812F0E94E0290E94254981E09A
:108980000F900F90DF91CF911F910F91FF90EF907B
:10899000DF900895CF93DF93FC01808D843029F020
:1089A000EF010E945B4484E0888FDF91CF910895AE
:1089B000CF92DF92EF92FF920F931F93CF93DF93AB
:1089C0001F921F92CDB7DEB7FC01F484F4E0FF16CE
:1089D00099F18C01CE0101960E94F02989819A813A
:1089E0000E94264968E070E08F2D0E94E0290E94D5
:1089F00025490E944F626B017C01C8010E94F52944
:108A00008823B9F062E370E080E090E00E94156294
:108A10000E944F62DC01CB018C199D09AE09BF0990
:108A2000883E9340A105B10540F3F80184850E947A
:108A30005B4484E0F80184870F900F90DF91CF9121
:108A40001F910F91FF90EF90DF90CF900895CF93FB
:108A5000DF9390E00496982F8827EC01C60FD71F6C
:108A60000E94AA368FE00E9495438D2F0E94954365
:108A70008C2F0E94954380E00E949543C82F0E944E
:108A8000A8368C2FDF91CF910895CF92DF92FF927D
:108A90000F931F93CF93DF931F921F92CDB7DEB733
:108AA000F82E6B01CE0101960E94F02989819A81EE
:108AB0000E94264968E270E08F2D0E942745082F0A
:108AC00010E069E270E08F2D0E942745702F662725
:108AD000682B21E030E0A6018F2D0E943F560E94B6
:108AE000254981E090E00F900F90DF91CF911F9189
:108AF0000F91FF90DF90CF900895CF93DF931F9257
:108B0000CDB7DEB7FC01218D328D232B49F0BE019C
:108B10006F5F7F4F808D0E944545898190E002C044
:108B20008FEF9FEF0F90DF91CF9108958F929F92DB
:108B3000BF92CF92DF92EF92FF920F931F93CF934A
:108B4000DF931F921F92CDB7DEB7B82E6B017A016B
:108B5000CE0101960E94F02989819A810E942649BE
:108B6000812C912C8B2D0E9426378C01892B21F092
:108B70008B2D0E9426374C010815190599F7011510
:108B8000110599F463E070E08B2D0E942745843134
:108B9000D9F18823C9F101E010E08C3111F400E033
:108BA00010E01195019511092FC0E016F1060CF4A3
:108BB00087011016110644F568E270E08B2D0E94C3
:108BC0002745E82EF12C69E270E08B2D0E942745A5
:108BD000FE2CEE24E82A9801A601B7018B2D0E94F5
:108BE0003F56E00EF11E4F2D68E270E08B2D0E9483
:108BF00051444E2D69E270E08B2D0E94514460E497
:108C000070E08B2D0E94E0290E942549C8010F9039
:108C10000F90DF91CF911F910F91FF90EF90DF9018
:108C2000CF90BF909F908F900895CF93DF93FC01DA
:108C3000218D328D2115310519F48FEF9FEF11C071
:108C4000EC014217530708F0A901888D0E94964550
:108C50001816190694F7298D3A8D281B390B3A8F6F
:108C6000298FDF91CF9108950F931F93CF93DF93B7
:108C70001F92CDB7DEB7FC01218D328D232B61F021
:108C80008C0141E050E0BE016F5F7F4F808D0E94FC
:108C90009645181619061CF08FEF9FEF08C0F801D3
:108CA000818D928D0197928F818F898190E00F90B5
:108CB000DF91CF911F910F9108950F931F93CF9341
:108CC000DF93CDB7DEB728970FB6F894DEBF0FBE9F
:108CD000CDBF8C01D80159968D919C915A97892BC3
:108CE00041F0ED91FC910284F385E02DC8011995C6
:108CF000F1CFF801808D0E949C431816190654F597
:108D000048E050E0BE016F5F7F4FD80158968C91CC
:108D10000E94964518161906FCF4D801509684E076
:108D2000FE01319601900D928A95E1F78D8190E0D8
:108D3000982F88272E81820F911DF801958B848BA7
:108D40008F8190E0982F88272885820F911D928F20
:108D5000818F02C080E090E028960FB6F894DEBFC5
:108D60000FBECDBFDF91CF911F910F9108951F933B
:108D7000CF93DF931F921F92CDB7DEB7182FCE018E
:108D800001960E94F02989819A810E94264963E018
:108D900070E0812F0E942745182F0E942549812FBE
:108DA0000F900F90DF91CF911F910895EF92FF9256
:108DB0001F93CF93DF93FC01208D243011F080E0CE
:108DC0001CC07B01EC0110E0812F0E94B74681118D
:108DD00002C0188F05C08831E1F31F5F1430A1F77E
:108DE000888D843061F3FD86EC861A8E198E20E022
:108DF000A70162E00E947E4481E0DF91CF911F9144
:108E0000FF90EF9008951F93CF93DF931F921F92CF
:108E1000CDB7DEB7FC01108DCE0101960E94F0297E
:108E200089819A810E94264960E270E0812F0E9428
:108E3000E02962E070E0812F0E94274584FD1DC07B
:108E400062E070E0812F0E94274583FF0BC048E15C
:108E500062E070E0812F0E9451440E94254980E029
:108E600090E015C00E942549CE0101960E94F0298C
:108E700089819A810E942649DCCF40E162E070E05E
:108E8000812F0E9451440E94254981E090E00F907B
:108E90000F90DF91CF911F910895CF93DF93C82F4B
:108EA000D62F472F60E170E00E9451444D2F61E1C1
:108EB00070E08C2FDF91CF910C94514490E0982F6B
:108EC000882744E050E0845F9B4F0C94DC36BF92CF
:108ED000CF92DF92EF92FF920F931F93CF93DF9386
:108EE00000D000D0CDB7DEB7FC01208D243009F0D2
:108EF0004CC06A017B018C01B12C63E070E08B2DCA
:108F00000E942745811103C0F801B08E06C0883148
:108F1000D9F3B394F4E0BF12F0CFF801808D843020
:108F2000A1F196E0E9E2F3E0DE01119601900D92E5
:108F30009A95E1F7F70193819F779C8394819D83B4
:108F400095819E83B7016E5F7F4F0E945E47B60199
:108F5000F801808D0E944D47F801808D90E0982F98
:108F6000882746E050E0BE016F5F7F4F8A5F9B4FCE
:108F70000E94DC36F801128E118E20E8A60162E014
:108F8000808D0E947E4481E001C080E026960FB66D
:108F9000F894DEBF0FBECDBFDF91CF911F910F912F
:108FA000FF90EF90DF90CF90BF900895DF92EF9207
:108FB000FF920F931F93CF93DF931F921F92CDB712
:108FC000DEB7FB01DC0157961C921E925697228158
:108FD000211109C02381211106C02481211103C060
:108FE00025812223F1F041155105D9F07A018F0135
:108FF000FC01D08CCE0101960E94F02989819A81D2
:109000000E942649B8016E5F7F4F8D2D0E945E47FA
:10901000B7018D2D0E944D470E94254981E090E0C7
:1090200002C080E090E00F900F90DF91CF911F91F0
:109030000F91FF90EF90DF900895CF93DF931F92F1
:10904000CDB7DEB76983DC01ED91FC910280F3813D
:10905000E02D41E050E0BE016F5F7F4F19950F900A
:10906000DF91CF910895DC01ED91FC91068CF78D95
:10907000E02D199591E089270895862F089581E0C4
:1090800086270895CF93DF931F92CDB7DEB78983EC
:109090002091180B3981E091190BF0911A0B822F56
:1090A00090E080959095F8940080082200824BE033
:1090B00000C05DE000005A95E9F70080082208949E
:1090C000379508F4022A00824A9599F778940F9010
:1090D000DF91CF91089585ED8093BC008091BC0015
:1090E00084FDFCCF1092F20A08954091CE0A262FFB
:1090F00030E0240F311D21323105DCF42091F20AD9
:109100002430C9F4FC0180E090E0861758F43091D7
:10911000CE0A2191DC01A255B54FA30FB11D2C93AE
:109120000196F3CF8091CE0A680F6093CE0A80E05B
:10913000089581E0089582E008958FEF9FEF0895EC
:109140008FEF9FEF08958091AD0A90E09195819502
:1091500091090895CF93DF93CB01EA01642F0E9418
:109160007548CE01DF91CF910895CF93DF931F9281
:10917000CDB7DEB7698361E0CE0101960E947548E4
:1091800081E090E00F90DF91CF9108950F931F93AE
:10919000CF93DF931F92CDB7DEB78C01DC01ED9149
:1091A000FC910084F185E02D1995892B51F0BE01C9
:1091B0006F5F7F4FF80184850E944545898190E06B
:1091C00002C08FEF9FEF0F90DF91CF911F910F9112
:1091D0000895FC0184850C949645CF93DF931F92EC
:1091E000CDB7DEB741E050E0BE016F5F7F4FFC01BD
:1091F00084850E949645181619061CF4898190E012
:1092000002C08FEF9FEF0F90DF91CF910895FC0187
:109210008485843011F00C949C4380E090E00895A4
:1092200044E050E0BC018FE090E00C94DC3644E078
:1092300050E0BC0185E090E00C94DC3644E050E066
:10924000BC0181E090E00C94DC3608958CBD9DBD9E
:1092500008956F927F928F929F92AF92BF92CF921A
:10926000DF92EF92FF921F93CF93DF931F921F9293
:10927000CDB7DEB75C013B016A01FC0114851430F7
:1092800041F481E090E0F5019383828380E090E0F7
:109290005BC07A014130584018F0E12C88E0F82E8C
:1092A000CE0101960E94F02989819A810E94264967
:1092B000812F0E94EC564C0163E070E0812F0E94E8
:1092C0002745873111F08C3121F48E149F0440F32F
:1092D00002C0E12CF12CCE0101960E94F029898177
:1092E0009A810E9426499701A30160E070E0812FD6
:1092F0000E94875660E270E0812F0E94E02962E0C0
:1093000070E0812F0E94274584FD14C063E070E067
:10931000812F0E942745811104C0812F0E945B4448
:10932000B0CFCE0101960E94F02989819A810E94D6
:109330002649E5CF40E162E070E0812F0E94514470
:10934000EF2809F49ECFC6010F900F90DF91CF91C7
:109350001F91FF90EF90DF90CF90BF90AF909F90C4
:109360008F907F906F9008958F929F92AF92BF924F
:10937000DF92EF92FF920F931F93CF93DF931F9291
:109380001F92CDB7DEB7FC012485243009F082C0DE
:109390005A018B017C01D12C8D2D0E94B746811181
:1093A00003C0F701D48607C08B7F8831D1F3D394F3
:1093B000F4E0DF12F1CFF7018485843009F46AC04C
:1093C00020910302309104022F5F3F4F11F420E0FF
:1093D00030EC309304022093030240910302509139
:1093E000040220E061E00E947E44F80182818F3F08
:1093F00051F483818F3F99F484818F3F81F485817B
:109400008F3F69F444C081110AC0F8018381811142
:1094100006C08481811103C085818823C1F1A11414
:10942000B104A9F1F701D484CE0101960E94F0297C
:1094300089819A810E942649B8016E5F7F4F8D2DE8
:109440000E945E47B5018D2D0E944D4764E070E09B
:109450008D2D0E94E0290E944F624B015C01F4E9CE
:109460008F0EF1E19F1EA11CB11CC7010E94F529BE
:10947000873141F161E070E080E090E00E94156288
:109480000E94252EC7010E94F529811106C084E0A3
:10949000F701848780E090E01DC00E944F6286162D
:1094A0009706A806B90608F7F70184850E945B4471
:1094B00084E0F701848763EB7DE087EB97E00E940F
:1094C0005E37E8CF68EA7DE087EB97E00E945E3781
:1094D00081E090E00F900F90DF91CF911F910F915D
:1094E000FF90EF90DF90BF90AF909F908F90089586
:1094F00078941F920F920FB60F9211240BB60F9211
:10950000CF92DF92EF92FF920F931F932F933F938F
:109510004F935F936F937F938F939F93AF93BF937B
:10952000CF93DF93EF93FF93809170008E7F8093B2
:1095300070000FE310E08BE1E82EF12C9BE2C92EC6
:10954000D12CC0911B0BD0911C0B2097F9F4033246
:10955000110508F43BC003521109E091190BF09179
:109560001A0B90812091180B822F8095982390835D
:109570009BE0D7011197F1F79150D9F78081822BA9
:109580008083C6010197F1F780E00DC00B30110513
:10959000E8F00B501109E0911D0BF0911E0BEC0F40
:1095A000FD1F319780810E9442482196D0931C0B69
:1095B000C0931B0B80910102909102028C179D07B2
:1095C00008F0BFCF10921C0B10921B0B8091700003
:1095D000816080937000FF91EF91DF91CF91BF91F7
:1095E000AF919F918F917F916F915F914F913F913B
:1095F0002F911F910F91FF90EF90DF90CF900F90E0
:109600000BBE0F900FBE0F901F90189581E08093B6
:10961000AC0A80910002282F30E0F901EE5AF24F97
:10962000E491F0E0EE0FFF1FEE56F34F4591549199
:1096300050931A0B4093190BF901E45FF24FE49138
:10964000E093180B61E00E94D96183E08093B10040
:10965000E0E7F0E08081816080830895CF93DF931D
:109660001816190644F0809170008E7F8093700068
:109670001092AC0A19C0EC0180911D0B90911E0B49
:109680000E94B46CCE01C130D24014F080E092E070
:1096900090930202809301020E941C6C90931E0B17
:1096A00080931D0B892B29F4109202021092010263
:1096B00008C08091AC0A811104C0DF91CF910C9455
:1096C000064BDF91CF910895FF920F931F93CF9395
:1096D000DF938C01F62E8091AC0A811102C00E94AA
:1096E000064BE8012197C11582E0D80798F48091D4
:1096F0000102909102028017910718F4C8010E949C
:109700002E4B80911D0B90911E0B009719F0C80FE6
:10971000D91FF882DF91CF911F910F91FF9008958B
:109720001F920F920FB60F9211240BB60F922F9328
:109730003F934F935F936F937F938F939F93AF93D9
:10974000BF93EF93FF938091B900887F803609F42F
:109750009CC068F5883209F45BC090F4803109F44C
:1097600054C038F4882309F4F2C0883009F44DC09D
:10977000F2C0883109F44CC0803209F45DC0EBC0FE
:10978000803409F468C048F4803309F455C0883344
:1097900009F0E1C08093F10AD4C0803509F44FC0CC
:1097A000883509F45DC0883409F0D5C0D2C0883945
:1097B00009F4C3C0A8F4883709F467C038F48836C0
:1097C00009F463C0803709F460C0C5C0883809F463
:1097D000B4C0803909F45FC0803809F0BCC05BC0F8
:1097E000803B09F484C038F4803A09F466C0883AB2
:1097F00009F47DC0B0C0803C09F4A3C0883C09F4E2
:10980000A0C0883B09F486C0A6C08091170B10C089
:109810009091160B8091150B981770F5E091160B2F
:1098200081E08E0F8093160BF0E0EB50F54F8081B6
:109830008093BB0085EC82C08093F10A8AC0E091DE
:10984000160B81E08E0F8093160B8091BB00F0E029
:10985000EB50F54F80839091160B8091150B6AC0E9
:10986000E091160B81E08E0F8093160B8091BB0068
:10987000F0E0EB50F54F80838091F40A811169C0CC
:1098800081E08093F30A84EA5DC083E08093F20A6A
:109890001092F00ACFCF8091F00A803208F04DC0CC
:1098A000E091F00A81E08E0F8093F00A8091BB0076
:1098B000F0E0E053F54F8083BDCF85EC8093BC0092
:1098C0001092F20A8091F00A803230F4E091F00AAE
:1098D000F0E0E053F54F10826091F00A70E080ED07
:1098E0009AE0E0E0F0E019951092F00A34C084E0CC
:1098F0008093F20A1092CF0A1092CE0AE0E0F0E0D4
:1099000019958091CE0A811105C081E08093CE0A1D
:109910001092AE0AE091CF0A81E08E0F8093CF0AB9
:10992000F0E0E255F54F80818093BB009091CF0A23
:109930008091CE0A981708F47DCF85E88093BC000B
:109940000AC085EC8093BC001092F20A04C0109209
:10995000F10A0E946B48FF91EF91BF91AF919F91E7
:109960008F917F916F915F914F913F912F910F90C8
:109970000BBE0F900FBE0F901F9018958F929F9265
:10998000AF92BF92CF92DF92EF92FF920F931F930D
:10999000CF93DF93CDB7DEB72B970FB6F894DEBF2A
:1099A0000FBECDBF8C01CE0101967C016C018AE017
:1099B000882E912CA12CB12CC6018E199F0941151E
:1099C00051056105710581F0CB01BA01A501940132
:1099D0000E948B76942F852F605DF60161936F0155
:1099E000A901692F782FE8CFFC013197EE0DFF1DFB
:1099F000D8019E012150310940814D933197E217E2
:109A0000F307D1F7F801E80FF91F10822B960FB674
:109A1000F894DEBF0FBECDBFDF91CF911F910F91A4
:109A2000FF90EF90DF90CF90BF90AF909F908F907E
:109A300008958F929F92AF92BF92CF92DF92EF9252
:109A4000FF920F931F93CF93DF938C014A0169011B
:109A5000E090AA0AF090AB0AC62F660FDD0BE11466
:109A6000F10449F1F7018085863029F564EE74E050
:109A7000C7010E947D375C01F2E08F16910439F036
:109A800083E08816910451F469EE74E002C06DEE33
:109A900074E0C7010E947D377C0102C0E12CF12CEB
:109AA000A114B10451F0F50161857285AE01C801C0
:109AB0000E94697B08C0E12CF12CAE0161EA7DE0D7
:109AC000C8010E942C6FAE0162EC73E0C8010E94D5
:109AD0004B7BE114F10421F0F701618572850FC021
:109AE000F2E08F169104A1F083E08816910461F0F2
:109AF0008A94892899F46091A80A7091A90AAE0104
:109B0000C8010E944B7B0AC0AE016BE97DE003C037
:109B1000AE0168E97DE0C8010E941C6FAE0162ECF5
:109B200073E0C8010E944B7BC114D10429F0AE013F
:109B3000B601C8010E944B7BC801DF91CF911F91F4
:109B40000F91FF90EF90DF90CF90BF90AF909F90DC
:109B50008F900895CF93DF931F921F92CDB7DEB7FA
:109B60008091490B90914A0B009711F485E59BE099
:109B7000BE016F5F7F4F681B790B072E000C880BAF
:109B8000990B0F900F90DF91CF910895AF92BF92F4
:109B9000CF92DF92EF92FF920F931F93CF93DF93B9
:109BA000CDB7DEB7AF970FB6F894DEBF0FBECDBF0F
:109BB0007C015B016A0101E213E01A8309831B82C5
:109BC0001C821D821E82CE0109960E94CC431BA7D7
:109BD0000AA71CA61DA61EA61FA680915C08909130
:109BE0005D08A0915E08B0915F088EA39FA3A8A70F
:109BF000B9A78B839C83AD83BE8318861F82AE0179
:109C0000465D5F4FB501CE0101960E94803E8130D6
:109C10009105B1F4D701ED91FC910684F785E02D13
:109C20001DA30CA38CA59DA5AEA5BFA58EA39FA328
:109C3000A8A7B9A7A601BE016C5D7F4FC701199502
:109C4000AF960FB6F894DEBF0FBECDBFDF91CF91B8
:109C50001F910F91FF90EF90DF90CF90BF90AF904A
:109C6000089568E67FE087EB97E00E94A85AE0E05D
:109C7000F0E01994CF93DF931F92CDB7DEB719822E
:109C8000892B21F0FB016281738103C0BE016F5FEC
:109C90007F4F86E390E00E94E02E64EB70E187EB5B
:109CA00097E00E94A85A0F90DF91CF910895CF932B
:109CB000DF93C0E0D0E060E0CE010E946D76219697
:109CC000C11582E0D807B9F764EA70E187EB97E045
:109CD000DF91CF910C94A85A0F931F93CF93DF93EA
:109CE000CDB7DEB72C970FB6F894DEBF0FBECDBF51
:109CF0008B0121E233E03A8329831B821C821D827F
:109D00001E8238872F8319861A861B861C8683300D
:109D10009105B9F144F48130910509F45BC00297D3
:109D200009F443C064C084309105B9F0059709F087
:109D30005EC0BE01695F7F4FF801808591850E94FA
:109D4000423EBE01892B19F0695F7F4F02C06F5FF1
:109D50007F4F82E190E00E94233EBE01695F7F4F0A
:109D6000F801868197810E94423EBE01892B19F03D
:109D7000695F7F4F02C06F5F7F4F8EE090E00E946F
:109D8000233EBE01695F7F4FF801848195810E9467
:109D9000423EBE01892B19F0695F7F4F02C06F5FA1
:109DA0007F4F8AE090E00E94233EBE01695F7F4FB3
:109DB000F801828193810E94423EBE01892B19F0F5
:109DC000695F7F4F02C06F5F7F4F86E090E00E9427
:109DD000233E0DC0BE016F5F7F4F86E090E00E9482
:109DE000233E64E970E187EB97E00E94A85A6DE892
:109DF00070E187EB97E00E94A85A2C960FB6F89472
:109E0000DEBF0FBECDBFDF91CF911F910F9108959F
:109E1000CF93DF93CDB7DEB72C970FB6F894DEBFA4
:109E20000FBECDBF1C821B821E821D828FEF9FEF53
:109E300098878F838CE693E09A83898386E490E009
:109E40009A8789871C861B8663E770E187EB97E01A
:109E50000E94A85A60910D0670910E06CE010196DF
:109E60000E94C5336FEFCE0101960E94A83263E6CF
:109E700070E187EB97E00E94A85A2C960FB6F894F1
:109E8000DEBF0FBECDBFDF91CF9108950F931F931B
:109E9000CF93DF93CDB7DEB769970FB6F894DEBFE7
:109EA0000FBECDBF8FE290E09A838983FE01339687
:109EB00087E1DF011D928A95E9F76EE470E187EB97
:109EC00097E00E94A85A27E93AE0DE011196AE0118
:109ED000435F5F4F8D01F90161919F01862F90E0F3
:109EE00074E0959587957A95E1F7895A9C4FFC0126
:109EF000808111968C931197E62FEF70F0E0E95A6C
:109F0000FC4F808112968C9312971296A417B50776
:109F100011F71E8662EF74E0C8010E94257BB8012C
:109F200087EB97E00E94765BC8010E94B53D1E86D4
:109F30006AEF74E0C8010E94257BB80187EB97E0C7
:109F40000E94765B64E075E0C8010E9489296996E9
:109F50000FB6F894DEBF0FBECDBFDF91CF911F913A
:109F60000F910895CF93C1E068EE73E080E090E038
:109F70000E9415626C2F87EB97E00E949837CF5FA5
:109F8000C43191F7CF9108950F931F93CF93DF932F
:109F9000CDB7DEB728970FB6F894DEBF0FBECDBFA2
:109FA0000E94332E61EC7DE087EB97E00E94A85A77
:109FB000CE0101960E94D155CE0101960E947B559B
:109FC00001E213E01A8309831B821C821D821E8218
:109FD000CE0107960E94F0298F8198850E9426491C
:109FE00044E050E0BE016D5F7F4F81E090E00E9451
:109FF000AC360E942549CE0101960E947B551A83FA
:10A0000009831B821C821D821E82CE0107960E943C
:10A01000F0298F8198850E94264944E050E0BE01D6
:10A020006D5F7F4F85E090E00E94AC360E9425492D
:10A03000CE0101960E947B5567EE7DE087EB97E0AD
:10A040000E94A85A28960FB6F894DEBF0FBECDBF67
:10A05000DF91CF911F910F9108957F928F929F92E0
:10A06000AF92BF92CF92DF92EF92FF920F931F9326
:10A07000CF93DF93CDB7DEB729970FB6F894DEBF45
:10A080000FBECDBF80910D0690910E06009709F48A
:10A0900036C266E075E00E947D379093280B80936E
:10A0A000270B009709F4A5C00E94123B082F10E06F
:10A0B0000115110509F49DC0000F111F000F111F9C
:10A0C0008091200B9091210B892B09F083C0C8014E
:10A0D0000E941C6C9093210B8093200B1092370BE5
:10A0E0001092360B10922A0B1092290B1092350BFE
:10A0F0001092390B1092380B7801013082E018076A
:10A100001CF0E12C32E0F32EC70101960E941C6C7A
:10A1100090933B0B80933A0B9093340B8093330BCB
:10A120008E0D9F1D90932E0B80932D0B0E944F62DE
:10A1300060932F0B7093300B8093310B9093320B05
:10A1400080E090E0E0913A0BF0913B0BE80FF91FB3
:10A1500010820196E816F906ACF782E090E0909341
:10A16000370B8093360B80E98093C9001092C800AA
:10A170001092CD0083E08093CC008EE08093CA00E3
:10A18000F0920702E092060220913A0B30913B0BCD
:10A190008091060290910702820F931F90932E0BDD
:10A1A00080932D0B232B09F438C161E97FE087EB05
:10A1B00097E00E94A85AB80187EB97E00E945637B3
:10A1C00087EB97E00E94725B8BE19FE190932C0BF1
:10A1D00080932B0B65EF7FE087EB97E00E94A85AF6
:10A1E000B80187EB97E00E94563787EB97E00E9413
:10A1F000725B6CE075E080910D0690910E060E94F6
:10A200007D378C01009791F10E94123B882371F1F8
:10A2100061E0C8010E947037FC01018512859091B0
:10A22000AC0A992359F0809170008E7F8093700062
:10A230001092AC0A109202021092010283E0809305
:10A24000000291110E94064BC8010E942E4B69ED3D
:10A250007FE087EB97E00E94A85AB80187EB97E070
:10A260000E94563787EB97E00E94725BE0900D06E4
:10A27000F0900E0660E175E0C7010E947D37909373
:10A28000260B8093250B67E175E0C7010E947D379F
:10A290008C0190930806809307066DE175E0C70175
:10A2A0000E947D379093AB0A8093AA0A1092A7056B
:10A2B0001092A6050115110511F1F801068117810B
:10A2C00021E7A22E22E0B22EE0900706F0900806C9
:10A2D000E114F10469F00115110551F0F8018085D0
:10A2E0008530B1F7C8010E94123B823088F39CC0D0
:10A2F000F701868197819093A7058093A605E0904A
:10A300000D06F0900E0669E075E0C7010E947D37EA
:10A310008C019093100680930F0664E275E0C701EC
:10A320000E947D379093240B8093230B0115110518
:10A33000A1F0F801068117810115110571F0F801EE
:10A340008085863031F41A830983CE0101960E94FC
:10A35000CC21F80102811381EFCF63EC7FE087EB22
:10A3600097E00E94A85A6BEB7FE087EB97E00E9492
:10A37000A85A81E02091070630910806232B09F4A2
:10A3800080E00E94152F62EB7FE087EB97E00E9450
:10A39000A85A81E020910F0630911006232B09F472
:10A3A00080E00E94152F69EA7FE087EB97E00E942A
:10A3B000A85A81E02091250B3091260B232B09F41C
:10A3C00080E00E94152F62EA7FE087EB97E00E9411
:10A3D000A85A81E02091230B3091240B232B09F400
:10A3E00080E00E94152F87EB97E00E94725B0E942D
:10A3F000AA4D6B017C016DE97FE087EB97E00E943D
:10A40000A85A2AE0B701A60187EB97E00E94E15A1B
:10A4100087EB97E00E94725B72C06AE77FE087EB90
:10A4200097E00E945E37D0CEBA82A9821C830B834C
:10A43000CE0101960E947820CE0101960E94A91FAC
:10A44000882309F458C060E070E0CE0101960E94B4
:10A4500012207C0197FF07C0F194E194F108882451
:10A460008394912C02C0812C912C60E0CE01019646
:10A470000E946520C82ED12C8985853019F0863040
:10A4800049F039C0C114D10429F462E0CE0101962B
:10A490000E9440207E2C61E08E2D0E94D96161E0F7
:10A4A000892821F0CA94CD2829F403C0CA94CD2864
:10A4B00009F060E0C62ED12C872D0E94004164ED8A
:10A4C0007FE087EB97E00E94A85AB70187EB97E0FF
:10A4D0000E94563762ED7FE087EB97E00E94A85A12
:10A4E000B60187EB97E00E94563760ED7FE087EB7F
:10A4F00097E00E94A85AF80102811381E5CE2996BF
:10A500000FB6F894DEBF0FBECDBFDF91CF911F9184
:10A510000F91FF90EF90DF90CF90BF90AF909F9002
:10A520008F907F900895CF93DF93CDB7DEB72C97B0
:10A530000FB6F894DEBF0FBECDBF63E370E187EBCB
:10A5400097E00E94A85A87EB97E00E94725B86E42E
:10A5500090E00E9465768B37A1F51C821B821E82DB
:10A560001D828FEF9FEF98878F838CE693E09A830D
:10A57000898386E490E09A8789871C861B860E94DF
:10A58000685FCE0101960E94BF2990930E068093CA
:10A590000D06892B19F466E170E115C06FE070E1DA
:10A5A00087EB97E00E94A85A87EB97E00E94725BC6
:10A5B0000E942D508DE19AE00E94D84481E090E005
:10A5C0000CC062E270E187EB97E00E94A85A87EB2B
:10A5D00097E00E94725B80E090E02C960FB6F894B2
:10A5E000DEBF0FBECDBFDF91CF9108950C94935283
:10A5F000CF92DF92EF92FF92CF93DF93EC010E9414
:10A600004F626B017C018091660890916708DC01C4
:10A61000ED91FC910084F185E02D1995892B79F459
:10A620000E944F62DC01CB018C199D09AE09BF0964
:10A6300088399A43A105B10530F380E00DC08091BF
:10A64000660890916708DC01ED91FC910284F38526
:10A65000E02D1995888381E0DF91CF91FF90EF90F5
:10A66000DF90CF9008954F925F926F927F928F927A
:10A670009F92AF92BF92CF92DF92EF92FF920F9391
:10A680001F93CF93DF931F921F92CDB7DEB75C016C
:10A6900088E698E00E94F85281113AC036C08C01D9
:10A6A000CE0101960E94F852882379F1C8010196E3
:10A6B0002981F70121937F01422F4F7750E0449D7C
:10A6C000B001459D700D549D700D1124C60ED71E0E
:10A6D00047E0440C551C661C771C4A95D1F727FFB0
:10A6E00027C085309105D9F68FEF9FEF909302092F
:10A6F000809301098091660890916708DC01ED91D3
:10A70000FC910488F589E02D199580E090E08EC0D9
:10A7100090906808198289E6E82E88E0F82E01E01A
:10A7200010E0C12CD12C412C512C32014394B8CFD4
:10A73000F92DF07FFA832FEF280FD5012C93F033FA
:10A7400019F58859974F0E94F8528823F1F2C801F1
:10A750008659974F0E94F8528823B9F2C801039690
:10A76000D501EC91F0E0EE59F74FE780F12CFE2C8B
:10A77000EE242085E20EF11C2091680821FF08C01C
:10A78000B2E0EB0EF11C04C020E0E12CF12C01C082
:10A7900022E0422E512CFC01EE59F74F4F018C0163
:10A7A000481A590A2EEF622E77247A94C801840D34
:10A7B000951D8C159D0578F5CE0101960E94F852E5
:10A7C000882309F4A2CF8091FF0890910009009797
:10A7D000B1F0FA81F03399F4D5012C91F301E21B29
:10A7E000F1099F01200F311FE216F30640F4DC014E
:10A7F000ED91FC910190F081E02D6981199500386F
:10A80000110518F48981F40186830F5F1F4FFFEF54
:10A810008F1A9F0ACBCF8091FF0890910009892B56
:10A8200021F40138110508F070CFC8010F900F9086
:10A83000DF91CF911F910F91FF90EF90DF90CF901C
:10A84000BF90AF909F908F907F906F905F904F9050
:10A8500008952F923F924F925F926F927F928F92C4
:10A860009F92AF92BF92CF92DF92EF92FF920F939F
:10A870001F93CF93DF931F92CDB7DEB70E94D226EE
:10A88000382E882309F422C10E944F622B013C011B
:10A890008091EE089091EF08A091F008B091F10836
:10A8A000A3019201281B390B4A0B5B0BDA01C9018A
:10A8B00089399A43A105B105A8F48091EA089091DD
:10A8C000EB08A091EC08B091ED08A3019201281BC0
:10A8D000390B4A0B5B0BDA01C90189399A43A1058F
:10A8E000B105C8F12091F20880916608909167083F
:10A8F000222371F02CEF3FEF3093020920930109DE
:10A90000DC01ED91FC910488F589E02D1995DDC0FD
:10A9100020EC2093680810926908DC01ED91FC910D
:10A920000280F381E02D42E050E068E678E019957E
:10A930004092EA085092EB086092EC087092ED08A1
:10A940004092EE085092EF086092F0087092F10881
:10A9500081E08093F2088091660890916708DC019D
:10A96000ED91FC910084F185E02D1995892B09F476
:10A97000ADC0CE0101960E9433535C01892B09F4CE
:10A98000A0C04092EE085092EF086092F0087092DA
:10A99000F10880916808807F803309F076C080914B
:10A9A000F3089091F408892B09F490C0E980F12C08
:10A9B000F701EE59F74F078110E0102F002780852F
:10A9C000080F111D97012659374F4901B7016559E5
:10A9D000774FA801C9010E94007BB8016E0D7F1D51
:10A9E000DB01AE59B74F18961C92189780916808F2
:10A9F0008670282EE091F308F091F40832E083137A
:10AA000037C01996CC901997D12CDC2CCC241A96EF
:10AA10008C91C80ED11C4BEF5FEF4E195F09401BA4
:10AA2000510B4A0D5B1D6359774FC401199580E4A2
:10AA30008093680820926908D0926A08C0926B08D7
:10AA40008091660890916708DC01ED91FC9102808D
:10AA5000F381E02D44E050E068E678E019954092FB
:10AA6000EA085092EB086092EC087092ED082EC054
:10AA70004DEF5FEF4E195F09401B510B4A0D5B1DF7
:10AA80006559774FC401199521C0803CA9F480ED28
:10AA90008093680810926908809166089091670811
:10AAA000DC01ED91FC910280F381E02D42E050E069
:10AAB00068E678E019950AC0803D41F41092F208EA
:10AAC00005C00E94D226811101C0312C832D0F9028
:10AAD000DF91CF911F910F91FF90EF90DF90CF907A
:10AAE000BF90AF909F908F907F906F905F904F90AE
:10AAF0003F902F900895AF92BF92CF92DF92EF9246
:10AB0000FF921F93CF93DF9300D000D0CDB7DEB775
:10AB10006C017C0110E08AE0A82EB12C1330A9F062
:10AB2000F701828190E0A0E0B0E089839A83AB8353
:10AB3000BC83BE82AD82BE016F5F7F4F87EB97E023
:10AB40000E94D22069EC70E114C0F601858190E08A
:10AB5000A0E0B0E089839A83AB83BC83BE82AD82E0
:10AB6000BE016F5F7F4F87EB97E00E94D22066ECBB
:10AB700070E10E94A85A1F5FFFEFEF1AFF0A14301E
:10AB800069F626960FB6F894DEBF0FBECDBFDF91F3
:10AB9000CF911F91FF90EF90DF90CF90BF90AF903B
:10ABA00008950F931F93CF93DF931F921F92CDB7FA
:10ABB000DEB78C0181E293E0F801918380831282F9
:10ABC000138214821582CE0101960E94F029898198
:10ABD0009A810E942649B8016E5F7F4F44E050E0A1
:10ABE0008FE090E00E94AC360E942549C8010F908A
:10ABF0000F90DF91CF911F910F910895CF93DF9325
:10AC0000C2E6D8E080EE8E831F828C819D81DC01BC
:10AC1000ED91FC910280F381E02D42E050E068E686
:10AC200078E019958FEF9FEF9093020980930109C7
:10AC30008C819D81DC01ED91FC910680F781E02DF6
:10AC400019958C819D81DC01ED91FC910488F58939
:10AC5000E02D19950E944F626093EA087093EB080B
:10AC60008093EC089093ED086093EE087093EF08E2
:10AC70008093F0089093F108DF91CF910895AF92FF
:10AC8000BF92CF92DF92EF92FF920F931F93CF93D9
:10AC9000DF931F921F92CDB7DEB77A836983BA0123
:10ACA000A901E981FA81F770082F10E0000F111F48
:10ACB00003501A4FD8018D919C918E0F9F1F9F01B9
:10ACC000240F351F21303840A0F07A015B0160E08D
:10ACD00078E06B01CE1ADF0AA601B5010E94AC36FE
:10ACE000A7014C195D09B5016C0D7D1DF80180812E
:10ACF00091810F900F90DF91CF911F910F91FF9055
:10AD0000EF90DF90CF90BF90AF900C94AC369F92B5
:10AD1000AF92BF92CF92DF92EF92FF920F931F9369
:10AD2000CF93DF93982E8B015A01690164E270E0A2
:10AD30000E942745E82EF12C65E270E0892D0E94E3
:10AD40002745FE2CEE24E82AE801CE0DDF1D9E01EA
:10AD50003770E92CF12CC701880F991FAC014B50BB
:10AD60005A4F7A01FA0180819181820F931FA901C4
:10AD70004C0D5D1D4130584090F000E018E0021B82
:10AD8000130BA801B5010E94DC36A601401B510B34
:10AD9000B501600F711FF7018081918102C0A6018A
:10ADA000B5010E94DC36CC0DDD1D4D2F64E270E054
:10ADB000892D0E9451444C2F65E270E0892DDF916E
:10ADC000CF911F910F91FF90EF90DF90CF90BF90A8
:10ADD000AF909F900C945144FF920F931F93CF9389
:10ADE000DF93F82E00E010E08F2D0E943E37EC013B
:10ADF000892B21F08F2D0E943E378C01C017D1077F
:10AE000099F7CE01DF91CF911F910F91FF90089597
:10AE100020E3FC0120833296862F82958F7090E18B
:10AE2000899F601911246A3014F4605D01C0695C67
:10AE30006293682F8111F0CF08952F923F924F9225
:10AE40005F926F927F928F929F92AF92BF92CF92BA
:10AE5000DF92EF92FF920F931F93CF93DF93CDB7C3
:10AE6000DEB7E2970FB6F894DEBF0FBECDBF7C0110
:10AE70002A013B0169010E944F624B015C0187017D
:10AE80000D5B1F4FC8010E945D4618161906A4F0FD
:10AE90000E944F62DC01CB0188199909AA09BB09FC
:10AEA000481659066A067B06D8F062E370E080E037
:10AEB00090E00E941562E6CF42E250E0BE016F5F73
:10AEC0007F4FC8010E9415468981823011F080E0D1
:10AED00060C1F8018489958983349105C1F702C066
:10AEE0008FEF57C16D817E818F8198850E94F676A4
:10AEF0004B015C01F601608371838283938346E09A
:10AF000050E0B701685F7F4FCE014D960E94F37A03
:10AF1000892BE9F6F70180819181A281B38188169E
:10AF20009906AA06BB0698F284819581A681B7810D
:10AF300088159905AA05BB0550F289899A89AB89BC
:10AF4000BC8986879787A08BB18B8EECC82ED12CBD
:10AF5000C8010E943446F1E0CF1AD108C9F7712C1C
:10AF6000C70182969AA789A7F701B696FCA7EBA717
:10AF700008969EA78DA73C974F01899698AB8FA7FF
:10AF80003897FAABE9AB1701F6E12F0E311C270118
:10AF90008EE1480E511CF801818D928D181619060C
:10AFA0000CF0F6C0C8010E9434468333910509F4C1
:10AFB000C9C0F4F481309105B9F11CF4892B59F31F
:10AFC000DBC083309105C1F1069709F0D5C0C801F7
:10AFD0000E9434466C0144E050E0B201C8010E9476
:10AFE0001546A12CB12CDD2494E0C91AD1083FC02C
:10AFF0008A33910509F47AC03CF48533910561F0F8
:10B00000C69709F43FC0B8C08B33910509F484C0DA
:10B010008F3F910501F2B0C0C8010E943446C801BB
:10B020000E943446782EB7CFC8010E94344644E0CF
:10B0300050E069A97AA93AC0C8010E9434466C015F
:10B0400044E050E0B101C8010E941546A12CB12C8A
:10B05000DD24F4E0CF1AD108AC14BD040CF09BCF72
:10B06000C8010E9434468FEFA81AB80AF5CFAC1475
:10B07000BD040CF090CFC8010E943446EFEFAE1A29
:10B08000BE0AF5CFC8010E943446682EF701828DB2
:10B09000811110C0838D81110DC0848D81110AC072
:10B0A000858D811107C044E050E0B401C8010E94C1
:10B0B000154671CFEFA5F8A9A080B180C280D380DA
:10B0C000B401CE0183960E94785B8DA19EA1AFA1B1
:10B0D000B8A5A816B906CA06DB0629F3662009F446
:10B0E0005ACFC8010E9434466A94F8CFC8010E9422
:10B0F000344644E050E06BA57CA5C8010E9415468B
:10B10000F70166A177A180A591A50E94F67666A3B6
:10B1100077A380A791A73FCFC8010E94344644E09F
:10B1200050E06DA57EA5C8010E941546F70162A5F5
:10B1300073A584A595A50E94F67662A773A784A738
:10B1400095A729CFC8010E94344644E050E069A584
:10B150007AA5C8010E941546F70162A173A184A1D6
:10B1600095A10E94F67662A373A384A395A366A714
:10B1700077A780AB91AB0FCFC8010E943446D82E81
:10B18000DD2009F408CFC8010E943446DA94F8CFD4
:10B19000872DE2960FB6F894DEBF0FBECDBFDF91CC
:10B1A000CF911F910F91FF90EF90DF90CF90BF90C4
:10B1B000AF909F908F907F906F905F904F903F9057
:10B1C0002F900895CF92DF92EF92FF920F931F93EB
:10B1D000CF93DF936C017A018B01C0E0D0E0CE15F4
:10B1E000DF0581F0D8016D918D01D601ED91FC91C3
:10B1F0000190F081E02DC6011995892B11F021965F
:10B20000EECF7E01C701DF91CF911F910F91FF908B
:10B21000EF90DF90CF900895FC01538D448D252F42
:10B2200030E0842F90E0821B930B541710F0CF96E0
:10B23000089501970895FC01918D828D981761F012
:10B24000828DDF01A80FB11D5D968C91928D9F5F5D
:10B250009F73928F90E008958FEF9FEF0895FC0108
:10B26000918D828D981731F0828DE80FF11D858DBB
:10B2700090E008958FEF9FEF0895FC01918D228D4E
:10B28000892F90E0805C9F4F821B91098F739927D3
:10B2900008958AE197E00E943D5921E0892B09F445
:10B2A00020E0822F089587EB97E00E943D5921E02E
:10B2B000892B09F420E0822F0895FC01848DDF01A1
:10B2C000A80FB11DA35ABF4F2C91848D90E0019619
:10B2D0008F739927848FA689B7892C93A089B18908
:10B2E0008C91837080648C93938D848D981306C0A9
:10B2F0000288F389E02D80818F7D80830895EF920D
:10B30000FF920F931F93CF93DF93EC0181E0888F1F
:10B310009B8D8C8D981305C0E889F989808185FD06
:10B3200026C0F62E0B8D10E00F5F1F4F0F731127F5
:10B33000E02E8C8DE8120CC00FB607FCFACFE8891E
:10B34000F989808185FFF5CFCE010E945D59F1CF4B
:10B350008B8DFE01E80FF11DE35AFF4FF0829FB77E
:10B36000F8940B8FEA89FB89808180620AC09FB7BD
:10B37000F894EE89FF896083E889F9898081837078
:10B38000806480839FBF81E090E0DF91CF911F9127
:10B390000F91FF90EF900895CF93DF93EC01888D8C
:10B3A0008823C9F0EA89FB89808185FD05C0A889C9
:10B3B000B9898C9186FD0FC00FB607FCF5CF80814F
:10B3C00085FFF2CFA889B9898C9185FFEDCFCE0199
:10B3D0000E945D59E7CFDF91CF91089580E090E022
:10B3E000892B21F00E945359811121C080E090E007
:10B3F000892B41F080E090E0892B21F00E94000031
:10B40000811118C080E090E0892B21F00E944959F9
:10B41000811113C080E090E0892BA1F080E090E0E2
:10B42000892B81F00E94000081110AC008950E94BA
:10B430000000DCCF0E940000E5CF0E940000EACFB0
:10B440000C94000008950E94D47AEF92FF920F931B
:10B450001F93CF93DF93EC018B017A010E944F621F
:10B46000FE01E857FF4F60837183828393838C8151
:10B470009D81DC01ED91FC910280F381E02DA7011B
:10B48000B801DF91CF911F910F91FF90EF90199428
:10B490001F93CF93DF93EC01162F0E944F62FE01A2
:10B4A000E857FF4F60837183828393838C819D81F2
:10B4B000DC01ED91FC910190F081E02D612FDF9195
:10B4C000CF911F911994DC01ED91FC910190F081D5
:10B4D000E02D19948F929F92AF92BF92CF92DF92FC
:10B4E000EF92FF920F931F93CF93DF937C018B0119
:10B4F0004C0182E0880E911C5701E5E0AE0EB11CB4
:10B50000C0E0D0E0F40161914F01C8010E9498377A
:10B510006C016EE2C8010E94635A8C0D9D1DC80F1C
:10B52000D91F8A149B0471F7F7016581C8010E9435
:10B5300098378C0F9D1FDF91CF911F910F91FF9036
:10B54000EF90DF90CF90BF90AF909F908F90089535
:10B55000EF92FF920F931F93CF93DF938C017B01A8
:10B56000C0E0D0E0F701EC0FFD1F6491662361F0AD
:10B57000D801ED91FC910190F081E02DC801199561
:10B58000892B11F02196EECFCE01DF91CF911F9143
:10B590000F91FF90EF9008956115710579F0FB010F
:10B5A00001900020E9F73197AF01461B570BDC01F2
:10B5B000ED91FC910280F381E02D199480E090E000
:10B5C00008958F929F92AF92BF92EF92FF920F9346
:10B5D0001F93CF93DF93CDB7DEB7A1970FB6F89443
:10B5E000DEBF0FBECDBF7C01FA01CB0119A2223014
:10B5F00008F42AE08E010F5D1F4F822E912CA12CA2
:10B60000B12CBF01A50194010E948B76F901CA01FA
:10B61000015011096A3014F4605D01C0695CD80101
:10B620006C93232B242B252B61F7B801C7010E94B3
:10B63000CC5AA1960FB6F894DEBF0FBECDBFDF91F6
:10B64000CF911F910F91FF90EF90BF90AF909F907F
:10B650008F900895CF92DF92EF92FF920F931F93F6
:10B66000CF93DF932115310581F4DC01ED91FC913D
:10B670000190F081E02D642FDF91CF911F910F9108
:10B68000FF90EF90DF90CF9019942A30310501F5AB
:10B6900077FF1DC06A017B01EC016DE20E94635AD5
:10B6A0008C0144275527BA014C195D096E097F09A1
:10B6B0002AE0CE010E94E15A800F911FDF91CF91C5
:10B6C0001F910F91FF90EF90DF90CF9008952AE0A7
:10B6D000DF91CF911F910F91FF90EF90DF90CF906E
:10B6E0000C94E15A6AE074E00C94CC5A0C94CC5A55
:10B6F000DC0181E293E08D939D9384E0FB01019056
:10B700000D928A95E1F708951F920F920FB60F924E
:10B7100011240BB60F922F933F934F935F936F9328
:10B720007F938F939F93AF93BF93EF93FF938AE1A0
:10B7300097E00E945D59FF91EF91BF91AF919F916A
:10B740008F917F916F915F914F913F912F910F90CA
:10B750000BBE0F900FBE0F901F9018951F920F9267
:10B760000FB60F9211240BB60F922F938F939F93C6
:10B77000EF93FF93E0912A07F0912B078081E091EE
:10B780003007F091310782FD12C09081809133071C
:10B790008F5F8F7320913407821751F0E091330748
:10B7A000F0E0E65EF84F958F8093330701C080810B
:10B7B000FF91EF919F918F912F910F900BBE0F9062
:10B7C0000FBE0F901F9018951F920F920FB60F92F9
:10B7D00011240BB60F922F933F934F935F936F9368
:10B7E0007F938F939F93AF93BF93EF93FF9387EBD9
:10B7F00097E00E945D59FF91EF91BF91AF919F91AA
:10B800008F917F916F915F914F913F912F910F9009
:10B810000BBE0F900FBE0F901F9018951F920F92A6
:10B820000FB60F9211240BB60F922F938F939F9305
:10B83000EF93FF93E091C707F091C8078081E091F3
:10B84000CD07F091CE0782FD12C090818091D00784
:10B850008F5F8F732091D107821751F0E091D0074D
:10B86000F0E0E954F84F958F8093D00701C08081B4
:10B87000FF91EF919F918F912F910F900BBE0F90A1
:10B880000FBE0F901F9018951F920F920FB60F9238
:10B8900011240BB60F922F933F934F935F938F9387
:10B8A0009F93EF93FF9320913A0B30913B0B809144
:10B8B000380B9091390BAC014F5F5F4F5093390BB0
:10B8C0004093380BF901E80FF91F80818093CE0077
:10B8D00080910602909107022091380B3091390B2C
:10B8E0008217930748F48FEF9FEF9093390B809363
:10B8F000380B88E48093C900FF91EF919F918F915D
:10B900005F914F913F912F910F900BBE0F900FBE03
:10B910000F901F9018951F920F920FB60F9211243F
:10B920002F933F938F939F932091360B3091370B3A
:10B930008091380B9091390B21303105A9F48F3F5C
:10B940002FEF920789F41092C8001092CD0089E081
:10B950008093CC0086E28093CA001092CE001092B1
:10B96000390B1092380B17C0892BA9F41092C8001C
:10B970001092CD0083E08093CC008EE08093CA00CB
:10B9800088E28093C9001092CE0081E090E090930D
:10B99000390B8093380B9F918F913F912F910F908E
:10B9A0000FBE0F901F9018951F920F920FB60F9217
:10B9B00011240BB60F922F933F934F935F936F9386
:10B9C0007F938F939F93AF93BF93EF93FF93909148
:10B9D000C8008091CE0094FF08C081E08093350BB1
:10B9E00080913A0B90913B0B57C09091350B913061
:10B9F00099F481110EC082E08093350B0E944F6252
:10BA000060932F0B7093300B8093310B9093320B1C
:10BA10003EC01092350B44C0923009F041C0E09115
:10BA2000330BF091340B9081891721F091E09093C2
:10BA3000050280832091330B3091340B80912D0BC4
:10BA400090912E0B2817390711F51092350B809124
:10BA500005028823D1F080912B0B90912C0B892B20
:10BA6000A1F01092C900E0912B0BF0912C0B1995CD
:10BA700080E98093C9001092C8001092CD0083E045
:10BA80008093CC008EE08093CA00109205028091D2
:10BA9000330B9091340B01969093340B8093330BBE
:10BAA000FF91EF91BF91AF919F918F917F916F9196
:10BAB0005F914F913F912F910F900BBE0F900FBE52
:10BAC0000F901F901895CF92DF92EF92FF920F93F5
:10BAD0001F93CF93DF936C018B0186E090E00E946F
:10BAE0001C6CEC0190933D0B80933C0BF601019094
:10BAF0000020E9F7CF018C199D090E941C6C7C0184
:10BB0000B6010E94447BF60101900020E9F73197CD
:10BB1000EC19FD09EE0DFF1D1082F982E8821B83EE
:10BB20000A838091A3059091A4059D838C83D09373
:10BB3000A405C093A305DF91CF911F910F91FF90B2
:10BB4000EF90DF90CF900895CF92DF92EF92FF9227
:10BB50000F931F93CF93DF93CDB7DEB7EC970FB65C
:10BB6000F894DEBF0FBECDBFDC012C91222309F477
:10BB700051C063E474E00E943B6F9A8389837E0125
:10BB8000B3E0EB0EF11C01E010E0D02EC12E63E417
:10BB900074E080E090E00E943B6FF7018193919305
:10BBA0007F010E31110539F400913C0B10913D0BD2
:10BBB000E980FA8008C00F5F1F4F892B31F7F4CF5F
:10BBC000F8010481158101151105A1F0D8016D91CD
:10BBD0007C91C7010E943B7B892B91F7D80112967B
:10BBE000ED91FC911397BE016F5F7F4F8D2D9C2DC2
:10BBF000199506C06FEC70E187EB97E00E945E3705
:10BC000087EB97E00E94725B6BEC70E187EB97E04B
:10BC10000E94A85AEC960FB6F894DEBF0FBECDBFB7
:10BC2000DF91CF911F910F91FF90EF90DF90CF9018
:10BC30000895FB0124813581428153812417350702
:10BC400058F440815181DA01A20FB31F8C93848193
:10BC5000958101969583848380E00895FC01848119
:10BC600095810895089580E090E00895AF92BF9285
:10BC7000CF92DF92EF92FF920F931F93CF93DF93B8
:10BC8000CDB7DEB7C154D1090FB6F894DEBF0FBEF1
:10BC9000CDBF5C016B018A016BE471E187EB97E03A
:10BCA0000E94A85AB50187EB97E00E94765B68E492
:10BCB00071E187EB97E00E94A85AC114D10409F4FE
:10BCC0009BC00C0D1D1DF80110820E94AA4D6A3FF9
:10BCD00071051CF463E471E14DC07601E016F106D4
:10BCE00041F0F70161917F0187EB97E00E94635A71
:10BCF000F5CF87EB97E00E94725B8091A805909149
:10BD0000A9059E012F5F3F4F790120E030E00497A5
:10BD100019F443E050E019C042E050E061E4C7018B
:10BD20000E94194DF70101900020E9F731978F012A
:10BD30000E191F09A801B701C5010E945B7B00977E
:10BD4000A9F020E030E041E050E061E4C7010E944A
:10BD5000194DF70101900020E9F731978F010E1975
:10BD60001F09A801B701C5010E945B7B892B39F02F
:10BD700068E371E187EB97E00E94A85A3DC00A0D85
:10BD80001B1D69E275E0C8010E943B7B892B21F4F1
:10BD9000C6010E94A45D30C06FE270E0C8010E943D
:10BDA000307B5C01009741F0FC011082818184327C
:10BDB00019F1FFEFAF1ABF0AF80180818432E1F078
:10BDC000B801C7010E94D125C7010E94A91F88237D
:10BDD00099F029858091A8059091A905273019F43B
:10BDE0008430910549F041E0049709F440E0950161
:10BDF000B601C7010E94C21BCF5BDF4F0FB6F8949C
:10BE0000DEBF0FBECDBFDF91CF911F910F91FF908D
:10BE1000EF90DF90CF90BF90AF900895CF92DF92D8
:10BE2000EF92FF921F93CF93DF9300D000D0CDB756
:10BE3000DEB760E571E187EB97E00E94A85A87E9D9
:10BE4000E82E8AE0F82E10E090E1C92ED12C1530B2
:10BE5000B9F0F701808190E0A0E0B0E089839A8397
:10BE6000AB83BC83DE82CD82BE016F5F7F4F87EBE9
:10BE700097E00E94D2206EE471E10E94A85A14C09B
:10BE800080919C0A90E0A0E0B0E089839A83AB8324
:10BE9000BC83DE82CD82BE016F5F7F4F87EB97E070
:10BEA0000E94D2200E94725B1F5FFFEFEF1AFF0A11
:10BEB000163069F626960FB6F894DEBF0FBECDBFDA
:10BEC000DF91CF911F91FF90EF90DF90CF90089579
:10BED000CF92DF92EF92FF9280910D0690910E0625
:10BEE000892B09F44CC00E94AA4D6B017C0160E2D1
:10BEF00071E187EB97E00E94A85A2AE0B701A601FA
:10BF000087EB97E00E94E15A80910D0690910E0612
:10BF10000E94942910920E0610920D06109210069F
:10BF200010920F0610920806109207061092AB0AA4
:10BF30001092AA0A1092240B1092230B1092280B35
:10BF40001092270B1092260B1092250B0E94AA4DDF
:10BF50006B017C016BE171E187EB97E00E94A85ACD
:10BF60002AE0B701A60187EB97E00E94E15A87EB30
:10BF700097E0FF90EF90DF90CF900C94725BFF9072
:10BF8000EF90DF90CF9008955F926F927F928F92A3
:10BF90009F92AF92BF92CF92DF92EF92FF920F9358
:10BFA0001F93CF93DF93CDB7DEB7E4970FB6F89426
:10BFB000DEBF0FBECDBF6C017B013A01590161E0CC
:10BFC0000E946520002361F0682F6062C6010E9414
:10BFD00040206AE071E187EB97E00E94A85AC0C058
:10BFE0001AA219A2FE01B3968EE0DF011D928A9576
:10BFF000E9F720E030E043E050E060E2CE01019656
:10C000000E94194DD6011296ED91FC911397608113
:10C01000718140E250E0CE0101960E944B7BB2E07C
:10C02000EB16F104C9F03CF4E114F104E1F0EA94F8
:10C03000EF2879F05FC086E0E816F10451F09EE049
:10C04000E916F10481F0A5E0EA16F10409F052C006
:10C0500003C064E674E002C067E674E0CE01819636
:10C060000E94447B50C0A114B10409F44CC0850166
:10C07000C12CD12C82E3A82E85E0B82E94E0592E55
:10C080007E01B1E3EB0EF11C4301E1E08E1A910851
:10C09000C614D704C4F5D8018C9111969C910E5FFB
:10C0A0001F4F9F938F93BF92AF921F925F92FF9209
:10C0B000EF920E94787B40E150E0B701CE0181967B
:10C0C0000E944B7B0FB6F894DEBF0FBECDBFC814E5
:10C0D000D90461F065E375E0C7010E94447B40E14B
:10C0E00050E0B701CE0181960E944B7BFFEFCF1A43
:10C0F000DF0ACECF6CEF70E187EB97E00E94A85A81
:10C100008FEF9FEF2FC066EF70E187EB97E00E9403
:10C11000A85ABE016F5F7F4F87EB97E00E94765B66
:10C1200063EF70E187EB97E00E94A85ABE016F5D54
:10C130007F4F87EB97E00E94765B87EB97E00E944A
:10C14000725B0E94D226882359F08091A505811147
:10C1500007C0BE016F5D7F4FCE0101960E94E427AC
:10C1600080E090E0E4960FB6F894DEBF0FBECDBF3E
:10C17000DF91CF911F910F91FF90EF90DF90CF90C3
:10C18000BF90AF909F908F907F906F905F90089539
:10C19000FF920F931F93CF93DF93CDB7DEB729970D
:10C1A0000FB6F894DEBF0FBECDBF8C010E94A91F51
:10C1B000882309F46BC060E0C8010E946520D801A3
:10C1C0001896FC90B7E0FB1671F0823009F45CC061
:10C1D00020F4813009F45DC006C0853009F454C0F4
:10C1E000863009F456C0C8010E94EE1F362F272F53
:10C1F0004F2D50E04A30510508F046C0FA0188271B
:10C20000EE51FF4F8F4F0C94EE76D8011496ED91BE
:10C21000FC91159780858530B9F567EE70E187EB65
:10C2200097E00E94A85AD8011496ED91FC911597B9
:10C23000068117810115110539F1F80161857285B3
:10C24000CE0101960E94D125CE0101960E94A91F20
:10C25000882311F1CE0101960E94C860892BE1F07C
:10C260006FED70E187EB97E00E94A85A12C0292F6A
:10C27000990F330B03C0832F922F9C0181E090E034
:10C28000232B81F480E00EC080E004C08FEF9FEF8D
:10C2900009C081E090E006C0D80112960D911C9172
:10C2A0001397C8CF29960FB6F894DEBF0FBECDBF47
:10C2B000DF91CF911F910F91FF9008953FB7F894B0
:10C2C0008091430B9091440BA091450BB091460B8C
:10C2D00026B5A89B05C02F3F19F00196A11DB11DE1
:10C2E0003FBFBA2FA92F982F8827820F911DA11D1C
:10C2F000B11DBC01CD0142E0660F771F881F991F59
:10C300004A95D1F7089590E0FC013197E231F105AB
:10C3100008F04EC08827E451FF4F8F4F0C94EE7603
:10C32000809180008F7703C0809180008F7D809303
:10C330008000089580918000877FF9CF84B58F7742
:10C3400002C084B58F7D84BD08958091B0008F7741
:10C3500003C08091B0008F7D8093B00008958091DC
:10C3600090008F7707C0809190008F7D03C08091EF
:10C370009000877F8093900008958091A0008F7730
:10C3800007C08091A0008F7D03C08091A000877FAF
:10C390008093A0000895809120018F7707C080913D
:10C3A00020018F7D03C080912001877F8093200131
:10C3B0000895CF93DF9390E0FC01E45FF24F249166
:10C3C000FC01EE5AF24F8491882361F190E0880FCE
:10C3D000991FFC01EE50F34FC591D491FC01EE562C
:10C3E000F34FA591B491611109C09FB7F89488816A
:10C3F000209582238883EC912E230BC0623061F458
:10C400009FB7F8948881322F309583238883EC91ED
:10C410002E2B2C939FBF06C08FB7F894E8812E2B4C
:10C4200028838FBFDF91CF9108958F929F92AF9213
:10C43000BF92CF92DF92EF92FF926B017C010E943C
:10C440005E614B015C01C114D104E104F104F1F01F
:10C450000E945E61DC01CB0188199909AA09BB0918
:10C46000883E9340A105B10570F321E0C21AD108BE
:10C47000E108F10888EE880E83E0981EA11CB11C2B
:10C48000C114D104E104F10419F7DDCFFF90EF905E
:10C49000DF90CF90BF90AF909F908F9008952FB76F
:10C4A000F89460913F0B7091400B8091410B9091FB
:10C4B000420B2FBF08951F920F920FB60F921124B7
:10C4C0002F933F938F939F93AF93BF9380913F0B95
:10C4D0009091400BA091410BB091420B30913E0BDB
:10C4E00023E0230F2D3720F40196A11DB11D05C0B7
:10C4F00026E8230F0296A11DB11D20933E0B8093C9
:10C500003F0B9093400BA093410BB093420B809153
:10C51000430B9091440BA091450BB091460B0196B3
:10C52000A11DB11D8093430B9093440BA093450B29
:10C53000B093460BBF91AF919F918F913F912F91F7
:10C540000F900FBE0F901F901895CF93DF93CDB72C
:10C55000DEB7C656D1090FB6F894DEBF0FBECDBF09
:10C56000789484B5826084BD84B5816084BD85B5CE
:10C57000826085BD85B5816085BD80916E008160DA
:10C5800080936E0010928100809181008260809380
:10C590008100809181008160809381008091800082
:10C5A0008160809380008091B10084608093B100AD
:10C5B0008091B00081608093B00080919100826092
:10C5C000809391008091910081608093910080918F
:10C5D00090008160809390008091A10082608093A0
:10C5E000A1008091A10081608093A1008091A000B2
:10C5F00081608093A000809121018260809321015D
:10C6000080912101816080932101809120018160CE
:10C610008093200180917A00846080937A008091D9
:10C620007A00826080937A0080917A0081608093A2
:10C630007A0080917A00806880937A001092C1001D
:10C640001092E6051092A4051092A30526E040E0A2
:10C6500052EC61E070E087EB97E00E94F6376BE503
:10C6600078E087EB97E00E94A85A64EC7FE486EDBF
:10C6700093E00E94635D68E07FE48BED93E00E94AD
:10C68000635D66EF72E580EE93E00E94635D68E5AE
:10C6900071E385EE93E00E94635D6FED7AE289EECF
:10C6A00093E00E94635D62EB7FE48DEE93E00E9475
:10C6B000635D66E47FE482EF93E00E94635D6CE675
:10C6C0007EE486EF93E00E94635D6AE37EE489EF97
:10C6D00093E00E94635D67E57EE48DEF93E00E9446
:10C6E000635D61E37EE483E094E00E94635D0E9409
:10C6F000332E57E9C52E5AE0D52E5601F12C00E015
:10C7000010E0C8010E946576F50181935F018150B8
:10C710008E3F10F4FF24F3940F5F1F4F0630110576
:10C7200081F7FF20B1F10E940E5F0E94935261E0F9
:10C730008DE00E94D96126E040E855E260E070E0BB
:10C740008AE197E00E94F6378AE19EE29093180A08
:10C750008093170A8BED9AE290931A0A8093190A34
:10C7600087ED9AE290931C0A80931B0A64E170E0C3
:10C7700080E090E00E94156286E39EE59093F408C5
:10C780008093F30864EF71E080E090E00E9415620E
:10C790005BC06FE578E087EB97E00E94A85A4DE90F
:10C7A000A42E4AE0B42E04EC13E040E150E060E037
:10C7B00070E0C8010E94DF6DF60161936F016AE3CA
:10C7C00070E0C8010E94307B009709F4ACCFFC01F7
:10C7D0002081222309F4A7CF8C010F5F1F4FAC14D7
:10C7E000BD0419F7A0CF87EB97E00E941B59182FC3
:10C7F0008A3061F5E091E605F0E0E655FA4F1082E7
:10C800006AE074E087EB97E00E94765B8AEA95E045
:10C810000E94A45D1092E60587EB97E00E943D59C7
:10C82000892B09F70E946411029714F00E94295481
:10C830000E9434228091070690910806892B49F5C1
:10C840000E943D2B0E94EE59A895E6CF8D3091F2C3
:10C85000883069F468E087EB97E00E94635A809122
:10C86000E6058823C9F281508093E605D5CF682F6D
:10C8700087EB97E00E94635AE091E605EB3360F6A0
:10C8800081E08E0F8093E605F0E0E655FA4F1083C5
:10C89000C3CF8091A8059091A905049709F4CAC354
:10C8A0000E944F620091E7051091E8052091E9058B
:10C8B0003091EA05061717072807390708F0BAC3A9
:10C8C00020E022242394312CE091A605F091A705C5
:10C8D000309709F4AFC32111ADC38085853009F0CD
:10C8E00092C321E732E063963FAF2EAF6397659620
:10C8F000FFAFEEAF6597CE018F5A9F4F0E94782011
:10C900000E944F622B013C016A968FAD6A9784307A
:10C9100061F008F460C3883009F45DC3893009F41C
:10C92000D8C0853009F05CC356C38091050690914C
:10C930000606892B09F0C5C0CE018F5A9F4F0E9471
:10C94000EF278111BEC06796AEACBFAC6797F5010B
:10C950008085853009F064C4C5010E94123BC82E51
:10C96000D12CF2E0CF16D1040CF45AC43092060652
:10C970002092050660E070E0CE018F5A9F4F0E9422
:10C9800012204C0161E070E0CE018F5A9F4F0E944F
:10C9900012208C01F5E0CF16D1040CF4B2C464E08F
:10C9A000C5010E947037FC01C184D28426E240E8B0
:10C9B00055E260E070E08AE197E00E94F6378092ED
:10C9C00005098AE197E09093040980930309109286
:10C9D000100A1092120A1092110AF1E0CF16D10437
:10C9E00009F43FC40CF423C432E0C316D10409F0A7
:10C9F0002AC410930709009306093092090920926E
:10CA0000080983E00E945B386F968FAF6F976F962F
:10CA10005FAD6F97511136C480910A0990910B094F
:10CA2000A1969FAF8EAFA197092E000CAA0BBB0B4E
:10CA300089839A83AB83BC83E0E1F0E0FE83ED83DE
:10CA40006596EEADFFAD6597C080D18067EE78E06A
:10CA500087EB97E00E94A85AB60187EB97E00E9407
:10CA6000765B60EE78E087EB97E00E94A85ABE0103
:10CA70006F5F7F4F87EB97E00E94D2200E94725B2E
:10CA8000A1966EAD7FADA197CE018F5A9F4F0E94A8
:10CA900029281092060610920506C090A605D0908F
:10CAA000A705F6018281938121E732E03A83298349
:10CAB0009C838B83CE0101960E947820CD2809F0BB
:10CAC00000C4CE018F5A9F4F0E94ED2880ED97E061
:10CAD00089C28091050690910606892B91F7CE01B7
:10CAE0008F5A9F4F0E94EF278111EBCF309206069D
:10CAF000209205060E94BC356C01892B19F086E056
:10CB0000F601808720E030E043E050E060E2CE01B3
:10CB100001960E94194D6596EEADFFAD6597608157
:10CB200071814FE150E0CE0101960E944B7B6DE098
:10CB300074E0CE0101960E94257B26E040E855E294
:10CB400060E070E08AE197E00E94F63760E070E014
:10CB5000CE018F5A9F4F0E941220809305098AE1CF
:10CB600097E090930409809303091092100A1092A1
:10CB7000120A1092110A24E338E030930709209337
:10CB800006094AE050E0509309094093080983E000
:10CB90000E945B388111C1C060EC78E087EB97E0C0
:10CBA0000E94A85A0AE019E02EE1A22E29E0B22E36
:10CBB000F801819191918F01092E000CAA0BBB0BFA
:10CBC00025968CAF9DAFAEAFBFAF259720E130E08B
:10CBD00027963FAF2EAF2797BE016F5B7F4F87EB46
:10CBE00097E00E94D2206EEB78E00E94A85AA0162F
:10CBF000B106F1F687EB97E00E94725B60910E0937
:10CC000070910F09072E000C880B990B0E94287851
:10CC100020E030E048EC52E40E947E779B01AC01BA
:10CC200063E174E0C6010E944C2900911209109141
:10CC30001309A80165E174E0C6010E94BC37609148
:10CC4000140970911509072E000C880B990B0E948E
:10CC5000287820E030E048EC52E40E947E779B0187
:10CC6000AC0169E174E0C6010E944C29609116098B
:10CC700070911709072E000C880B990B0E942878D9
:10CC800020E030E040E251E40E947E779B01AC015D
:10CC900067E174E0C6010E944C2940910A09509155
:10CCA0000B096BE174E0C6010E94BC37012B09F44B
:10CCB00052C067968EAD9FAD6797FC0120852530E9
:10CCC00009F049C061E00E947037009709F443C041
:10CCD00024E630E06C963FAF2EAF6C97FC01618587
:10CCE0007285CE018F5B9F4F0E94D125CE018F5B55
:10CCF0009F4F0E94A91F882371F1E12CF12C01E0C4
:10CD00009E01265A3F4F41E050E060E070E0CE01C6
:10CD10008F5B9F4F0E94DF081EC090E0A0E0B0E054
:10CD200025968CAF9DAFAEAFBFAF259720E130E029
:10CD300027963FAF2EAF279768EA78E087EB97E01A
:10CD40000E94A85ABE016F5B7F4F87EB97E00E945D
:10CD5000D2200E94725B80910A0983FF14C08EE387
:10CD600098E0909307098093060930920909209270
:10CD7000080983E00E945B3881110CC040910A09C8
:10CD800050910B0902C040E050E06EE174E0C60132
:10CD90000E94BC3762E370E080E090E00E94156280
:10CDA00043E150E0509307094093060984E090E086
:10CDB000909309098093080983E00E945B388111F0
:10CDC000A7C06EE978E087EB97E00E94A85A0AE0D6
:10CDD00019E092E1A92E99E0B92EF80161917191C3
:10CDE0008F0187EB97E00E9456376CE978E087EB7C
:10CDF00097E00E94A85AA016B10679F787EB97E052
:10CE00000E94725B00910A0910910B09011511052E
:10CE1000D1F0B801012E000C880B990B0E942878E4
:10CE20002DEE3EE94CE35EE30E94DD7822E538EB2F
:10CE300042E152E40E940C779B01AC0162E274E093
:10CE4000C6010E944C2960910C0970910D09072EB2
:10CE5000000C880B990B0E9428782DEE3EE94CE3DC
:10CE60005EE30E94DD7822E538EB42E152E40E9465
:10CE70000C774B015C019B01AC0161E174E0C601E0
:10CE80000E944C296091100970911109161617061D
:10CE9000A4F4072E000C880B990B0E94287820E040
:10CEA00030E040E251E40E947E779B01AC0166E2F3
:10CEB00074E0C6010E944C2907C040E050E066E2E1
:10CEC00074E0C6010E94BC3720E030E040E252E44A
:10CED000C501B4010E94D8781816B4F5012BA1F150
:10CEE0000E94D226882329F08091A505882309F481
:10CEF0002CC2E12CF12C01E020E030E040E050E0D9
:10CF000062E070E0CE018F5A9F4F0E94DF081CC084
:10CF100090E0A0E0B0E025968CAF9DAFAEAFBFAF84
:10CF2000259720E130E027963FAF2EAF279766E8A0
:10CF300078E087EB97E00E94A85ABE016F5B7F4FB5
:10CF400087EB97E00E94D22080E091E00E941C6C69
:10CF50008C01892B61F125961FAE1EAE2597279671
:10CF60001FAE1EAE27978FEF9FEF29969FAF8EAF14
:10CF700029978DE392E023969FAF8EAF23972B9650
:10CF80001FAE1EAE2B972D961FAF0EAF2D9780E0D4
:10CF900091E061969FAF8EAF61972F961FAE1EAE48
:10CFA0002F97B601CE018F5B9F4F0E94C5330E9421
:10CFB000D226882329F08091A505882309F4D0C1C1
:10CFC000C8010E94B46CC6010E9494291092060602
:10CFD0001092050676CDCE018F5A9F4F0E94ED2804
:10CFE00084E690E0092E000CAA0BBB0B480E591EDC
:10CFF0006A1E7B1E4092E7055092E8056092E905A3
:10D000007092EA0521E0E091A605F091A7058281E2
:10D0100093819093A7058093A605892B09F054CCA2
:10D02000E0910706F0910806868197819093A70505
:10D030008093A6050E944F620091EB051091EC05CC
:10D040002091ED053091EE05601771078207930777
:10D0500008F4F6CBE0910706F0910806309709F442
:10D06000EFCB06811781F12C0115110541F1F80173
:10D070008085853001F560E0C8010E947037FC01B1
:10D0800081859285A385B4850597A105B10599F49D
:10D09000C8010E94123B90E005976CF064E0C80163
:10D0A0000E9470371C01892B31F0C1010E94123B94
:10D0B000823008F05BC1F80102811381D5CF0E9454
:10D0C0004F62DC01CB0188579C4EAF4FBF4F80931E
:10D0D000EB059093EC05A093ED05B093EE050E944F
:10D0E000AA4D2B013C010E944F624B015C010E9442
:10D0F000D226882309F462C020E030E041E050E00D
:10D1000060E4CE0101960E94194D40E450E067E2D0
:10D1100079E0CE0101960E941C6F62EC73E0CE01B3
:10D1200001960E94257B40E450E06EE179E0CE015B
:10D1300001960E941C6FB301A201CE018F5B9F4F2D
:10D140000E94BE4CBE016F5B7F4FCE0101960E94D4
:10D15000E42720E030E041E050E060E4CE010196B9
:10D160000E94194D40E450E067E279E0CE0101965B
:10D170000E941C6F62EC73E0CE0101960E94257B39
:10D1800040E450E067E179E0CE0101960E941C6F17
:10D19000C501B40128EE33E040E050E00E948B76F8
:10D1A000BA01A901CE018F5B9F4F0E94BE4CBE0108
:10D1B0006F5B7F4FCE0101960E94E427FF20C1F0F4
:10D1C0000E94AA4D4B015C0162E379E087EB97E096
:10D1D0000E94A85A2AE0B501A40187EB97E00E94BB
:10D1E000E15A63E474E087EB97E00E94765B28CB1A
:10D1F0000E94AA4D4B015C0160E379E087EB97E068
:10D200000E94A85A2AE0B501A40187EB97E00E948A
:10D21000E15A6EE279E087EB97E00E94A85A10CBC2
:10D2200064E079E087EB97E00E94A85A4ACCCD28C9
:10D2300011F510930709009306093092090920920D
:10D24000080981E0DFCB43E0C416D104A1F41093B8
:10D25000070900930609309209092092080984E021
:10D26000D1CB1093070900930609D0920909C09207
:10D27000080982E0C7CB6CEE78E087EB97E00E946C
:10D28000A85AC5CB6F96FFAD6F978F2F90E0A0E0A7
:10D29000B0E089839A83AB83BC8320E130E03E8396
:10D2A0002D836AEC78E087EB97E00E94A85ABE01D4
:10D2B0006F5F7F4F87EB97E00E94D2200E94725BE6
:10D2C000E8CBCE0101960E94A91F882309F4F9CB6F
:10D2D0008985843009F0F5CB60E070E0CE010196DD
:10D2E0000E9412208816990609F0EBCB61E070E0ED
:10D2F000CE0101960E9412200817190709F0E1CB10
:10D3000004C082E0C82ED12C51CBA1966EAD7FAD6A
:10D31000A197CE0101960E942928E091A605F091DF
:10D32000A705828193819093A7058093A605892BF9
:10D3300009F0C7CBE0910706F09108068681978136
:10D340009093A7058093A605BCCB6596EEADFFAD87
:10D3500065976081718186E394E00E948929C9CD37
:10D36000B801CE0101960E9489292ACE61E0C80148
:10D370000E947037FC01F184D28462E0C8010E94EF
:10D380007037FC0181849284A384B48463E0C80173
:10D390000E947037FC012185328543855485A5960E
:10D3A0002CAF3DAF4EAF5FAFA59760E0C1010E94CB
:10D3B0007037FC01418452846384748461E0C1014C
:10D3C0000E947037FC014185528563857485411543
:10D3D00051056105710571F4F8016081718187EB78
:10D3E00097E00E94765B67E679E087EB97E00E9422
:10D3F000A85A14C04150510961097109FC014187C3
:10D40000528763877487452B462B472B39F4F801E5
:10D41000608171818AE294E00E94892920E030E0F5
:10D4200048E152E4C301B2010E94D87818163CF4D6
:10D43000F8016081718186E394E00E9489296D96EC
:10D44000FFAE6D976E96DFAE6E97C501B4010E9478
:10D4500028784B015C01A396CEACDFACA397F80112
:10D460000190F081E02DA796FFAFEEAFA79787EB75
:10D4700097E00E94725BA7966EAD7FADA79787EB92
:10D4800097E00E94765B61E679E087EB97E00E9487
:10D49000A85A42E0C501B4010E94FD296BE579E07C
:10D4A00087EB97E00E94A85A42E0C301B2010E94B4
:10D4B000FD2965E579E087EB97E00E94A85AA396DD
:10D4C0006EAD7FADA39787EB97E00E9456376E96BF
:10D4D0002EAD3FAD6E9761E08F2D37FF08C081956F
:10D4E0000E94D96132E0C316D10449F41FC00E94E2
:10D4F000D96142E0C416D10409F069C01CC035E00E
:10D50000C316D10499F061E0C1010E947037FC019B
:10D5100081859285A385B485892B8A2B8B2B91F4E9
:10D520006E962EAD3FAD6E9737FF05C060E08F2D34
:10D5300081950E94004160E08F2D0E94004160E5CE
:10D5400079E021C020E030E040E85FE3C501B401AC
:10D550000E940C779B01AC01C301B2010E94797754
:10D5600087FF18C06E962EAD3FAD6E9737FF05C092
:10D5700060E08F2D81950E94004161E08F2D0E9417
:10D5800000416CE479E087EB97E00E94A85AFF2401
:10D59000F39491CDA3019201C501B4010E94797762
:10D5A000181694F06E964EAD5FAD6E9757FF05C09E
:10D5B00061E08F2D81950E94004160E08F2D0E94D7
:10D5C000004167E479E0DFCF68E379E0DCCF45E054
:10D5D000C416D10409F4AFCF96CFEAE1F7E0138285
:10D5E000128248EE53E060E070E044835583668326
:10D5F00077838FE892E09183808325ED30E0358753
:10D60000248724ED30E03787268720ED30E0318B0A
:10D61000208B21ED30E0338B228B22ED30E0358BF7
:10D62000248B26ED30E0378B268B118E128E138ED5
:10D63000148EE7EBF7E013821282448355836683EE
:10D6400077839183808385EC90E09587848784EC51
:10D6500090E09787868780EC90E0918B808B81ECBF
:10D6600090E0938B828B82EC90E0958B848B86ECA0
:10D6700090E0978B868B118E128E138E148EEAE2B9
:10D68000FAE081E293E09183808312821382148214
:10D690001582E0E3FAE09183808312821382148280
:10D6A0001582E6E3FAE0918380831282138214826A
:10D6B0001582E4E5F8E0918380831282138214825C
:10D6C0001582ECE3FAE09183808312821382148244
:10D6D0001582E2E4FAE0918380831282138214823D
:10D6E0001582E8E4FAE09183808312821382148227
:10D6F0001582EEE4FAE09183808312821382148211
:10D700001582EAE5F8E09183808312821382148205
:10D710001582E4E5FAE0138212824483558366831E
:10D72000778321EA32E031832083E0E6FAE09183D7
:10D7300080831282138214821582E6E6FAE09183D6
:10D7400080831282138214821582EDE1FAE0138243
:10D75000128244835583668377832BEF32E03183D3
:10D76000208324E024871092180A1092170A10923E
:10D770001A0A1092190A10921C0A10921B0AA2E6A9
:10D78000B8E013961C921E92129723EB32E011968A
:10D790003C932E939093F6088093F5081092F70827
:10D7A0001092F8081092F9081092FA082FEF3FEF44
:10D7B00030930209209301091596FC93EE93149778
:10D7C000109200091092FF08ECE6FAE09183808342
:10D7D0001282138214821582E2E7FAE09183808339
:10D7E0001282138214821582E8E7FAE09183808323
:10D7F0001282138214821582EEE7FAE0918380830D
:10D800001282138214821582E4E8FAE09183808305
:10D810001282138214821582EAE8FAE08FEF808385
:10D8200012821182148613868FEF9FEFDC018783AB
:10D830009087A187B28708950F931F93CF93DF93AB
:10D840008230910510F482E090E0E0914B0BF09172
:10D850004C0B20E030E0A0E0B0E0309719F14081BF
:10D8600051810281138148175907C8F08417950721
:10D8700069F4109731F012960C93129713961C933B
:10D8800027C000934B0B10934C0B22C02115310580
:10D8900019F04217530718F49A01BD01EF01DF0197
:10D8A000F801DBCF21153105F9F0281B390B2430A5
:10D8B000310580F48A819B816115710521F0FB019E
:10D8C0009383828304C090934C0B80934B0BFE0197
:10D8D000329644C0FE01E20FF31F819391932250D0
:10D8E0003109398328833AC02091490B30914A0B82
:10D8F000232B41F420910A0230910B0230934A0B02
:10D900002093490B2091080230910902211531051D
:10D9100041F42DB73EB740910C0250910D02241BEB
:10D92000350BE091490BF0914A0BE217F307A0F495
:10D930002E1B3F0B2817390778F0AC014E5F5F4F65
:10D940002417350748F04E0F5F1F50934A0B409342
:10D95000490B8193919302C0E0E0F0E0CF01DF91A9
:10D96000CF911F910F910895CF93DF93009709F402
:10D9700081C0FC01329713821282A0914B0BB091AF
:10D980004C0B109781F420813181820F931F2091DD
:10D99000490B30914A0B2817390751F5F0934A0B80
:10D9A000E093490B67C0ED0120E030E0CE17DF07C0
:10D9B00040F44A815B819E0141155105F1F0EA0175
:10D9C000F5CFD383C28340815181840F951FC8173F
:10D9D000D90759F488819981840F951F0296918304
:10D9E00080838A819B81938382832115310529F469
:10D9F000F0934C0BE0934B0B3DC0E901FB83EA83B2
:10DA000049915991C40FD51FEC17FD0761F480812E
:10DA10009181840F951F0296E90199838883828101
:10DA200093819B838A83E0E0F0E012968D919C9134
:10DA30001397009719F0FD01DC01F7CF8D919C91B0
:10DA400011979D012E5F3F4F820F931F2091490B2D
:10DA500030914A0B2817390769F4309729F410924E
:10DA60004C0B10924B0B02C013821282B0934A0BE4
:10DA7000A093490BDF91CF9108958F929F92AF921F
:10DA8000BF92CF92DF92EF92FF92CF93DF93EC01A0
:10DA9000688179818A819B81611571058105910574
:10DAA00021F464E279ED8BE597E02DE133EF41E07D
:10DAB00050E00E94AD7649015A019B01AC01A7EAF2
:10DAC000B1E40E94CC766B017C01ACEEB4EFA50111
:10DAD00094010E94DA76DC01CB018C0D9D1DAE1DF8
:10DAE000BF1DB7FF03C00197A109B0488883998380
:10DAF000AA83BB83BC01CD019F77DF91CF91FF90BB
:10DB0000EF90DF90CF90BF90AF909F908F9008954F
:10DB10008F929F92AF92BF92CF92DF92EF92FF923D
:10DB200060910E0270910F0280911002909111028B
:10DB3000611571058105910521F464E279ED8BE5AC
:10DB400097E02DE133EF41E050E00E94AD764901CE
:10DB50005A019B01AC01A7EAB1E40E94CC766B01AB
:10DB60007C01ACEEB4EFA50194010E94DA76DC01F1
:10DB7000CB018C0D9D1DAE1DBF1DB7FF03C00197CE
:10DB8000A109B04880930E0290930F02A093100257
:10DB9000B0931102BC01CD019F77FF90EF90DF9011
:10DBA000CF90BF90AF909F908F90089560930E029A
:10DBB00070930F02809310029093110208953F9288
:10DBC0004F925F926F927F928F929F92AF92BF928D
:10DBD000CF92DF92EF92FF920F931F93CF93DF9339
:10DBE0005C016B017A016115710519F0FB019183EC
:10DBF0008083E114F10429F0C7010297839708F0AC
:10DC0000C9C0E5012196F5011081812F90E00E94A5
:10DC10000A6F892B11F05E01F4CF1D3229F4219691
:10DC2000F501118101E007C01B3221F4E5012296C4
:10DC3000F501118100E0E114F104B1F0F0E1EF161B
:10DC4000F10429F4B0C010E3E114F10401F12AE079
:10DC5000E216F104B1F180E1E816F10471F0E8E0B8
:10DC6000EE16F104F1F413C0103341F588818F7D75
:10DC7000883549F7198122960260F0E1EF2EF12CE8
:10DC800088248A94982CA82CAFE0BA2E20C078E083
:10DC9000E72EF12C88248A94982CA82CEFE1BE2E34
:10DCA00016C06FEF7FEFCB0197010F2C000C440BD8
:10DCB000550B0E948B7649015A0109C08AE0E82E73
:10DCC000F12C69E9862E982CA82C69E1B62E40E04B
:10DCD00060E070E0CB0127010F2C000C660877088C
:10DCE000FE0150ED352E310E29E0231570F42FEB97
:10DCF000210F2A3118F439EC332E06C02FE9210FF9
:10DD00002A3130F529EA322E310E232D30E02E153E
:10DD10003F05F4F44F3FC9F086169706A806B906EA
:10DD200088F0A30192010E947B76232D30E040E031
:10DD300050E0620F731F841F951F621773078407DB
:10DD4000950710F44FEF01C041E021961081C8CF34
:10DD5000C114D10451F0442311F0219703C001FFF5
:10DD600004C02297F601D183C08300FF07C09095BD
:10DD70008095709561957F4F8F4F9F4F4F3F79F4FE
:10DD800082E290E09093540B8093530B3FEF2FEF80
:10DD90009FEF0DC040E030E020E090E008C0462F4B
:10DDA000372F282F04C0103309F067CF5FCF642FBF
:10DDB000732F822FDF91CF911F910F91FF90EF90E2
:10DDC000DF90CF90BF90AF909F908F907F906F909B
:10DDD0005F904F903F900895FC0188279927E89421
:10DDE00021912032E9F3293010F02E30C8F32B3284
:10DDF00041F02D3239F4689404C00E94716F820F93
:10DE0000911D219120532A30C0F31EF490958195E5
:10DE10009F4F089591110C947775803219F08950B5
:10DE20008550C8F70895FB01DC018D91059080199C
:10DE30000110D9F3990B0895FB01DC010D9000202E
:10DE4000E9F711974150504028F0059000200D92BD
:10DE5000C9F708951C920895FB01DC014150504020
:10DE600048F005900D920020C9F701C01D92415065
:10DE70005040E0F7089547E45BE00C943F6FFA01EF
:10DE8000A191B081009719F41097E1F0CD01DC0168
:10DE9000CD010D90002011F4C00113C0FB012191B0
:10DEA000222319F02015D9F7F3CFFB01219120157A
:10DEB00019F41E92119606C02223C1F70D9000207E
:10DEC000A1F7D001FA01A193B0830895BB274A308E
:10DED00031F4992322F4BDE2909581959F4F0C94E3
:10DEE0007A6F7AE0979F902D879F802D910D112456
:10DEF0000895BB27FB015527AA27880F991FAA1F42
:10DF0000A41710F0A41B83955051B9F7A05DAA3354
:10DF100008F0A95DA193009779F7B111B19311921F
:10DF2000CB010C94A275FC01238127FF10C0EDE406
:10DF3000FBE0208131818217930711F41182108256
:10DF400032962BE0E335F207A1F70E94B46C80E033
:10DF500090E008950F931F93CF93DF93009731F4D0
:10DF60006115710519F480E090E03AC08B01EC0175
:10DF70006EE070E081E090E00E945B75FC01892B0F
:10DF800091F380E883830115110571F013870287EF
:10DF900081E8838380914D0B90914E0B892B21F466
:10DFA000F0934E0BE0934D0B2097C9F0D187C087BB
:10DFB00083818260838380914F0B9091500B892BDA
:10DFC00071F4F093500BE0934F0B8091510B9091B3
:10DFD000520B892B21F4F093520BE093510BCF019C
:10DFE000DF91CF911F910F910895CF93DF93EC01B3
:10DFF0002B8120FF33C026FF0AC02F7B2B838E810D
:10E000009F8101969F838E838A8190E029C022FFA1
:10E010000FC0E881F9818081082E000C990B0097D0
:10E0200019F420622B831AC03196F983E8830EC05D
:10E03000EA85FB85199597FF09C02B81019611F0A0
:10E0400080E201C080E1822B8B8308C02E813F815A
:10E050002F5F3F4F3F832E83992702C08FEF9FEFA3
:10E06000DF91CF9108950F931F93CF93DF93CDB797
:10E07000DEB708851985F801838188608383AE0146
:10E08000445F5F4F6A857B85C8010E946D70F8010F
:10E090002381277F2383DF91CF911F910F910895D3
:10E0A0000F931F93CF93DF93CDB7DEB70885198504
:10E0B000F801838188608383AE01445F5F4F6A8586
:10E0C0007B85C8010E943674F8012381277F238352
:10E0D000DF91CF911F910F9108952F923F924F9210
:10E0E0005F926F927F928F929F92AF92BF92CF92E8
:10E0F000DF92EF92FF920F931F93CF93DF93CDB7F1
:10E10000DEB72B970FB6F894DEBF0FBECDBF6C0104
:10E110007B018A01FC0117821682838181FFCCC1B9
:10E12000CE0101963C01F6019381F70193FD8591A3
:10E1300093FF81917F01882309F4BAC1853239F4B4
:10E1400093FD859193FF81917F01853229F4B6017A
:10E1500090E00E94B275E7CF912C212C312CFFE189
:10E16000F315D8F08B3279F038F4803279F08332BD
:10E17000A1F4232D20611DC08D3261F0803369F43C
:10E18000232D216016C0832D8260382EE32DE4609C
:10E190003E2E2AC0F32DF8601DC037FC2DC020EDA7
:10E1A000280F2A3040F08E32B9F436FC81C1232D7D
:10E1B0002064322E19C036FE06C08AE0989E200DDB
:10E1C0001124922E11C0EAE02E9E200D1124222E41
:10E1D000F32DF0623F2E08C08C3621F4832D806829
:10E1E000382E02C0883641F4F70193FD859193FFE4
:10E1F00081917F018111B3CF982F9F7D95549330EA
:10E2000028F40C5F1F4F9FE399830DC0833631F0D4
:10E21000833771F0833509F059C021C0F80180813E
:10E2200089830E5F1F4F88248394912C530113C060
:10E230002801F2E04F0E511CF801A080B18036FE9B
:10E2400003C0692D70E002C06FEF7FEFC5010E942F
:10E2500097754C018201F32DFF773F2E16C02801E0
:10E2600022E0420E511CF801A080B18036FE03C0AE
:10E27000692D70E002C06FEF7FEFC5010E948575C8
:10E280004C01F32DF0683F2E820133FC1BC0822D20
:10E2900090E088169906B0F4B60180E290E00E9402
:10E2A000B2752A94F4CFF50137FC859137FE819140
:10E2B0005F01B60190E00E94B27521102A9421E01E
:10E2C000821A91088114910471F7E8C0843611F024
:10E2D000893641F5F80137FE07C06081718182817E
:10E2E00093810C5F1F4F08C060817181072E000C65
:10E2F000880B990B0E5F1F4FF32DFF763F2E97FF74
:10E3000009C090958095709561957F4F8F4F9F4F75
:10E31000F0683F2E2AE030E0A3010E940776882EA5
:10E32000861845C0853731F4232D2F7EB22E2AE082
:10E3300030E025C0932D997FB92E8F36C1F018F4A7
:10E34000883579F0B5C0803719F0883721F0B0C032
:10E35000E92FE061BE2EB4FE0DC0FB2DF460BF2E90
:10E3600009C034FE0AC0292F2660B22E06C028E05C
:10E3700030E005C020E130E002C020E132E0F801E9
:10E38000B7FE07C060817181828193810C5F1F4F4E
:10E3900006C06081718180E090E00E5F1F4FA30195
:10E3A0000E940776882E8618FB2DFF773F2E36FEBB
:10E3B0000DC0232D2E7FA22E891458F434FE0BC0DD
:10E3C00032FC09C0832D8E7EA82E05C0B82CA32C4C
:10E3D00003C0B82C01C0B92CA4FE0FC0FE01E80D8B
:10E3E000F11D8081803321F49A2D997EA92E09C0D8
:10E3F000A2FE06C0B394B39404C08A2D867809F0B7
:10E40000B394A3FC11C0A0FE06C0B21488F4280C7B
:10E41000922C9B180EC0B21460F4B60180E290E01A
:10E420000E94B275B394F7CFB21418F42B1802C03F
:10E43000982C212CA4FE10C0B60180E390E00E942D
:10E44000B275A2FE17C0A1FC03C088E790E002C02D
:10E4500088E590E0B6010CC08A2D867859F0A1FEBF
:10E4600002C08BE201C080E2A7FC8DE2B60190E021
:10E470000E94B275891438F4B60180E390E00E94DE
:10E48000B2759A94F7CF8A94F301E80DF11D80815B
:10E49000B60190E00E94B2758110F5CF222009F4F8
:10E4A00042CEB60180E290E00E94B2752A94F6CF87
:10E4B000F6018681978102C08FEF9FEF2B960FB6F2
:10E4C000F894DEBF0FBECDBFDF91CF911F910F91AA
:10E4D000FF90EF90DF90CF90BF90AF909F908F9084
:10E4E0007F906F905F904F903F902F90089520FD08
:10E4F00009C0FC0123FD05C022FF02C073836283B3
:10E5000051834083089544FD17C046FD17C0AB01F9
:10E51000BC01DA01FB01AA0FBB1FEE1FFF1F109405
:10E52000D1F74A0F5B1F6E1F7F1FCB01BA01660F29
:10E53000771F881F991F09C033E001C034E0660FC0
:10E54000771F881F991F3150D1F7620F711D811DF0
:10E55000911D08950F931F93CF93DF938C01C801F2
:10E560000E94F56FEC0197FD08C00E940A6F892B8D
:10E57000B1F7B801CE010E94EE75CE01DF91CF91C7
:10E580001F910F9108958F929F92AF92BF92EF9239
:10E59000FF920F931F93CF93DF938C01D62F7A01B5
:10E5A000B22E0E94F56F9C0133272B32310531F0DA
:10E5B0002D32310561F48B2D8068B82ED15011F4C5
:10E5C00080E068C0C8010E94F56F97FDF9CFCB2DA0
:10E5D000CD7F2B2D207309F58033F9F4AA24AA945A
:10E5E000AD0E09F443C0C8010E94F56F97FD3EC00F
:10E5F0009C012F7D33272835310549F4C264D25060
:10E60000A9F1C8010E94F56F97FF07C02FC0B6FEA1
:10E6100002C0C26001C0C261DA2D812C912C54016C
:10E6200020ED280F283080F0C4FF04C0B8010E94FC
:10E63000EE7519C02A3040F0C6FFF8CF2F7D3FEEAF
:10E64000320F363098F727504C2FC501B4010E9485
:10E6500083724B015C01C260D15059F0C8010E9425
:10E66000F56F97FFDDCFC1FD04C0AACF812C912C9F
:10E670005401C7FF08C0B094A09490948094811C6A
:10E68000911CA11CB11C2C2FB501A401C7010E9433
:10E69000777281E0DF91CF911F910F91FF90EF9002
:10E6A000BF90AF909F908F9008955F926F927F92EE
:10E6B0008F929F92AF92BF92CF92DF92EF92FF9292
:10E6C0000F931F93CF93DF93CDB7DEB7A0970FB60D
:10E6D000F894DEBF0FBECDBF5C01962E7A01F90122
:10E6E0008E010F5F1F4F680180E2D8011D928A954D
:10E6F000E9F7D50113968C9080E090E0612C712CA5
:10E7000030E061E070E083FC259183FE21918F0170
:10E71000522E211103C080E090E092C02E3511F4FA
:10E72000009751F1432F50E0481759073CF42D351D
:10E7300059F12D3219F4772009F103C0772009F43B
:10E740006AC0452D469546954695D601A40FB11D44
:10E75000452D47708B0102C0000F111F4A95E2F74B
:10E76000A8015C91452B4C93651459F0561410F494
:10E770005394E7CF5A94E5CF31E004C077247394E3
:10E7800001C0712C0196BFCF772019F08E81806275
:10E790008E83311103C08824839417C0F6019E0133
:10E7A0002F5D3F4F8081809581932E173F07D1F7D2
:10E7B000F2CFE114F10429F0D7018C93F7013196DF
:10E7C0007F019A94812C9920F9F0C5010E94F56F80
:10E7D00097FD18C0FC01FF2723E0F595E7952A95E2
:10E7E000E1F7EC0DFD1D208130E0AC0147705527AD
:10E7F00002C0359527954A95E2F720FDDACFB5019D
:10E800000E94EE75811087CFE114F10411F0D70159
:10E810001C92C80115C0422F469546954695D601D3
:10E82000A40FB11D422F47708B0102C0000F111FB2
:10E830004A95E2F7A8015C91452B4C93622EA2CF3A
:10E84000A0960FB6F894DEBF0FBECDBFDF91CF917B
:10E850001F910F91FF90EF90DF90CF90BF90AF90FE
:10E860009F908F907F906F905F9008955F926F92CE
:10E870007F928F929F92AF92BF92CF92DF92EF9250
:10E88000FF920F931F93CF93DF936C01EB015A011B
:10E89000FC0117821682512CF601E380FE01E3FC95
:10E8A0008591E3FE8191182FEF01882309F4EEC0D2
:10E8B00090E00E940A6F892B21F0C6010E94AA7283
:10E8C000EBCF153241F4FE01E3FC1591E3FE11910B
:10E8D000EF01153281F4C6010E94F56F97FDD4C097
:10E8E000412F50E09C01332724173507A9F2B601C8
:10E8F0000E94EE75CBC01A3239F4E3FC1591E3FEA9
:10E900001191EF0101E001C000E0F12C20ED210F99
:10E910002A3080F402606F2D70E080E090E040E2E9
:10E920000E948372F62EFE01E3FC1591E3FE119125
:10E93000EF01ECCF01FF03C0F11003C0A7C0FF241B
:10E94000FA94183619F01C3651F010C0FE01E3FCA1
:10E950001591E3FE1191EF01183641F4086004604F
:10E96000FE01E3FC1591E3FE1191EF01112309F47F
:10E970008DC0612F70E082E095E00E947A75892B4E
:10E9800009F484C000FD07C0F50180809180C501B5
:10E9900002965C0102C0812C912C1E3651F4F601C6
:10E9A0004681578160E070E0202FC4010E94777299
:10E9B00073CF1336A9F401FD02C0FF24F394C601FE
:10E9C0000E94F56F97FD60C08114910429F0F40155
:10E9D0008083C40101964C01FA94F110F0CF50C02D
:10E9E0001B3559F49E01A4016F2DC6010E94557379
:10E9F000EC01892B09F044C03EC0C6010E94AA72F6
:10EA000097FD42C01F3661F128F4143639F11936EA
:10EA100051F128C0133771F0153701F123C081146B
:10EA2000910429F0F4016082C40101964C01FA942A
:10EA3000FF2071F0C6010E94F56F3C0197FD08C0F0
:10EA40000E940A6F892B59F3B601C3010E94EE752B
:10EA500081149104A9F0F401108212C0006203C075
:10EA6000006101C00064202FA4016F2DC6010E9427
:10EA7000C372811105C0F6018381807329F406C039
:10EA800000FD0ACF539408CF552019F0852D90E052
:10EA900002C08FEF9FEFDF91CF911F910F91FF90F9
:10EAA000EF90DF90CF90BF90AF909F908F907F902E
:10EAB0006F905F9008950F931F93CF93DF93869F7E
:10EAC0008001879F100D969F100D1124C8010E9490
:10EAD0001C6CEC01009729F0A80160E070E00E9436
:10EAE0009075CE01DF91CF911F910F9108959927D5
:10EAF00088270895FC010590061621F00020D9F71B
:10EB0000C00108953197CF010895FC01059061502F
:10EB100070400110D8F7809590958E0F9F1F089533
:10EB2000DC0101C06D9341505040E0F70895FC01B5
:10EB30006150704001900110D8F7809590958E0F2C
:10EB40009F1F0895DC01FC01672F71917723E1F786
:10EB5000329704C07C916D9370836291AE17BF07AA
:10EB6000C8F308950F931F93CF93DF93FB01238185
:10EB700021FD03C08FEF9FEF2CC022FF16C04681FE
:10EB80005781248135814217530744F4A081B18114
:10EB90009D012F5F3F4F318320838C9326813781E6
:10EBA0002F5F3F4F3783268314C08B01EC01FB019D
:10EBB0000084F185E02D1995892BE1F6D801169690
:10EBC0008D919C911797019617969C938E9316970B
:10EBD000CE01DF91CF911F910F910895FB01238109
:10EBE00020FF12C026FD10C08F3F3FEF930761F05A
:10EBF00082832F7D20642383268137812150310930
:10EC000037832683992708958FEF9FEF0895FA01A0
:10EC1000AA27283051F1203181F1E8946F936E7F5B
:10EC20006E5F7F4F8F4F9F4FAF4FB1E03ED0B4E04C
:10EC30003CD0670F781F891F9A1FA11D680F791F8D
:10EC40008A1F911DA11D6A0F711D811D911DA11D9E
:10EC500020D009F468943F912AE0269F11243019AE
:10EC6000305D3193DEF6CF010895462F4770405D49
:10EC70004193B3E00FD0C9F7F6CF462F4F70405DF8
:10EC80004A3318F0495D31FD4052419302D0A9F753
:10EC9000EACFB4E0A6959795879577956795BA954D
:10ECA000C9F700976105710508959B01AC010A2E13
:10ECB00006945795479537952795BA95C9F7620FEA
:10ECC000731F841F951FA01D0895F999FECF92BD53
:10ECD00081BDF89A992780B50895262FF999FECF1E
:10ECE0001FBA92BD81BD20BD0FB6F894FA9AF99A69
:10ECF0000FBE01960895DB018F939F930E94CC76FF
:10ED0000BF91AF91A29F800D911DA39F900DB29FC7
:10ED1000900D11240895A1E21A2EAA1BBB1BFD0120
:10ED20000DC0AA1FBB1FEE1FFF1FA217B307E407EA
:10ED3000F50720F0A21BB30BE40BF50B661F771F42
:10ED4000881F991F1A9469F7609570958095909522
:10ED50009B01AC01BD01CF010895052E97FB1EF468
:10ED600000940E94C47657FD07D00E948B7607FC62
:10ED700003D04EF40C94C47650954095309521956F
:10ED80003F4F4F4F5F4F08959095809570956195D7
:10ED90007F4F8F4F9F4F08950E94DF76A59F900D64
:10EDA000B49F900DA49F800D911D11240895B7FF6D
:10EDB0000C94CC760E94CC76821B930B0895A29F74
:10EDC000B001B39FC001A39F700D811D1124911D3F
:10EDD000B29F700D811D1124911D0895EE0FFF1F2C
:10EDE000881F8BBF0790F691E02D1994692796270D
:10EDF000692778278727782708950E94DF763323AD
:10EE000012F48A1B9B0B0C9407770E94DF76B7FFE6
:10EE10000895821B930B08955058BB27AA270E9480
:10EE200024770C949E780E94907838F00E9497780E
:10EE300020F039F49F3F19F426F40C948D780EF4E9
:10EE4000E095E7FB0C948778E92F0E94AF7858F3A0
:10EE5000BA17620773078407950720F079F4A6F5BF
:10EE60000C94D1780EF4E0950B2EBA2FA02D0B0147
:10EE7000B90190010C01CA01A0011124FF27591BFF
:10EE800099F0593F50F4503E68F11A16F040A22F05
:10EE9000232F342F4427585FF3CF46953795279576
:10EEA000A795F0405395C9F77EF41F16BA0B620B75
:10EEB000730B840BBAF09150A1F0FF0FBB1F661FBC
:10EEC000771F881FC2F70EC0BA0F621F731F841FFF
:10EED00048F4879577956795B795F7959E3F08F025
:10EEE000B0CF9395880F08F09927EE0F97958795E7
:10EEF00008950E94637808F481E008950E94927753
:10EF00000C949E780E94977858F00E94907840F078
:10EF100029F45F3F29F00C94877851110C94D27832
:10EF20000C948D780E94AF7868F39923B1F3552340
:10EF300091F3951B550BBB27AA276217730784070C
:10EF400038F09F5F5F4F220F331F441FAA1FA9F3A2
:10EF500035D00E2E3AF0E0E832D091505040E69590
:10EF6000001CCAF72BD0FE2F29D0660F771F881FF1
:10EF7000BB1F261737074807AB07B0E809F0BB0BE4
:10EF8000802DBF01FF2793585F4F3AF09E3F5105F8
:10EF900078F00C9487780C94D2785F3FE4F3983E35
:10EFA000D4F3869577956795B795F7959F5FC9F7E1
:10EFB000880F911D9695879597F90895E1E0660F62
:10EFC000771F881FBB1F621773078407BA0720F0DB
:10EFD000621B730B840BBA0BEE1F88F7E095089544
:10EFE0000E94F7776894B1110C94D27808950E942A
:10EFF000B77888F09F5798F0B92F9927B751B0F09C
:10F00000E1F0660F771F881F991F1AF0BA95C9F7AC
:10F0100014C0B13091F00E94D178B1E008950C9401
:10F02000D178672F782F8827B85F39F0B93FCCF3B4
:10F03000869577956795B395D9F73EF49095809529
:10F04000709561957F4F8F4F9F4F0895E89409C049
:10F0500097FB3EF490958095709561957F4F8F4F0B
:10F060009F4F9923A9F0F92F96E9BB279395F69521
:10F07000879577956795B795F111F8CFFAF4BB0F9F
:10F0800011F460FF1BC06F5F7F4F8F4F9F4F16C003
:10F09000882311F096E911C0772321F09EE8872F8D
:10F0A000762F05C0662371F096E8862F70E060E049
:10F0B0002AF09A95660F771F881FDAF7880F9695C2
:10F0C000879597F90895990F0008550FAA0BE0E866
:10F0D000FEEF16161706E807F907C0F0121613061A
:10F0E000E407F50798F0621B730B840B950B39F45A
:10F0F0000A2661F0232B242B252B21F408950A26C0
:10F1000009F4A140A6958FEF811D811D089597F9FF
:10F110009F6780E870E060E008959FEF80EC0895BD
:10F1200000240A94161617061806090608950024E6
:10F130000A9412161306140605060895092E039460
:10F14000000C11F4882352F0BB0F40F4BF2B11F4D4
:10F1500060FF04C06F5F7F4F8F4F9F4F089557FD33
:10F160009058440F551F59F05F3F71F04795880F35
:10F1700097FB991F61F09F3F79F0879508951216CC
:10F1800013061406551FF2CF4695F1DF08C0161678
:10F1900017061806991FF1CF869571056105089429
:10F1A0000895E894BB2766277727CB0197F9089540
:10F1B0000E94637808F48FEF08950E94F0780C9411
:10F1C0009E780E94907838F00E94977820F09523DE
:10F1D00011F00C9487780C948D7811240C94D278CB
:10F1E0000E94AF7870F3959FC1F3950F50E0551FC3
:10F1F000629FF001729FBB27F00DB11D639FAA278C
:10F20000F00DB11DAA1F649F6627B00DA11D661FDA
:10F21000829F2227B00DA11D621F739FB00DA11DFB
:10F22000621F839FA00D611D221F749F3327A00DB5
:10F23000611D231F849F600D211D822F762F6A2F51
:10F2400011249F5750409AF0F1F088234AF0EE0FB6
:10F25000FF1FBB1F661F771F881F91505040A9F7E3
:10F260009E3F510580F00C9487780C94D2785F3FD4
:10F27000E4F3983ED4F3869577956795B795F7951F
:10F28000E7959F5FC1F7FE2B880F911D9695879597
:10F2900097F90895FA01EE0FFF1F30962105310509
:10F2A000A1F16115710561F48038BFE39B0749F155
:10F2B00068949038810561F08038BFEF9B0741F07A
:10F2C00099234AF5FF3FE1053105210519F1E8943D
:10F2D0000894E795D901AA2329F4AB2FBE2FF85F34
:10F2E000D0F310C0FF5F70F4A695E0F7F73950F047
:10F2F00019F0FF3A38F49F779F930DD00F9007FCD9
:10F300009058089546F00C948D7860E070E080E8A5
:10F310009FE308954FE79F775F934F933F932F931A
:10F320000E944A7A2F913F914F915F910E94DD7820
:10F330000C94A7790E946378880B990B089529F49F
:10F3400016F00C9487780C94D1780C948D780E94E8
:10F35000B778A8F39638A0F707F80F92E8942BE354
:10F360003AEA48EB5FE70E94F3780F920F920F9210
:10F370004DB75EB70F920E94927AECEFF1E00E94D7
:10F38000D9794F915F91EF91FF91E595EE1FFF1FA6
:10F3900049F0FE57E0684427EE0F441FFA95E1F765
:10F3A0004195550B0E940C7A0F9007FE0C94007A41
:10F3B0000895DF93CF931F930F93FF92EF92DF9205
:10F3C0007B018C01689406C0DA2EEF010E94F07870
:10F3D000FE01E894A5912591359145915591A6F3AB
:10F3E000EF010E942477FE019701A801DA9469F7E2
:10F3F000DF90EF90FF900F911F91CF91DF910895D3
:10F400009B01AC0160E070E080E89FE30C947E77A4
:10F410000C9487780C94C67A0E94B778D8F3992315
:10F42000C9F3940F511DA3F39150504094F059F03B
:10F43000882332F0660F771F881F91505040C1F724
:10F440009E3F51052CF7880F911D9695879597F94A
:10F4500008955F3FACF0983E9CF0BB27869577956A
:10F460006795B79508F4B1609395C1F7BB0F58F74E
:10F4700011F460FFE8CF6F5F7F4F8F4F9F4FE3CF57
:10F480000C94D27816F00C94C67A0C948D7868940B
:10F490000C9487780E94B778A8F39923C1F3AEF350
:10F4A000DF93CF931F930F93FF92C92FDD278823FC
:10F4B0002AF02197660F771F881FDAF720E030E0E7
:10F4C00040E85FEB9FE3883920F0803E38F02196DA
:10F4D0008F770E940D77E4E2F2E004C00E940D777E
:10F4E000E1E5F2E00E94D9798B01BE01EC01FB2E2F
:10F4F0006F5771097595771F880B990B0E942878B3
:10F5000028E132E741E35FE30E94F078AF2D9801F4
:10F51000AE01FF900F911F91CF91DF910E94247750
:10F520000C949E78FA01DC01AA0FBB1F9B01AC0171
:10F53000BF5728F4222733274427507820C0B751DB
:10F5400090F4AB2F0024469537952795011CA39581
:10F55000D2F3002071F0220F331F441FB395DAF36A
:10F560000ED00C940C7761307105A0E88A07B9467B
:10F5700030F49B01AC016627772788279078309676
:10F5800021F0208331834283538308959F3F31F0DC
:10F59000915020F4879577956795B795880F911DC1
:10F5A0009695879597F9089581E090E0F8940C94EA
:10F5B0000F7C0F931F93CF93DF938C01FC0101907D
:10F5C0000020E9F7CF01801B910B0E941C6CEC011D
:10F5D000009719F0B8010E94447BCE01DF91CF91D2
:10F5E0001F910F910895FB01DC0104C08D910190E2
:10F5F000801921F441505040C8F7881B990B089599
:10F600006817790768F4FB01DC01E40FF51FA40F0C
:10F61000B51F02C002900E9241505040D8F7089595
:10F620000C94067CFB01DC018D9181341CF08B3540
:10F630000CF4805E619161341CF06B350CF4605EFB
:10F64000861B611189F3990B0895FB01DC010D9074
:10F650000020E9F7119701900D920020E1F708953D
:10F66000FC018191861721F08823D9F79927089505
:10F670003197CF010895FB01DC018D910190801934
:10F680000110D9F3990B0895FB01DC0101900D9253
:10F690000020E1F70895FB01DC010D900020E9F75F
:10F6A00011974150504028F0019000200D92C9F769
:10F6B00008951C920895FB01DC014150504030F048
:10F6C0008D910190801919F40020B9F7881B990BCE
:10F6D0000895FB01DC014150504048F001900D922B
:10F6E0000020C9F701C01D9241505040E0F7089535
:10F6F0000F931F93CF93DF93CDB7DEB72E970FB63F
:10F70000F894DEBF0FBECDBF0E891F89888D998DFD
:10F7100026E02C831A83098397FF02C080E090E8DB
:10F7200001979E838D83AE01445E5F4F6A8D7B8D12
:10F73000CE0101960E946D704D815E8157FD0AC019
:10F740002F813885421753070CF49A01F801E20F14
:10F75000F31F10822E960FB6F894DEBF0FBECDBFFA
:10F76000DF91CF911F910F9108950F931F93CF9326
:10F77000DF93CDB7DEB72E970FB6F894DEBF0FBE7E
:10F78000CDBF0E891F8986E08C831A8309838FEF92
:10F790009FE79E838D83AE01465E5F4F688D798DB6
:10F7A000CE0101960E946D70EF81F885E00FF11F88
:10F7B00010822E960FB6F894DEBF0FBECDBFDF913C
:10F7C000CF911F910F910895CF93DF93CDB7DEB7FF
:10F7D0002E970FB6F894DEBF0FBECDBF85E08C83A9
:10F7E0008C899D899A838983AE01485E5F4F6E89BB
:10F7F0007F89CE0101960E9436742E960FB6F8943A
:10F80000DEBF0FBECDBFDF91CF910895FB01DC01BC
:10F8100002C001900D9241505040D8F70895F894DD
:02F82000FFCF18
:10F8220003100000C00120000000550B8000010001
:10F83200000000044D515454040000000000000078
:10F8420000000000000000000000000000000000B6
:10F85200000000000000000000000000007131E222
:10F8620058335E6231B0318E31BE3123322E5E00AA
:10F87200000000E931E258335E62312A32E632BEDC
:10F882003123322E5E000000000000000000000064
:10F8920000DF08C21B00000000E931E258335E625B
:10F8A200312A32D632BE3123322E5E000000007F72
:10F8B20059E2580C59CC593D591B592F5900000097
:10F8C20000B548AA48335EDF42A348A0489D4800DD
:10F8D200000000485A255A335E325E0000000023C1
:10F8E2005AE258335E325E235A235A235A000000EA
:10F8F20000235AE258335E325E00000000235A238E
:10F902005A335E235A235A235A235A235A235A23F9
:10F912005A235A235A235A000000001D482949330A
:10F922005E2A430749ED48C648B449C64DE948D85E
:10F9320044714322433F483D481743334800000087
:10F94200006A5A00000000235A01005E0000000015
:10F95200000000E0422B43335EDF42F64234467D34
:10F9620045D6466747CA44D647E64303475D461530
:10F97200460E43FE42FA423031323334353637389E
:10F98200394142434445460000000000A832E25893
:10F99200335E6231FB31B932BE3123322E5E4C6F9F
:10F9A200616465642066726F6D20666C61736820A5
:10F9B20049503A0020444E533A002047573A00201B
:10F9C2004D41534B3A000A4E6F20495020646174F6
:10F9D2006120666F756E6420696E20666C61736863
:10F9E2000A002F0064653A61643A62653A65663AD4
:10F9F20066653A65640068656C70007361766500DF
:10FA02006C6F616400676574006D6163006B696CA3
:10FA12006C007265710069700070776400636C65D8
:10FA22006172007265626F6F74000D0A005F737419
:10FA3200617400560052504D004900737700666CA5
:10FA4200740073657400707772002F616C61726D5F
:10FA52002F736E7372002F616C61726D2F6F7672ED
:10FA62006874002000232532582532582532580068
:10FA72006974656D0073636D640072636D64006523
:10FA82006D6974004F4E004F464600540053003BD0
:10FA9200006E756C6C0066616C73650074727565DE
:10FAA200006E616E00696E66006F76660025783AB8
:10FAB20025783A25783A25783A25783A257825D155
:10FAC20081006D6170002F253032782D253032781B
:10FAD2002D253032782D253032782D253032782D73
:10FAE200253032782E636F6E6669672E6A736F6E89
:10FAF2000022002D002E0025252532780057495A74
:10FB02006E657400726F6F74006F75740062637358
:10FB120074002F726573702F23002F7265712F632B
:10FB22006F6E66003100646D78696E00646D7800F6
:10FB32006D6F64627573006974656D7300746F70C4
:10FB4200696373006D7174740024636F6D6D616E0F
:08FB520064002564002C000092
:00000001FF
